:100000000C94F6170C947E6B0C94536B0C94286B29
:100010000C94FD6A0C94D26A0C94A76A0C947C6AC6
:100020000C94516A0C9422390C9413390C940439B1
:100030000C9427180C9427180C9427180C94271844
:100040000C9427180C94CD6E0C9427180C94271838
:100050000C9427180C9427180C94A8970C94076AF2
:100060000C9427180C94033E0C9427180C94271812
:100070000C9427180C9427180C9427180C94271804
:100080000C9427180C9427180C9427180C942718F4
:100090000C9427180C9427180C9427180C942718E4
:1000A0000C9427180C9427180C9427180C942718D4
:1000B0000C9427180C9427180C9427180C942718C4
:1000C0000C9427180C9427180C9427180C942718B4
:1000D0000C9427180C9427180C9427180C942718A4
:1000E0000C9427181056195623562C563556505630
:1000F0005D5666563E564756A267A5679467986751
:100100009E67DC67A967AD67B367B767BB67C16701
:10011000C567C967DC67CF67D367D7672369286975
:100120002D6937694169BA694B6953695B696569CA
:100130006F69796988699269BA699C69A669B069C9
:10014000084AD73B3BCE016E84BCBFFDC12F3D6C3E
:1001500074319ABD56833DDA3D00C77F11BED9E4A4
:10016000BB4C3E916BAAAABE000000803F05A84C84
:10017000CDB2D44EB93836A9020C50B99186880850
:100180003CA6AAAA2ABE000000803F004E414E496C
:100190004E495459494E46CDCCCC3D0AD7233C1745
:1001A000B7D13877CC2B329595E6241FB14F0A0092
:1001B0000020410000C84200401C4620BCBE4CCA82
:1001C0001B0E5AAEC59D74434F4D4D554E4943418C
:1001D00054494F4E0044525952554E004552524FC9
:1001E000525300494E464F004543484F0020746F1C
:1001F0006F206C6F6E6720657874727573696F6EAF
:100200002070726576656E7465640A0020636F6C99
:100210006420657874727573696F6E20707265768C
:10022000656E7465640A0047322F4733206261644B
:1002300020706172616D65746572730A00536C653C
:1002400065702E2E2E00536E6170707933207265AA
:100250006164792E00436C69636B20746F20726552
:1002600073756D652E2E2E004E6F206D6F76652E88
:10027000002569730025696D20256973002569686B
:100280002025696D2025697300256964202569682A
:100290002025696D20256973002569792025696409
:1002A000202569682025696D2025697300507269D1
:1002B0006E742074696D653A200050726F746563C6
:1002C0007465642050696E0A004525692025730015
:1002D000536E61707079332072656164792E00E825
:1002E00001E301DC01D501C7016F666600444542A8
:1002F00055473A004B494C4C45442E20004D313176
:10030000332053006F6B0048656174696E67206429
:100310006F6E652E0020573A004525692025730031
:10032000536E61707079332072656164792E005369
:100330006E6170707933204F66662E004361703AAB
:10034000454D455247454E43595F504152534552E2
:100350003A300A004361703A434153455F4C494784
:1003600048545F4252494748544E4553533A300A25
:10037000004361703A544F47474C455F4C494748EA
:1003800054533A300A004361703A534F4654574130
:1003900052455F504F5745523A300A004361703A18
:1003A0004C4556454C494E475F444154413A300A0A
:1003B000004361703A5A5F50524F42453A300A004A
:1003C0004361703A4155544F4C4556454C3A300ABA
:1003D000004361703A5052494E545F4A4F423A319D
:1003E0000A004361703A50524F47524553533A30D6
:1003F0000A004361703A4155544F5245504F525490
:100400005F54454D503A310A004361703A454550BA
:10041000524F4D3A310A004649524D574152455FBD
:100420004E414D453A4D61726C696E20312E312E30
:100430003620284769746875622920534F55524306
:10044000455F434F44455F55524C3A68747470732E
:100450003A2F2F6769746875622E636F6D2F4D6137
:10046000726C696E4669726D776172652F4D61724B
:100470006C696E2050524F544F434F4C5F5645525B
:1004800053494F4E3A312E30204D414348494E4555
:100490005F545950453A536E617070793320455816
:1004A0005452554445525F434F554E543A312055AE
:1004B0005549443A63656465326132662D34316171
:1004C000322D343734382D396231322D633535636E
:1004D00036326633363766660A002F2F20007A32AE
:1004E0005F6D696E3A20007A5F6D696E3A2000791F
:1004F0005F6D696E3A2000785F6D696E3A20005238
:1005000065706F7274696E6720656E6473746F7066
:10051000207374617475730A004D31343520533C77
:10052000696E6465783E206F7574206F6620726115
:100530006E67652028302D31290A0053657474696F
:100540006E672054726176656C20416363656C65EB
:10055000726174696F6E3A200053657474696E67D6
:10056000205265747261637420416363656C6572C7
:100570006174696F6E3A200053657474696E672008
:100580005072696E7420416363656C657261746951
:100590006F6E3A200053657474696E6720507269FB
:1005A0006E7420616E642054726176656C204163C4
:1005B00063656C65726174696F6E3A20005A2045FC
:1005C0006E6473746F702041646A7573746D656EC8
:1005D000742073657420746F20286D6D293A002093
:1005E0005A00205900580020204D61783A20002000
:1005F0005A00205900580020204D696E3A20004FC3
:100600006E20004F666600536F667420656E6473DB
:10061000746F70733A2000000136372603FF3C3DAB
:10062000380EFF2E303E1213FF0C0809FFFFFF1A91
:100630001C18FFFF08440AFF4324221EFFFFFFFF90
:10064000FFFF4F666673657473206170706C696537
:1006500064004572723A20546F6F20666172210007
:10066000546F6F206661722066726F6D20726566CE
:100670006572656E636520706F696E740A004E6FF7
:100680002063617365206C696768740A0041637454
:100690006976652045787472756465723A200055F4
:1006A0006E6B6E6F776E20636F6D6D616E643A2056
:1006B00022004E6F204C696E65204E756D6265722A
:1006C000207769746820636865636B73756D2C208F
:1006D0004C617374204C696E653A20004B494C4C58
:1006E00045442E200053544F505045442E20005076
:1006F00072696E7465722073746F707065642064C3
:10070000756520746F206572726F72732E20466952
:100710007820746865206572726F7220616E642043
:10072000757365204D39393920746F207265737483
:100730006172742E202854656D70657261747572D3
:10074000652069732072657365742E20536574206B
:100750006974206166746572207265737461727465
:10076000696E67290A004E6F20436865636B737575
:100770006D2077697468206C696E65206E756D6296
:1007800065722C204C617374204C696E653A2000B0
:10079000636865636B73756D206D69736D617463F8
:1007A000682C204C617374204C696E653A20004CB3
:1007B000696E65204E756D626572206973206E6F7B
:1007C00074204C617374204C696E65204E756D62A7
:1007D00065722B312C204C617374204C696E653A24
:1007E00020004D3131300020496E76616C69642003
:1007F0006578747275646572200000000000000066
:1008000000000000000000004643000046430000D6
:100810005C43202F0020403A00205A3A0020593AE9
:100820000020436F756E7420583A0020453A00202E
:100830005A3A0020593A00583A004B494C4C45442A
:100840002E2000202D20496E76616C696420657829
:10085000747275646572206E756D62657220210A0E
:10086000004572726F723A002020506C616E6E65A6
:100870007242756666657242797465733A2000202B
:1008800046726565204D656D6F72793A2000436F41
:100890006D70696C65643A204665622020312032B3
:1008A0003031380A00207C20417574686F723A201C
:1008B0002852657661724261742C20536E617070AB
:1008C0007920636F6E666967290A00323031372DEF
:1008D00031302D31302031323A303000204C6173CC
:1008E0007420557064617465643A2000312E312E95
:1008F000360A004D61726C696E0020536F66747722
:100900006172652052657365740A002057617463D3
:1009100068646F672052657365740A002042726FC5
:10092000776E206F75742052657365740A002045D8
:10093000787465726E616C2052657365740A00503C
:100940006F77657255700A0073746172740A00459E
:100950006E6473746F707320256320256320256394
:1009600020256300205A3A0020593A0020583A00C6
:10097000656E6473746F7073206869743A200065E3
:1009800063686F3A004261636B004E657874206360
:100990006F726E6572004D34323800507265686552
:1009A000617420504C4100436F6F6C646F776E0030
:1009B0004368616E67652066696C616D656E740081
:1009C00044697361626C65207374657070657273DD
:1009D000004D38340053657420686F6D65206F6674
:1009E0006673657473005072656865617420414276
:1009F00053004C6576656C20636F726E6572730090
:100A0000486F6D65205A00473238205A00486F6D94
:100A100065205900473238205900486F6D652058CD
:100A2000004732382058004175746F20686F6D653B
:100A300000473238004D6F76652061786973004D4C
:100A400061696E004D6F76652058004D6F766520A8
:100A500059004D6F7665205A00457874727564654B
:100A600072004D6F766520302E316D6D004D6F76C2
:100A70006520316D6D004D6F76652031306D6D00F4
:100A80004D6F76652061786973004578747275647E
:100A90006572004D6F7665205A004D6F766520595E
:100AA000004D6F76652058004578747275646572E4
:100AB000004D6F7665205A004D6F76652059004DC8
:100AC0006F76652058005072657061726500496EDE
:100AD000697469616C697A6520454550524F4D00D3
:100AE000436F6E74726F6C00526573746F72652021
:100AF0006661696C73616665004C6F616420736543
:100B00007474696E677300496E697469616C697A9F
:100B10006520454550524F4D0053746F72652073E8
:100B2000657474696E67730046696C616D656E7497
:100B3000004D6F74696F6E0054656D7065726174FD
:100B4000757265004D61696E004D3330332055314B
:100B500020452569205325690050726568656174D8
:100B60002041425320636F6E660050726568656174
:100B70007420504C4120636F6E6600504944204100
:100B800075746F74756E6500504944204175746FBB
:100B900074756E65005049442D44005049442D44FD
:100BA000005049442D49005049442D4900504944C2
:100BB0002D50005049442D50002008204661637498
:100BC0000020082046616374002008204D617800F1
:100BD0002008204D6178002008204D617800200811
:100BE000204D696E002008204D696E002008204DC0
:100BF000696E004F6666004F6E20004175746F7419
:100C0000656D700046616E207370656564004661B5
:100C10006E207370656564004E6F7A7A6C65004E65
:100C20006F7A7A6C6500436F6E74726F6C005374E8
:100C30006F72652073657474696E6773004E6F7AA6
:100C40007A6C65004E6F7A7A6C650046616E20732F
:100C5000706565640046616E20737065656400545C
:100C6000656D70657261747572650020204E6F7AD3
:100C70007A6C653A20006368616E6765006F662074
:100C80007468652066696C616D656E740057616992
:100C90007420666F72207374617274005052494EF2
:100CA00054205041555345440020204E6F7A7A6CB1
:100CB000653A2000200066696C616D656E74207570
:100CC0006E6C6F6164005761697420666F720050CA
:100CD00052494E54205041555345440020204E6FF8
:100CE0007A7A6C653A20002000506C65617365204B
:100CF000776169742E2E2E0048656174696E6720D5
:100D00006E6F7A7A6C65005052494E5420504155AE
:100D10005345440020204E6F7A7A6C653A200020BB
:100D20000068656174206E6F7A7A6C652E0050726F
:100D300065737320627574746F6E20746F00505207
:100D4000494E54205041555345440020204E6F7A5F
:100D50007A6C653A2000746F20636F6E74696E75EB
:100D6000652E2E2E00616E64207072657373206292
:100D70007574746F6E00496E736572742066696C69
:100D8000616D656E74005052494E54205041555368
:100D900045440020204E6F7A7A6C653A200020008E
:100DA00066696C616D656E74206C6F61640057617B
:100DB000697420666F72005052494E54205041555C
:100DC0005345440020204E6F7A7A6C653A2000200B
:100DD0000066696C616D656E742065787472756407
:100DE00065005761697420666F72005052494E5415
:100DF0002050415553454400746F20726573756DE2
:100E000065005761697420666F72207072696E7434
:100E1000005052494E542050415553454400506CA7
:100E200065617365207265736574005052494E5454
:100E300045522048414C544544005072696E7465D7
:100E4000722068616C7465642E206B696C6C282953
:100E50002063616C6C6564210A00656E717565754F
:100E600065696E672022000000000000000000009D
:100E7000000000000048420000484200008040009E
:100E80000000005761726E696E673A20486F6D69A5
:100E90006E672042756D702044697669736F7220A9
:100EA0003C20310A000202040000A0400000A040E3
:100EB00000000040000046430000464300005C4341
:100EC000FFFFFF4D36303020486F74656E6420742C
:100ED0006F6F20636F6C6420746F206368616E674E
:100EE000652066696C616D656E740A004572726F8B
:100EF000722077726974696E6720746F204545505F
:100F0000524F4D210A00290A002062797465733B13
:100F100020637263200053657474696E6773205395
:100F2000746F72656420280000060900FE070192B4
:100F3000032120FFFF08FF07FF000000060000015B
:100F4000070706020080808080800080030202067E
:100F50000105A0A00507070600005050F850F85002
:100F6000500507070600002078A07028F02005072C
:100F700007060000C0C810204098180507070600A3
:100F8000006090A040A89068020303060104C040DE
:100F9000800307070601002040808080402003076F
:100FA000070601008040202020408005050506003E
:100FB0000120A870A8200505050600012020F820C2
:100FC000200203030602FFC0408005010106000362
:100FD000F8020202060200C0C0050505060001086D
:100FE00010204080050707060000708888888888E0
:100FF0007003070706010040C040404040E005077D
:1010000007060000708808708080F8050707060052
:1010100000F81020100808F005070706000010303F
:101020005090F81010050707060000F880F0080837
:101030008870050707060000708080F088887005BA
:101040000707060000F808102020202005070706E3
:101050000000708888708888700507070600007097
:10106000888878080870020505060200C0C000C024
:10107000C00206060602FFC0C000C0408004070789
:1010800006000010204080402010050303060002E7
:10109000F800F80407070601008040201020408077
:1010A00005070706000070880810200020050707C4
:1010B00006000070880868A8A870050707060000E9
:1010C000708888F8888888050707060000F08888F7
:1010D000F08888F005070706000070888080808807
:1010E00070050707060000F08888888888F00507E3
:1010F00007060000F88080F08080F80507070600EA
:1011000000F88080F0808080050707060000708866
:1011100080B8888870050707060000888888F888E6
:101120008888010707060200808080808080800513
:10113000070706000038101010109060050707061A
:1011400000008890A0C0A0908805070706000080D6
:101150008080808080F805070706000088D8A8886E
:101160008888880507070600008888C8A8988888A6
:1011700005070706000070888888888870050707BB
:10118000060000F08888F0808080050707060000D0
:1011900070888888A89068050707060000F088888E
:1011A000F0A0908805070706000078808070080886
:1011B000F0050707060000F8202020202020050762
:1011C0000706000088888888888870050707060059
:1011D00000888888888850200507070600008888CE
:1011E000888888A850050707060000888850205086
:1011F0008888050707060000888888502020200579
:101200000707060000F80810204080F803070706CB
:101210000100E08080808080E005050506000180F7
:1012200040201008030707060100E02020202020AE
:10123000E0050303060004205088050101060000B4
:10124000F80202020602058040050505060000704E
:10125000087888780507070600008080B0C888886D
:10126000F0050505060000708080887005070706F8
:101270000000080868988888780505050600007051
:1012800088F880700507070600003048E0404040BD
:10129000400506060600FF70888878087005070775
:1012A0000600008080B0C888888801070706020011
:1012B000800080808080800308080601FF200020D5
:1012C000202020A040040707060000808090A0C0D6
:1012D000A090030707060100C04040404040E005E1
:1012E0000505060000D0A8A8A8A805050506000069
:1012F000B0C8888888050505060000708888887051
:101300000506060600FFF08888F0808005060606C0
:1013100000FF788888780808050505060000B0C831
:1013200080808005050506000070807008F00407C5
:10133000070600004040E04040403005050506003B
:101340000088888898680505050600008888885008
:10135000200505050600008888A8A8500505050693
:10136000000088502050880506060600FF888888FF
:10137000780870050505060000F8102040F80307FE
:101380000706010020404080404020010707060278
:1013900000808080808080800307070601008040F5
:1013A00040204040800502020600026890000000D4
:1013B000060000000000060000000000060000001B
:1013C000000006000000000006000000000006000B
:1013D0000000000006000000000006000000000001
:1013E00006000000000006000000000006000000EB
:1013F00000000600000000000600000000000600DB
:1014000000000000060000000000060000000000D0
:1014100006000000000006000000000006000000BA
:1014200000000600000000000600000000000600AA
:1014300000000000060000000000060000000000A0
:10144000060000000000060000000000060000008A
:10145000000006000000000006000000000006007A
:101460000000000006000000000006000000000070
:1014700006000000000006000001070706020080C9
:101480000080808080800507070600002070A8A0EB
:10149000A87020050707060000304040E04050A833
:1014A00005050506000088705070880507070600CE
:1014B00000885020F820F8200107070602008080ED
:1014C00080008080800508080600003048205050C9
:1014D000209060030101060107A005070706000030
:1014E000F888B8B8B888F8050707060001700878CA
:1014F000887800F80505050600012850A050280549
:101500000303060001F808080202020602064080F2
:10151000050707060000F888A88898A8F8050101C3
:10152000060006F8040404060003609090600507B6
:10153000070600002020F8202000F804050506001A
:101540000360902040F0030505060003E020E02042
:10155000E002020206020640800508080600FF8835
:1015600088888898E88080050707060000789898A2
:1015700078181818020202060202C0C0020202060F
:1015800002FF408003050506000340C04040E0051F
:101590000707060001708888887000F805050506B1
:1015A0000001A0502850A00507070600008890A859
:1015B00058B808080507070600008890B848982022
:1015C00038050808060000C040C048D8380808059B
:1015D00007070600002000204080887005080806E4
:1015E00000004020007088F8888805080806000080
:1015F0001020007088F88888050808060000205030
:10160000007088F888880508080600006890007057
:1016100088F888880508080600005000708888F857
:1016200088880508080600002050207088F88888FF
:101630000507070600003860A0B8E0A0B805080854
:101640000600FF708880808870206005080806000A
:1016500000402000F880F080F80508080600000827
:101660001000F880F080F8050808060000205000FF
:10167000F880F080F80507070600005000F880F0B9
:1016800080F8030808060100804000E0404040E088
:10169000030808060100204000E0404040E0030845
:1016A0000806010040A000E0404040E003070706B4
:1016B0000100A000E0404040E00507070600007080
:1016C0004848E84848700508080600006890008807
:1016D000C8A89888050808060000402070888888F7
:1016E00088700508080600001020708888888870B7
:1016F00005080806000020500070888888700508DA
:101700000806000068900070888888700508080640
:101710000000500070888888887005050506000163
:1017200088502050880508080600FF1070A8A8A857
:10173000A87040050808060000402088888888882E
:1017400070050808060000102088888888887005C1
:10175000080806000020500088888888700508085E
:1017600006000050008888888888700508080600F0
:101770000010208850202020200509090600FFC005
:1017800040704848704040E00408080601FF60903F
:1017900090A09090E08005080806000040200070AE
:1017A000087888780508080600001020007008787E
:1017B00088780508080600002050007008788878AE
:1017C000050808060000689000700878887805070A
:1017D00007060000500070087888780508080600A1
:1017E000002050207008788878050606060000D092
:1017F0002878A0A8500506060600FF708088702093
:10180000600508080600004020007088F880700518
:1018100008080600001020007088F880700508088D
:101820000600002050007088F88070050707060049
:101830000050007088F8807003080806010080409E
:101840000040C04040E0030808060100204000407E
:10185000C04040E003080806010040A00040C0402E
:1018600040E0030707060100A00040C04040E0053B
:101870000707060000A040A0107888700508080639
:101880000000689000B0C888888805080806000035
:101890004020007088888870050808060000102025
:1018A00000708888887005080806000020500070C5
:1018B000888888700508080600006890007088888D
:1018C000887005070706000050007088888870053A
:1018D00005050600012000F800200507070600FFA7
:1018E0001070A8A8A8704005080806000040200055
:1018F00088888898680508080600001020008888F5
:101900008898680508080600002050008888889894
:101910006805070706000050008888889868050950
:10192000090600FF102000888888F808700407075F
:101930000601FFC04060506040E00508080600FF57
:101940005000888888780870000021002400270053
:101950002A002D00300033000101000004010701BE
:101960000A0100002200250028002B002E00310073
:10197000340002010000050108010B0100002000F5
:101980002300260029002C002F0032000001000057
:1019900003010601090105050505070508080808F2
:1019A000020202020A0A08080404040401010101F7
:1019B00001010101030303030303030304070707F2
:1019C0000C0C0C0C0C0C0C0C020202020606060697
:1019D000060606060B0B0B0B0B0B0B0B0102102064
:1019E0002008081020401020408002010201080455
:1019F00002010102040810204080804020100804E9
:101A00000201800402018040201008040201080441
:101A10000201010204081020408001020408102085
:101A2000408000000A0B02090C0D0E080703040198
:101A300000000000000000000000000000000000A6
:101A40000000000000000000000000000000121173
:101A50001000000000000000000000000000000076
:101A6000000000000000000024F4D43050C38E2099
:101A7000C2A24017828B7011127A910D816CD90A23
:101A8000A861E108C7586607615143061E4B5D0512
:101A9000C145A7041A411104093D98037139310366
:101AA0004036DB0265339102D4305402802E1D0291
:101AB000632CEE01752AC501B028A0011027810111
:101AC0008F2564012B244B01E0223401AC211F013E
:101AD0008D200D01801FFC00841EED00971DDF008E
:101AE000B81CD200E61BC600201BBC00641AB20062
:101AF000B219A8000A19A0006A189900D11791001C
:101B000040178B00B516840031167E00B31579009E
:101B10003A157300C7146F0058146A00EE1366007C
:101B20008813630025135E00C7125B006C12570018
:101B300015125400C111510070114F0021114B00BA
:101B4000D61049008D104700461044000210420094
:101B5000C00F4000800F3E00420F3C00060F3B00CC
:101B6000CB0E3800930E37005C0E3500270E340084
:101B7000F30D3200C10D3100900D3000600D2E00CC
:101B8000320D2D00050D2C00D90C2B00AE0C2900B8
:101B9000850C29005C0C2700350C27000E0C260054
:101BA000E80B2400C40B2400A00B23007D0B2300B2
:101BB0005A0B2100390B2100180B2000F80A1F00D6
:101BC000D90A1E00BB0A1E009D0A1D00800A1D00C6
:101BD000630A1C00470A1B002C0A1B00110A1A008A
:101BE000F7091A00DD091900C4091900AB09190029
:101BF000920917007B091800630917004C091600A9
:101C000036091600200916000A091500F508150006
:101C1000E0081400CC081400B8081400A40814004C
:101C2000900813007D0812006B081300580812007A
:101C30004608120034081100230811001208110090
:101C400001081100F0071000E0071000D007100095
:101C5000C0071000B0070F00A107100091070E0089
:101C600083070F0074070F0065070E0057070E006B
:101C700049070E003B070D002E070E0020070D0040
:101C800013070D0006070D00F9060C00ED060D0008
:101C9000E0060C00D4060C00C8060C00BC060C00C4
:101CA000B0060C00A4060B0099060C008D060B0074
:101CB00082060B0077060B006C060B0061060A001B
:101CC00057060B004C060A0042060A0038060A00B6
:101CD0002E060A0024060A001A060A001006090049
:101CE00007060A00FD050900F4050900EB050900D7
:101CF000E2050900D9050900D0050900C70509005A
:101D0000BE050900B5050800AD050800A5050900D8
:101D10009C050800940508008C050800840508004F
:101D20007C050800740508006C05070065050800BF
:101D30005D050700560508004E050700470507002A
:101D40004005080038050700310507002A0507008F
:101D5000230507001C050600160507000F050700F0
:101D60000805060002050700FB040600F50407004D
:101D7000EE040600E8040600E2040700DB040600A7
:101D8000D5040600CF040600C9040600C3040600FB
:101D9000BD040600B7040600B1040500AC0406004B
:101DA000A6040600A00405009B0406009504050097
:101DB000900406008A0405008504050080040600DE
:101DC0007A04050075040500700405006B04050025
:101DD00066040500610405005C0405005704050065
:101DE000520405004D0405004804050043040500A5
:101DF0003E0404003A0405003504050030040400E4
:101E00002C04050027040400230405001E0404001C
:101E10001A04040016040500110404000D04040053
:101E2000090405000404040000040400FC03040089
:101E3000F8030400F4030400F0030400EC030400BE
:101E4000E8030400E4030400E0030400DC030400EE
:101E5000D8030400D4030400D0030400CC0304001E
:101E6000C8030300C503030024F404D9201BC40CD9
:101E70005C0E9804C4095F0265077101F405F9005E
:101E8000FB04B30048048700C103690058035500F0
:101E900003034500BE023A008402310053022A00C7
:101EA0002902250004022000E4011C00C8011900D9
:101EB000AF01170098011400840113007101100094
:101EC0006101100051010E0043010D0036010B00AD
:101ED0002B010B0020010B00150109000C0109006A
:101EE00003010800FB000800F3000800EB000700F6
:101EF000E4000600DE000600D8000600D20006005E
:101F0000CC000500C7000500C2000500BD000400AC
:101F1000B9000400B5000400B1000400AD000400E5
:101F2000A9000400A5000300A20003009F00040014
:101F30009B0003009800030095000200930003003B
:101F4000900003008D0002008B0003008800020057
:101F50008600020084000300810002007F0002006E
:101F60007D0002007B000200790002007700010082
:101F7000760002007400020072000100710002008D
:101F80006F0002006D0001006C0002006A00010099
:101F900069000200670001006600010065000100A1
:101FA00064000200620001006100010060000100A5
:101FB0005F0002005D0001005C0001005B000100A9
:101FC0005A000100590001005800010057000100AB
:101FD00056000100550001005400010053000000AC
:101FE00053000100520001005100010050000100A7
:101FF0004F0001004E0000004E0001004D000100A6
:102000004C0001004B0000004B0001004A000100A1
:10201000490001004800000048000100470001009D
:102020004600000046000100450000004500010098
:102030004400010043000000430001004200000092
:102040004200010041000000410001004000010089
:102050003F0000003F0001003E0000003E00010084
:102060003D0000003D0001003C0000003C0000007D
:102070003C0001003B0000003B0001003A00000072
:102080003A0001003900000039000100380000006A
:102090003800000038000100370000003700010060
:1020A0003600000036000000360001003500000058
:1020B000350000003500010034000000340000004D
:1020C0003400010033000000330000003300010041
:1020D0003200000032000000320001003100000038
:1020E000310000003100010030000000300000002D
:1020F000300001002F0000002F0000002F00000022
:102100002F0001002E0000002E0000002E00010014
:102110002D0000002D0000002D0000002D0001000A
:102120002C0000002C0000002C0000002C000100FE
:102130002B0000002B0000002B0000002B000100F2
:102140002A0000002A0000002A0000002A000100E6
:1021500029000000290000002900000029000000DB
:1021600029000100280000002800000028000000CD
:1021700028000000280001002700000027000000C0
:1021800027000000270000002700010026000000B3
:1021900026000000260000002600000026000100A6
:1021A000250000002500000025000000250000009B
:1021B000250000002500010024000000240000008C
:1021C000240000002400000024000100230000007F
:1021D0002300000023000000230000002300000073
:1021E0002300000023000100220000002200000064
:1021F0002200000022000000220000002200010056
:10220000210000002100000021000000210000004A
:10221000210000002100000021000100200000003A
:10222000200000002000000020000000200000002E
:102230002000000020000000200001001F0000001E
:102240001F0000001F0000001F0000001F00000012
:102250001F0000001F0001001E0000001E00000003
:102260001E0000001E000000544845524D414C2005
:1022700052554E4157415900546865726D616C204A
:1022800052756E617761790056652D6A65726B00D3
:1022900056652D6A65726B0056652D6A65726B0016
:1022A000567A2D6A65726B00567A2D6A65726B00DC
:1022B00056792D6A65726B0056792D6A65726B00CE
:1022C00056792D6A65726B0056782D6A65726B00BF
:1022D00056782D6A65726B0056782D6A65726B00B0
:1022E0004D6F74696F6E004573746570732F6D6DFB
:1022F000004573746570732F6D6D005A737465704B
:10230000732F6D6D005A73746570732F6D6D005966
:1023100073746570732F6D6D005973746570732FCE
:102320006D6D005873746570732F6D6D0058737404
:102330006570732F6D6D004D6F74696F6E0053740F
:102340006570732F6D6D004A65726B004163636544
:102350006C65726174696F6E0056656C6F63697449
:102360007900436F6E74726F6C0046696C2E204466
:1023700069612E0046696C2E204469612E004F660B
:1023800066004F6E20004520696E206D6D3300435E
:102390006F6E74726F6C0020204E6F7A7A6C653AA3
:1023A000200020004261636B004D696E696D756DA0
:1023B0002054656D70206973203137302E004865D8
:1023C0006174696E67206661696C65640045787444
:1023D00072756465206D6F726500526573756D6509
:1023E000207072696E7400524553554D45204F5010
:1023F00054494F4E533A0020746F6F206C6F6E67D4
:1024000020657874727573696F6E20707265766579
:102410006E7465640A0020636F6C64206578747262
:102420007573696F6E2070726576656E7465640A87
:102430000000060900FE000000000001090008FE7F
:10244000000005080806000040F0C8888898781049
:10245000050808060000C0F88888888888F80505FF
:10246000050600012030F83020050808060000208D
:1024700070F820202020E00509090600FF2070A840
:10248000A8B8888870200509090600FFE080C0B060
:10249000A8283028280509090600FFF8A888888898
:1024A0008888A8F8050A0A0600FE20505050508877
:1024B000A8A8887003030306000340A0405A0059EF
:1024C000005800092000000000000000000000008B
:1024D00000007FFFE000000000000000000000009E
:1024E000007000E00000000000000000000000009C
:1024F00061F86000000000000000000000000041E2
:10250000F82000000000000000000000000040F083
:1025100020000000000000000000000000406020DB
:102520000000000000000000000000005801A07F33
:1025300080000000000000000000005C63A0FFC0FD
:10254000000000000000000000005EF7A0FFC000D7
:102550000000000000000000005EF7A0FFC00000C7
:1025600000000000000000005C63A07F800000000D
:10257000000000000000005801A07F800000000063
:10258000000000000000406020FFC00000000000CC
:10259000000000000040F020FFC00000000000002C
:1025A0000000000041F820FFC00000000000000013
:1025B00000000061F8603F00000000000000000023
:1025C00000007000E01E000000000000000000009D
:1025D000007FFFE00C000000000000000000000091
:1025E0000000000000000000000000000000007F6C
:1025F000FFE000000000000000000000000070008C
:10260000E0000000000000000000000000630C601B
:10261000000000000000000000000000470E200045
:1026200000000000000000000000004F0F2000002C
:10263000000000000000000000005F0FA00000008C
:102640000000000000000000005E07A07F80000086
:102650000000000000000000406020FFC0000000FB
:102660000000000000000040F020FFC0000000005B
:1026700000000000000040F020FFC000000000004B
:1026800000000000004060207F800000000000008B
:10269000000000005E07A07F800000000000000036
:1026A0000000005F0FA0FFC000000000000000005D
:1026B00000004F0F20FFC0000000000000000000DD
:1026C00000470E20FFC000000000000000000000D6
:1026D000630C603F0000000000000000000000707C
:1026E00000E01E00000000000000000000007FFF6E
:1026F000E00C0000000000000000000000000000EE
:1027000070012C0190012701B0012201C0011D01BF
:10271000F00118011002130130020E0160020901DC
:1027200090020401C002FF000003FA004003F5001C
:102730008003F000D003EB002004E6007004E10009
:10274000E004DC004005D700C005D2004006CD0003
:10275000D006C8008007C3003008BE00F008B900EA
:10276000C009B400B00AAF00B00BAA00D00CA5009D
:10277000000EA000500F9B00C01096005012910058
:1027800000148C00C0158700B0178200B0197D00BE
:10279000D01B7800001E730040206E00902269005C
:1027A000F024640040275F0090295A00E02B550078
:1027B000102E500020304B0010324600E033410014
:1027C00090353C001037370070383200A0392D00AA
:1027D000B03A2800A03B2300603C1E00103D1900C9
:1027E000903D1400103E0F00703E0A00C03E0500F0
:1027F000003F0000403FFBFF803FF6FFC03FF1FF7E
:102800006265640A002C2073797374656D2073749B
:102810006F7070656421204865617465725F49441A
:102820003A200048656174696E67206661696C656D
:10283000640048656174696E67206661696C6564EF
:10284000004572723A204D494E54454D50004D4955
:102850004E54454D50207472696767657265640017
:102860004572723A204D415854454D50004D4158E3
:1028700054454D5020747269676765726564002025
:10288000440020490020204D333031205000504971
:10289000442073657474696E67733A0A00204600B9
:1028A00020420020480020204D3134352053004D77
:1028B0006174657269616C206865617475702070FF
:1028C0006172616D65746572733A0A0020204D363D
:1028D0003636205A005A3220456E6473746F702069
:1028E00061646A7573746D656E743A0A00205A00EB
:1028F00020590020204D323036205800486F6D6539
:10290000206F66667365743A0A00204500205A00FD
:1029100020590020580020420020540020204D3231
:102920003035205300416476616E6365643A20530C
:102930003C6D696E5F66656564726174653E2054C6
:102940003C6D696E5F74726176656C5F6665656427
:10295000726174653E20423C6D696E5F7365676DA0
:10296000656E745F74696D655F6D733E20583C6D74
:1029700061785F78795F6A65726B3E205A3C6D6161
:10298000785F7A5F6A65726B3E20453C6D61785F67
:10299000655F6A65726B3E0A002054002052002079
:1029A000204D323034205000416363656C657261A4
:1029B00074696F6E2028756E6974732F7332293AAB
:1029C00020503C7072696E745F616363656C3E2079
:1029D000523C726574726163745F616363656C3EDF
:1029E00020543C74726176656C5F616363656C3E14
:1029F0000A00204500205A0020590020204D323086
:102A0000312058004D6178696D756D2041636365B3
:102A10006C65726174696F6E2028756E6974732FAE
:102A20007332293A0A00204500205A00205900201C
:102A3000204D3230332058004D6178696D756D201E
:102A40006665656472617465732028756E69747358
:102A50002F73293A0A00204500205A0020590020EF
:102A6000204D3932205800537465707320706572A0
:102A700020756E69743A0A0020204D3230302044AF
:102A8000300A0020204D3230302044002044697349
:102A900061626C65640A0046696C616D656E7420E4
:102AA00073657474696E67733A0020204D31343950
:102AB0002043203B20556E69747320696E20436566
:102AC0006C736975730A0020204732312020202062
:102AD0003B20556E69747320696E206D6D0A001F6E
:102AE000FFFFFFFFFFFF600000000001FF4000004C
:102AF000000000FF8000000000007F83CF00000C7A
:102B0000303F87FF80000C301F867980000C000F5B
:102B10008C30C7838C30E78C30CFC7CC31F38C300E
:102B2000DCECEC33B98C30D86C6C33198C30D06C55
:102B30000C33198C30D86C0C33198C30DC6C0E3B98
:102B4000198C30CF7C079F198C30C77C038F1940BC
:102B5000000000000002600000000000061FFFFFF0
:102B6000FFFFFFF8202863616C63756C6174656416
:102B700029210A0020213D2000454550524F4D207B
:102B8000435243206D69736D61746368202D202862
:102B900073746F726564292000290A0020627974B9
:102BA00065733B2063726320002073746F726564E9
:102BB0002073657474696E677320726574726965D9
:102BC000766564202800204D61726C696E3D563434
:102BD00031290A0028454550524F4D3D004545508A
:102BE000524F4D2076657273696F6E206D69736DFB
:102BF00061746368200048617264636F6465642077
:102C000044656661756C742053657474696E67738E
:102C1000204C6F616465640A00E8030000E803006B
:102C2000000A0000001027000000001643000016F4
:102C3000430000A0400000C84100002042000020E6
:102C4000420000C8430000C04220643A0020693AB4
:102C50000020703A0043290A0061626C65642028F4
:102C60006D696E2074656D702000436F6C64206523
:102C700078747275646573206172652000236465E1
:102C800066696E65202044454641554C545F4B644F
:102C9000200023646566696E6520204445464155E1
:102CA0004C545F4B69200023646566696E65202083
:102CB00044454641554C545F4B70200050494420D8
:102CC0004175746F74756E652066696E69736865A9
:102CD00064212050757420746865206C61737420C1
:102CE0004B702C204B6920616E64204B6420636F15
:102CF0006E7374616E74732066726F6D2062656CA2
:102D00006F7720696E746F20436F6E6669677572A6
:102D10006174696F6E2E680A0050494420417574D1
:102D20006F74756E65206661696C656421207469D5
:102D30006D656F75740A00504944204175746F7455
:102D4000756E65206661696C6564212054656D70DF
:102D50006572617475726520746F6F206869676849
:102D60000A00204B643A2000204B693A2000204B97
:102D7000703A20000A20436C6173736963205049E4
:102D800044200A002054753A2000204B753A200058
:102D9000206D61783A2000206D696E3A2000206431
:102DA0003A200020626961733A20005654726176BD
:102DB000206D696E005654726176206D696E005602
:102DC00054726176206D696E00566D696E00566DA5
:102DD000696E00566D696E00566D6178204500562B
:102DE0006D6178204500566D6178204500566D6113
:102DF00078205A00566D6178205A00566D6178200F
:102E00005A00566D6178205900566D61782059003E
:102E1000566D6178205900566D6178205800566DC6
:102E20006178205800566D61782058004D6F7469A4
:102E30006F6E00416D6178204500416D61782045DD
:102E400000416D6178205A00416D6178205A00413F
:102E50006D6178205900416D6178205900416D61A4
:102E600078205800416D6178205800412D747261BE
:102E700076656C00412D74726176656C00412D722F
:102E800065747261637400412D726574726163745C
:102E900000416363656C00416363656C004D6F7452
:102EA000696F6E00436F6E74726F6C005072657064
:102EB0006172650054756E6500496E666F207363BC
:102EC0007265656E004261627973746570205A00A4
:102ED0004D363030204230004368616E67652066B1
:102EE000696C616D656E74004261627973746570BE
:102EF000205A00466C6F7700466C6F770046616E13
:102F00002073706565640046616E2073706565644A
:102F1000004E6F7A7A6C65004E6F7A7A6C6500535A
:102F200070656564005370656564004D61696E008D
:102F3000526573656E643A20006F6B006275737939
:102F40003A2070617573656420666F7220696E70D7
:102F500075740A00627573793A20706175736564DF
:102F600020666F7220757365720A00627573793A14
:102F70002070726F63657373696E670A004B494C0A
:102F80004C45442E20004B494C4C206361757365C1
:102F900064206279204B494C4C20627574746F6ECA
:102FA0002F70696E0A004B494C4C45442E20004B53
:102FB000494C4C2063617573656420627920746F9D
:102FC0006F206D75636820696E6163746976652032
:102FD00074696D65202D2063757272656E7420634F
:102FE0006F6D6D616E643A20000085C211241FBEB2
:102FF000CFEFD1E2DEBFCDBF00E00CBF13E0A0E019
:10300000B2E0EEE8F2EA01E00BBF02C007900D92D9
:10301000AE3AB107D9F72FE0AEEAB3E001C01D9296
:10302000A936B207E1F717E1C6EFD7E100E006C025
:1030300021970109802FFE010E94FBD0C53FD107D7
:1030400080E00807A9F70E9498BB0C9445D10C9426
:1030500000002F923F924F925F926F927F928F92D9
:103060009F92AF92BF92CF92DF92EF92FF920F9317
:103070001F93CF93DF93CDB7DEB7C759D1090FB6F2
:10308000F894DEBF0FBECDBF0091010620E6029F7F
:10309000800111240E521C4F8091BB0E80FF1AC07C
:1030A000EFE7F9E084917F013FEFE31AF30A811122
:1030B00002C0780104C00E94593AF701F3CFD7014A
:1030C0008D917D01882319F00E94593AF8CF8AE04A
:1030D0000E94593A81E090E090937F0680937E06AB
:1030E00010925905109258058FE380935C05109259
:1030F0005B0510925A051092C8031092C9031092F2
:10310000CA031092CB03F80180810F5F1F4F8032FA
:10311000D1F38E34B1F4818190ED980F9A3020F084
:103120008D3211F08B3269F43296DF0131962C9199
:1031300020532A30D0F3CD01FC01019620812032AA
:10314000D9F3F0934E0FE0934D0F7F01BFEFEB1AD1
:10315000FB0A10816AE270E0C7010E940DD100975E
:1031600031F0FC01319780818032E1F311821D340E
:1031700029F0143519F0173409F0CEC0F701808119
:103180002FEFE21AF20A8032C9F380538A3008F036
:10319000C3C010935C0520915A0530915B054AE04D
:1031A0003196429FC001439F900D1124DF0111977A
:1031B0002C91022E000C330B20533109280F391F9C
:1031C000808180538A3060F330935B0520935A05E9
:1031D000DF0131968C918032D9F31D3451F000918A
:1031E0004D0F609158057091590588248394912C56
:1031F00055C02E31310591F03CF42731310571F085
:103200002C31310561F70AC02537310544F32737E2
:10321000310524F0203A43E0340709F7B09359050B
:10322000A093580579C0413209F442C0EFEBE40F96
:10323000EA3108F05DC0DC017D015D915032E1F3BF
:10324000C701A0EDA50FAA3008F046C0DC01EE2EA4
:10325000F12C6701F3E0D594C794FA95E1F7A60144
:1032600048535C4F6A014E2F4770F40102C0EE0FC5
:10327000FF1F4A95E2F7AF01F6015081452B4083CD
:103280001097A1F1A01BA70142555C4FFA01A08342
:10329000DC014C9141544A3180F5DC01CD010196AD
:1032A0004C914111C0CF709359056093580534C0BB
:1032B0001D3409F0BBCF2032310509F0B7CF909310
:1032C00059058093580563E270E00E940DD1009784
:1032D00019F1DC011C9220C0A3EDA50FA23008F467
:1032E000B5CF5B3211F00C94EA32B0CFA0E0CBCF77
:1032F0006115710569F6BD01CBCFAD011196FA01DB
:10330000908190539A30C8F3CA014F5F5F4FFC0120
:10331000A081A032C9F3C1CF80915C058D3411F436
:103320000C940726843511F40C949132873411F0F3
:103330000C94CC3280915A0590915B0584309105B4
:1033400009F41FC65CF497FF02C00C94E33220918D
:103350007F02823091050CF00DC11CC08A359105A9
:1033600011F40C94792554F48530910509F450C674
:103370004C9711F40C94C2240C94E3328B359105D4
:1033800011F40C947D258C35910511F40C94822553
:103390000C94E332222311F40C94E3320E94DF39BF
:1033A0008EE696E00E945CB70E944E3A8091BB0E7A
:1033B00083FD8FC0C0907A06D0907B06E0907C069B
:1033C000F0907D062091F20B3091F30B4091F40BBD
:1033D0005091F50BC701B6010E94DDC9882309F49D
:1033E00078C080911606811138C0609119027091E1
:1033F0001A02072E000C880B990B0E94E3C99B014F
:10340000AC016091120670911306809114069091A0
:1034100015060E94DDC987FF20C0C092F20BD09232
:10342000F30BE092F40BF092F50BEFE7F9E08491E7
:103430008F010F5F1F4F882321F00E94593AF80136
:10344000F6CFECE0F2E084918F010F5F1F4F8823ED
:1034500021F00E94593AF801F6CFC0907A06D09038
:103460007B06E0907C06F0907D062091F20B309177
:10347000F30B4091F40B5091F50BC701B6010E947C
:10348000F3CD20E030E048E453E40E941AD018164F
:1034900004F5C092F20BD092F30BE092F40BF09291
:1034A000F50BEFE7F9E084918F010F5F1F4F882341
:1034B00021F00E94593AF801F6CFEDEEF1E0849147
:1034C0008F010F5F1F4F882321F00E94593AF801A6
:1034D000F6CF20916E0630916F06409170065091A4
:1034E00071066091E60B7091E70B8091E80B90916B
:1034F000E90B0E94DDC981111DC020917206309137
:10350000730640917406509175066091EA0B7091B4
:10351000EB0B8091EC0B9091ED0B0E94DDC98111BA
:1035200009C06091000270910102809102029091A5
:1035300003021AC06091990270919A02072E000C42
:10354000880B990B0E94E3C920910002309101027F
:1035500040910202509103020E9442CA2AE037EDD4
:1035600043E25CE30E9442CA0E9490370E94863781
:103570000C94E332222311F40C94E33211E002970D
:1035800009F010E00E94DF3982E50E94D3398823D8
:1035900009F43CC10E9471396B017C014090E60B3B
:1035A0005090E70B6090E80B7090E90B2091EA0BCC
:1035B0003091EB0B4091EC0B5091ED0B2EA73FA7F8
:1035C00048AB59AB80916E0690916F06A091700642
:1035D000B09171068AAB9BABACABBDAB20917206D0
:1035E0003091730640917406509175062AAF3BAF37
:1035F0004CAF5DAF20E030E0A901C701B6010E94E9
:10360000DDC9882309F4A3C4A30192016AA97BA997
:103610008CA99DA90E94DDC981110DC02EA53FA5D1
:1036200048A959A96AAD7BAD8CAD9DAD0E94DDC99D
:10363000882309F48CC420E030E0A901C701B60159
:103640000E94DDC9881F8827881F18130BC080E0DF
:1036500090E0A0E8BFE32A968CAF9DAFAEAFBFAFBE
:103660002A970AC020E030E040E85FEB2A962CAFB2
:103670003DAF4EAF5FAF2A97A30192016AA97BA924
:103680008CA99DA90E94F3CD22966CAF7DAF8EAF21
:103690009FAF22972EA53FA548A959A96AAD7BAD3A
:1036A0008CAD9DAD0E94F3CD26966CAF7DAF8EAFF5
:1036B0009FAF269722962CAD3DAD4EAD5FAD2297C4
:1036C000CA01B9010E9442CA4B015C0126962CAD89
:1036D0003DAD4EAD5FAD2697CA01B9010E9442CA09
:1036E0009B01AC01C501B4010E94F4CD0E945FD0E2
:1036F0006EAB7FAB88AF99AF20E030E040E05FE396
:103700000E9442CA4B015C01A7019601C701B601A4
:103710000E9442CA6B017C01A5019401C501B4015C
:103720000E9442CA9B01AC01C701B6010E94F3CDC1
:103730000E945FD09B01AC012A966CAD7DAD8EAD31
:103740009FAD2A970E9442CA4B015C012AA93BA95E
:103750004CA95DA9C301B2010E94F4CD20E030E084
:1037600040E05FE30E9442CA6B017C0126966CAD8B
:103770007DAD8EAD9FAD269790582EA93FA948AD3F
:1037800059AD0E94D0CE9B01AC01C501B4010E948D
:1037900042CA9B01AC01C701B6010E94F4CDA3014E
:1037A00092010E94F3CD6B017C012AAD3BAD4CAD83
:1037B0005DAD6EA57FA588A999A90E94F4CD20E0F2
:1037C00030E040E05FE30E9442CA2B013C012EA999
:1037D0003FA948AD59AD22966CAD7DAD8EAD9FAD84
:1037E00022970E94D0CE9B01AC01C501B4010E947A
:1037F00042CA9B01AC01C301B2010E94F4CD2EA5C7
:103800003FA548A959A90E94F3CD14C089E40E949C
:10381000D339882329F00E9471396B017C0103C0E0
:10382000C12CD12C76018AE40E94D3398823D9F0A7
:103830000E9471396AAF7BAF8CAF9DAF20E030E062
:10384000A901C701B6010E94DDC981111AC020E09B
:1038500030E0A9016AAD7BAD8CAD9DAD0E94DDC9A4
:1038600081110FC074C320E030E0A901C701B60187
:103870000E94DDC9882309F46AC31AAE1BAE1CAED0
:103880001DAED701C601B0588EA79FA7A8ABB9AB94
:103890002AAD3BAD4CAD5DAD50582AAB3BAB4CAB0C
:1038A0005DAB9C01AD01BC01CD010E9442CA4B0140
:1038B0005C012AA93BA94CA95DA9CA01B9010E94D2
:1038C00042CA9B01AC01C501B4010E94F4CD0E9423
:1038D0005FD0A2966CAF7DAF8EAF9FAFA297809165
:1038E000E60B9091E70BA091E80BB091E90B8EAB42
:1038F0009FABA8AFB9AFA7019601BC01CD010E9453
:10390000F4CD2A966CAF7DAF8EAF9FAF2A97A09073
:10391000EA0BB090EB0BC090EC0BD090ED0B229625
:10392000ACAEBDAECEAEDFAE22972AAD3BAD4CAD58
:103930005DADC601B5010E94F4CD2E966CAF7DAF92
:103940008EAF9FAF2E97C0906E06D0906F06E0901E
:103950007006F09071066296CCAEDDAEEEAEFFAEB4
:1039600062972A962CAD3DAD4EAD5FAD2A97C7014B
:10397000B6010E94F3CD6B017C012091720630915B
:103980007306409174065091750666962CAF3DAF54
:103990004EAF5FAF66972E962CAD3DAD4EAD5FAD91
:1039A0002E9766966CAD7DAD8EAD9FAD66970E94ED
:1039B000F3CD4B015C018091EE0B9091EF0BA09148
:1039C000F00BB091F10B6A968CAF9DAFAEAFBFAF6D
:1039D0006A979C01AD01609176067091770680919F
:1039E0007806909179060E94F3CD26966CAF7DAF54
:1039F0008EAF9FAF269720917A0630917B0640913B
:103A00007C0650917D06A6962CAF3DAF4EAF5FAFC2
:103A1000A6978091F20B9091F30BA091F40BB091CB
:103A2000F50B6E968CAF9DAFAEAFBFAF6E97A70193
:103A300096016EA57FA588A999A90E9442CA2B016B
:103A40003C01A50194016AA97BA98CA99DA90E94AA
:103A500042CA9B01AC01C301B2010E94F4CD2B010B
:103A60003C01A50194016EA57FA588A999A90E9492
:103A700042CA4B015C01A70196016AA97BA98CA9E6
:103A80009DA90E9442CA9B01AC01C501B4010E94DC
:103A9000F3CDA30192010E9467CE6B017C0120E06F
:103AA00030E0A9010E94DDC987FF0AC02BED3FE08D
:103AB00049EC50E4C701B6010E94F4CD6B017C01D2
:103AC000112351F02BED3FE049EC50E4C701B60162
:103AD0000E94F3CD6B017C0120E030E0A901C70119
:103AE000B6010E94DDC9811126C062962CAD3DADA4
:103AF0004EAD5FAD62976EA97FA988AD99AD0E946A
:103B0000DDC9811118C066962CAD3DAD4EAD5FADDF
:103B1000669722966CAD7DAD8EAD9FAD22970E94CB
:103B2000DDC9811108C06BEDC62E6FE0D62E69ECA1
:103B3000E62E60E4F62EA2962CAD3DAD4EAD5FAD07
:103B4000A297C701B6010E9442CA9B01AC010E9424
:103B500042CA4B015C0126962CAD3DAD4EAD5FAD2A
:103B60002697CA01B9010E9442CA9B01AC01C50156
:103B7000B4010E94F4CD0E945FD04B015C012FE69E
:103B800032E143E85AE30E94DDC987FDDCC1C5018B
:103B9000B4010E9469CF0E943DCF7FAF6EAF672B0B
:103BA00021F421E030E03FAF2EAFAEACBFACB501A9
:103BB00080E090E00E94E1C94B015C019B01AC01F7
:103BC000C701B6010E94D0CE6EAB7FAB88AF99AF74
:103BD000A501940126966CAD7DAD8EAD9FAD269767
:103BE0000E94D0CEA2966CAF7DAF8EAF9FAFA29752
:103BF0006E962CAD3DAD4EAD5FAD6E97A6966CAD9D
:103C00007DAD8EAD9FADA6970E94F3CDA501940129
:103C10000E94D0CEA6966CAF7DAF8EAF9FAFA69719
:103C20002EA93FA948AD59ADCA01B9010E9442CAA7
:103C300020E030E040E05FE30E9442CA9B01AC011B
:103C400060E070E080E89FE30E94F3CD26966CAFC1
:103C50007DAF8EAF9FAF26976A96CCACDDACEEAC55
:103C6000FFAC6A97C986DA86EB86FC866E96ACACAA
:103C7000BDACCEACDFAC6E97AD86BE86CF86D88AA3
:103C80006091990270919A02072E000C880B990B93
:103C90000E94E3C92091000230910102409102028A
:103CA000509103020E9442CA2AE037ED43E25CE3EE
:103CB0000E9442CA62966CAF7DAF8EAF9FAF629793
:103CC0000E94FB699B01AC0128533F4F4F4F5F4F50
:103CD00066962CAF3DAF4EAF5FAF66974EA45FA424
:103CE00068A879A822242394312C59E1D52EAEACB2
:103CF000BFAC2A143B0409F412C10E94A8990E9487
:103D0000FB69DC01CB0166962CAD3DAD4EAD5FADE0
:103D10006697821B930BA40BB50BB7FD11C00E94D5
:103D2000FB699B01AC0128533F4F4F4F5F4F669695
:103D30002CAF3DAF4EAF5FAF669780E00E949DB461
:103D4000DA94DD2009F441C026962CAD3DAD4EAD90
:103D50005FAD26976AA97BA98CA99DA90E9442CA3A
:103D60004B015C012EA93FA948AD59ADB201C30179
:103D70000E9442CAA50194010E94F4CD7B018C01EE
:103D800026962CAD3DAD4EAD5FAD2697B201C30179
:103D90000E9442CA4B015C012EA93FA948AD59AD12
:103DA0006AA97BA98CA99DA90E9442CA9B01AC016A
:103DB000C501B4010E94F3CD2B013C01C701D8011C
:103DC0008AAB9BABACABBDAB4FC0B10180E090E028
:103DD0000E94E1C92EA93FA948AD59AD0E9442CA2F
:103DE0004B015C010E94CDCE6B017C01C501B40189
:103DF0000E9455D04B015C01A70196016EA57FA5DD
:103E000088A999A90E9442CA2B013C01A5019401ED
:103E10006AAD7BAD8CAD9DAD0E9442CA9B01AC01E9
:103E2000C301B2010E94F4CD2B013C01A501940114
:103E30006EA57FA588A999A90E9442CA4B015C0181
:103E4000A70196016AAD7BAD8CAD9DAD0E9442CAC3
:103E50009B01AC01C501B4010E94F3CD6AAB7BAB01
:103E60008CAB9DAB39E1D32E9201A3012A966CADA8
:103E70007DAD8EAD9FAD2A970E94F4CD69837A8384
:103E80008B839C832AA93BA94CA95DA92E966CAD76
:103E90007DAD8EAD9FAD2E970E94F4CD6D837E8358
:103EA0008F839887A2962CAD3DAD4EAD5FADA297A6
:103EB00069857A858B859C850E94F4CD69877A8790
:103EC0008B879C87A6962CAD3DAD4EAD5FADA6977A
:103ED0006D857E858F8598890E94F4CD6D877E875C
:103EE0008F87988BCE0101960E945CB7C090030625
:103EF0006296ECACFDAC0EAD1FAD62979E01235FE8
:103F00003F4FAE01475F5F4FBE016B5F7F4FCE01FA
:103F100001960E9474833FEF231A330AE8CEC090C3
:103F200003066296ECACFDAC0EAD1FAD62972AE7BE
:103F300036E046E756E062E776E08EE696E00E94DD
:103F400074830E9486370E944E3A0C94E332E1E675
:103F5000F8E084918F010F5F1F4F882321F00E94AA
:103F6000593AF801F6CFE7E2F2E084918F010F5F52
:103F70001F4F882311F40C94E3320E94593AF80140
:103F8000F4CF80E50E94D339882329F00E9431398B
:103F90006B017C0103C0C12CD12C760183E50E940A
:103FA000D339882361F00E94713920E030E04AE77C
:103FB00054E40E9442CA0E943DCF6B017C010E94E2
:103FC000A19A80913C02811105C060E08DE392E0EE
:103FD0000E9494640E944E3A80914F0F9091500F2E
:103FE000A091510FB091520FC80ED91EEA1EFB1EB0
:103FF0000E94FB69DC01CB018C199D09AE09BF0948
:10400000B7FD02C00C94E33280E00E949DB4F0CF73
:1040100080917F02882311F40C94E3320E94DF39EF
:1040200089E40E94D339882329F00E9471392B0139
:104030003C0103C0412C512C32018AE40E94D33947
:10404000882329F00E9471394B015C0103C0812C47
:10405000912C540180E50E94D339882329F00E94D5
:1040600071396B017C0103C0C12CD12C760181E533
:104070000E94D339882339F00E9471396EA77FA737
:1040800088AB99AB04C01EA61FA618AA19AA209136
:104090000306C157DF4F2883CF58D0406091990263
:1040A00070919A02072E000C880B990B0E94E3C9AD
:1040B00020910002309101024091020250910302CE
:1040C0000E9442CA2AE037ED43E25CE30E9442CA02
:1040D000C057DF4F688379838A839B83C059D04060
:1040E0008091E60B9091E70BA091E80BB091E90B62
:1040F0008AAB9BABACABBDABA3019201BC01CD01C4
:104100000E94F4CDA2966CAF7DAF8EAF9FAFA29709
:104110004090EA0B5090EB0B6090EC0B7090ED0B25
:10412000A5019401C301B2010E94F4CDA6966CAF23
:104130007DAF8EAF9FAFA69720916E0630916F0630
:104140004091700650917106C701B6010E94F4CDEE
:10415000AE966CAF7DAF8EAF9FAFAE9720917206DB
:104160003091730640917406509175066EA57FA537
:1041700088A999A90E94F4CDE2966CAF7DAF8EAF6D
:104180009FAFE297AAA8BBA8CCA8DDA8A982BA8253
:10419000CB82DC824D825E826F8278860E94FB69D0
:1041A0009B01AC0128533F4F4F4F5F4FC657DF4F26
:1041B000288339834A835B83CA58D0402DEC822EF2
:1041C0002CEC922EA92C2DE3B22E1EA61AAA1AAE02
:1041D0001EAA0E94A8990E94FB698B019C01C657E8
:1041E000DF4FC880D980EA80FB80CA58D0400C19C4
:1041F0001D092E093F0937FD11C09B01AC01285351
:104200003F4F4F4F5F4FC657DF4F288339834A8355
:104210005B83CA58D04080E00E949DB4A501940100
:10422000BEA5AAA9FAADEEA96B2F7A2F8F2F9E2FCC
:104230000E94F4CD2B011C0120E030E040E85FE358
:104240000E941AD0181634F4412C512C80E8282EE4
:104250009FE3392E80916E0690916F06A0917006B3
:10426000B0917106E6968CAF9DAFAEAFBFAFE6974B
:10427000A090E60BB090E70BC090E80BD090E90B54
:10428000EA96ACAEBDAECEAEDFAEEA973F922F92CD
:104290005F924F92E696ACACBDACCEACDFACE6978D
:1042A000AE96ECACFDAC0EAD1FADAE97A2962CADAC
:1042B0003DAD4EAD5FADA297EA966CAD7DAD8EADD6
:1042C0009FADEA970E94B3750F900F900F900F90DB
:1042D0006EAF23967FAF239727968FAF27972B96A6
:1042E0009FAF2B97C0907206D0907306E090740633
:1042F000F0907506EE96CCAEDDAEEEAEFFAEEE976C
:104300002091EA0B3091EB0B4091EC0B5091ED0BAF
:10431000C258DF4F288339834A835B83CE57D0400E
:104320003F922F925F924F92EE96ACACBDACCEAC6A
:10433000DFACEE97E296ECACFDAC0EAD1FADE297B4
:10434000A6962CAD3DAD4EAD5FADA697C258DF4FE2
:10435000688179818A819B81CE57D0400E94B37554
:104360000F900F900F900F902F966FAF2F9763962F
:104370007FAF639767968FAF67976B969FAF6B978B
:1043800089819A81AB81BC81CE57DF4F8883998325
:10439000AA83BB83C258D040AD80BE80CF80D88472
:1043A000CA57DF4FA882B982CA82DB82C658D04082
:1043B000A7961FAEA7977EA56AA99AAD8EA9272FAB
:1043C000362F492F582F642D752D822D932D0E9445
:1043D000F3CD2FE632E143E05BE30E94DDC987FFC6
:1043E00006C0A796BFACA797B11011C2F7C1242D84
:1043F000352D422D532DBEA5AAA9FAADEEA96B2FDE
:104400007A2F8F2F9E2F0E94F4CD20E030E040E0E5
:104410005FE30E9442CA3B014C019F928F937F92BF
:104420006F93E696ACACBDACCEACDFACE697AE9687
:10443000ECACFDAC0EAD1FADAE97A2962CAD3DAD74
:104440004EAD5FADA297EA966CAD7DAD8EAD9FADE2
:10445000EA970E94B3750F900F900F900F90A89657
:104460006FAFA897A9967FAFA997AA968FAFAA9783
:10447000C257DF4F9883CE58D0409F928F927F9241
:104480006F92EE96ACACBDACCEACDFACEE97E296E4
:10449000ECACFDAC0EAD1FADE297A6962CAD3DADDC
:1044A0004EAD5FADA697C258DF4F688179818A8192
:1044B0009B81CE57D0400E94B3750F900F900F9004
:1044C0000F905B018C012EAD23963FAD239727966D
:1044D0004FAD27972B965FAD2B97CE57DF4F688157
:1044E00079818A819B81C258D0400E94F4CD20E01E
:1044F00030E040E05FE30E9442CA9B01AC01A89615
:104500006FADA897A9967FADA997AA968FADAA97E8
:10451000C257DF4F9881CE58D0400E94F3CD6B0137
:104520007C01E894F7F82F962FAD2F9763963FAD57
:10453000639767964FAD67976B965FAD6B97CA575A
:10454000DF4F688179818A819B81C658D0400E9463
:10455000F4CD20E030E040E05FE30E9442CA9B01DE
:10456000AC01B501C8010E94F3CD9B01AC015F779E
:10457000C701B6010E94F4CD2DEC3CEC4CEC5DE3A0
:104580000E94DDC918160CF02CCF2F96AFAE2F97D6
:104590006396BFAE639767960FAF67976B961FAF33
:1045A0006B97A896CFACA897CEAEA996DFACA9978B
:1045B0002396DFAE2397AA96EFACAA972796EFAE85
:1045C0002797C257DF4FF880CE58D0402B96FFAECA
:1045D0002B972301140121E0A7962FAFA797EBCECD
:1045E000A7019601C701B6010E94F4CD9B01AC0161
:1045F000BEA5AAA9FAADEEA96B2F7A2F8F2F9E2FF9
:104600000E94F4CD962E872E782E692E20E030E081
:1046100040E85FE3D401F3016B2F7A2F8F2F9E2F99
:104620000E941AD087FFF3C06F927F928F929F9261
:10463000E696ACACBDACCEACDFACE697AE96ECACDF
:10464000FDAC0EAD1FADAE97A2962CAD3DAD4EADFF
:104650005FADA297EA966CAD7DAD8EAD9FADEA974A
:104660000E94B3750F900F900F900F90A7966FAFA9
:10467000A797A8967FAFA897A9968FAFA997AA9654
:104680009FAFAA976F927F928F929F92EE96ACAC5B
:10469000BDACCEACDFACEE97E296ECACFDAC0EADB3
:1046A0001FADE297A6962CAD3DAD4EAD5FADA69782
:1046B000C258DF4F688179818A819B81CE57D04073
:1046C0000E94B3750F900F900F900F905B018C01BB
:1046D000A7962FADA797A8963FADA897A9964FADDF
:1046E000A997AA965FADAA97CE57DF4F68817981C7
:1046F0008A819B81C258D0400E94F4CD20E030E0F6
:1047000040E05FE30E9442CA9B01AC016EAD23967C
:104710007FAD239727968FAD27972B969FAD2B972D
:104720000E94F3CD6B017C01E894F7F89501A80194
:10473000CA57DF4F688179818A819B81C658D040F2
:104740000E94F4CD20E030E040E05FE30E9442CAE6
:104750009B01AC012F966FAD2F9763967FAD63974A
:1047600067968FAD67976B969FAD6B970E94F3CD61
:104770009B01AC015F77C701B6010E94F4CD2DEC1F
:104780003CEC4CEC5DE30E941AD018160CF43FC0D0
:104790002F96AFAE2F976396BFAE639767960FAF16
:1047A00067976B961FAF6B97A7963FADA7973EAFE6
:1047B000A8964FADA89723964FAF2397A9965FADC4
:1047C000A99727965FAF2797AA968FADAA972B96A2
:1047D0008FAF2B97492C582C272C362C7EA56AA9F5
:1047E0009AAD8EA9272F362F492F582F642D752D5E
:1047F000822D932D0E94F3CD6B017C012DEC3CECBE
:104800004CEC5DE30E941AD018160CF0E9CE7EA5A0
:104810006AA99AAD8EA9272F362F492F582F642DBC
:10482000752D822D932D0E94F3CD4B015C018EAD31
:1048300023969FAD23972796AFAD27972B96BFADB5
:104840002B9789839A83AB83BC832F968FAD2F9749
:1048500063969FAD63976796AFAD67976B96BFAD55
:104860006B978D839E83AF83B887242D352D422D82
:10487000532D60E070E080E89FE30E94F3CD6B0170
:104880007C012091EE0B3091EF0B4091F00B509199
:10489000F10B0E9442CA6EA77FA788AB99AB20910B
:1048A0007606309177064091780650917906642D0E
:1048B000752D822D932D0E9442CA9B01AC016EA5DD
:1048C0007FA588A999A90E94F4CD69877A878B87EB
:1048D0009C872091F20B3091F30B4091F40B509197
:1048E000F50BC701B6010E9442CA6B017C01209101
:1048F0007A0630917B0640917C0650917D06642DAE
:10490000752D822D932D0E9442CA9B01AC01C701D7
:10491000B6010E94F4CD6D877E878F87988BCE017C
:1049200001960E945CB7C157DF4FC880CF58D04076
:10493000C057DF4FE880F9800A811B81C059D04001
:104940009E01235F3F4FAE01475F5F4FBE016B5F2C
:104950007F4FCE0101960E94748320E030E040E852
:104960005FE3642D752D822D932D0E94DDC987FF95
:1049700005C04EA65AAA2AAE3EAA2BCC0E94863764
:104980000C94E3320E94A19A80910002909101025E
:10499000A0910202B09103028093540590935505B3
:1049A000A0935605B09357058091990290919A0271
:1049B000909353058093520584E690E090939A0279
:1049C000809399020E944E3A81E08093D00588E559
:1049D0000E94A439E82E89E50E94A439082F8AE5AF
:1049E0000E94A439F82EE11005C0011105C011E0A4
:1049F000182705C0011102C010E001C0182F0E9445
:104A00007C37111105C0E11003C0002309F444C034
:104A100020E030E040EA50E460910C0670910D0611
:104A200080910E0690910F060E94F4CD6093760659
:104A30007093770680937806909379062091EE0B19
:104A40003091EF0B4091F00B5091F10B0E941AD076
:104A500018167CF419821A821B821C829E012F5F19
:104A60003F4F46E756E06AEE7BE086EE9BE00E9411
:104A70009B36111105C0E11003C0011107C00CC025
:104A800080E090E00E94BE5C1123B9F381E090E0E9
:104A90000E94BE5C111102C0FF2021F082E090E074
:104AA0000E94BE5C0E9493388091720E8093D00564
:104AB0008091540590915505A0915605B0915705E8
:104AC0008093000290930102A0930202B09303022C
:104AD000809152059091530590939A028093990288
:104AE0000E944E3A83E080933B020E94073D0C9463
:104AF000E3321092D1030C94E33281E08093D1032E
:104B00000C94E33285E40E94D339B82E811102C09F
:104B10000E94A19AB0EA8B2EB2E09B2E16EEC12E17
:104B20001BE0D12E01E6E02E06E0F02E00E010E0C2
:104B3000A12CD4018D914D010E94D339882309F411
:104B40004EC0F6012081318142815381CC56DF4F26
:104B50002883C459D040CB56DF4F3883C559D04045
:104B6000CA56DF4F4883C659D040C956DF4F5883D5
:104B7000C759D0400E947139D6016D937D938D93B2
:104B80009C931397CC56DF4F2881C459D040CB5605
:104B9000DF4F3881C559D040CA56DF4F4881C659CA
:104BA000D040C956DF4F5881C759D0400330110556
:104BB000B1F00E94F3CD9B01AC01F70160817181DE
:104BC000828193810E94F4CDD7016D937D938D9363
:104BD0009C931397C8010E94A937AA24A3940F5F3E
:104BE0001F4FB4E0CB0ED11CE4E0EE0EF11C0430FC
:104BF000110509F09ECFAA2019F00E94933803C036
:104C0000B1100E94EA790E94073D0C94E332809132
:104C10005A0590915B058837910509F48FC70CF010
:104C200095C08C35910509F4AFC50CF04FC08B349D
:104C3000910509F4EBC2BCF48131910509F4BFC1BF
:104C40002CF4029708F438C10C94E3328F319105AB
:104C500009F4C8C18A32910509F499C2429711F04A
:104C60000C94E33243C58235910509F438C514F537
:104C70008D34910509F4E8C20CF4CCC2813591055C
:104C800011F00C94E3320E9407970E94A19A0E94AF
:104C90004BB710923F0610923E0668EE73E080E03C
:104CA00090E00E94AC6360E08FE293E00E94946425
:104CB0000C94E3328435910509F418C50CF412C53F
:104CC0008535910509F447C50C94E3328F3691057B
:104CD00009F428C3C4F48B36910509F462C464F462
:104CE0008936910509F4DAC30CF03CC48836910585
:104CF00009F4AEC20C94E3328D36910509F416C462
:104D00000CF481C3FCC28337910509F4CBC554F47C
:104D10008137910509F47FC30CF0BFC584EF92E0A1
:104D20000E940C5E8637910509F44DC60CF082C6D0
:104D30008537910511F00C94E33260E080915805BD
:104D4000909159050E94B4640C94E332823E91051F
:104D500011F40C947C300CF051C0893C910509F49D
:104D60009EC7ECF48C38910509F481C354F489375B
:104D7000910509F4E9C68D37910509F424C40C9412
:104D8000E3328B39910509F4A6C3883C910509F4F7
:104D90003EC78139910511F00C94E332DAC68E3C9E
:104DA000910511F40C945A2FB4F48C3C910509F43C
:104DB000ACC714F00C94EF2E8B3C910511F00C94C1
:104DC000E332E7E8EE2EEEE0FE2E00EA12E0F4E039
:104DD000DF2ED00E8BC78C3D910511F40C9456300C
:104DE0008D3D910511F40C946330833D910511F0D4
:104DF0000C94E332EFE7F9E00C94C02F8C3AF1E029
:104E00009F0711F40C94DA305CF58F3231E0930790
:104E100011F40C94D43084F48D3251E0950711F4E0
:104E20000C94CE3014F00C94D1308C32914011F4AB
:104E30000C94A5300C94E3328039E1E09E0711F424
:104E40000C94D7308A39F1E09F0709F4E0C2833629
:104E5000914011F00C94E332E1E6F8E00C946C32EE
:104E6000873F31E0930711F40C94CA3194F4853FE5
:104E700051E0950711F40C94C43114F00C94C7312F
:104E8000843F914011F00C94E3320E94D6560C946A
:104E9000E3328A39E2E09E0711F40C94A12F873E99
:104EA000F3E09F0711F40C9481328835924011F0A1
:104EB0000C94E3320C94D631A0905805B09059056B
:104EC00080E50E94D339882359F00E9431396B0163
:104ED0007C0111E0672B682B692B31F410E004C0D2
:104EE00010E0C12CD12C760183E50E94D3398823B0
:104EF000F1F00E94713920E030E04AE754E40E946A
:104F000042CA0E943DCF6B017C01111112C0672B78
:104F1000682B692B71F4A114B10459F0D5018C915F
:104F2000882339F061E0C5010E94B46407C01123F1
:104F300091F360E085E592E00E94946483E090E064
:104F400090937F0680937E0681E08093A0060E9466
:104F5000A19A0E944E3AC114D104E104F104F1F087
:104F600080914F0F9091500FA091510FB091520F1F
:104F7000C80ED91EEA1EFB1E0E94FB69DC01CB0194
:104F80008C199D09AE09BF09B7FF15C08091A00615
:104F9000882389F080E00E949DB4EECF8091A00626
:104FA000882321F080E00E949DB4F8CF60E086E481
:104FB00092E00E9494641092A0060C94E33260E0A8
:104FC00088E692E00E9494645F988A989FB7F8946C
:104FD000809108018E7F809308019FBF47981298A7
:104FE0000C94E33280918D0C90918E0C019719F402
:104FF0000E94FB6908C06091970C7091980C809199
:10500000990C90919A0C0091930C1091940C209112
:10501000950C3091960C601B710B820B930B28EE54
:1050200033E040E050E00E94B8CD80918F0C909129
:10503000900CA091910CB091920CBC01CD01620F2B
:10504000731F841F951FACE3CA2ED12CE12CF12CC9
:10505000A70196010E94B8CD762E672ECA01B9012C
:10506000A70196010E94B8CD6B017C01CA01B9016C
:1050700028E130E040E050E00E94B8CD4B015C01F7
:10508000C9016DE671E00E94B8D08E010F5F1F4F1D
:105090006115710599F06F927F92DF92CF929F9286
:1050A0008F929F938F937F936F9389E992E09F9361
:1050B0008F931F930F930E9476C912C00097B1F08F
:1050C0006F927F92DF92CF929F928F929F938F9356
:1050D00089E892E09F938F931F930F930E9476C964
:1050E0000FB6F894DEBF0FBECDBF36C08114910459
:1050F000A104B10479F06F927F92DF92CF929F92D8
:105100008F928DE792E09F938F931F930F930E944E
:1051100076C9E6CFC114D104E104F10469F06F92BD
:105120007F92DF92CF9285E792E09F938F931F93B8
:105130000F930E9476C9D4CF6F927F9281E792E05D
:105140009F938F931F930F930E9476C90F900F9098
:105150000F900F900F900F9060E0C8010E94B46410
:10516000EFE7F9E084917F019FEFE91AF90A8823BC
:1051700021F00E94593AF701F5CFB8018DEA92E08B
:105180000E948B758AE00E94593A0C94E33283E5C1
:105190000E94D339882311F40C94E3320E945139D0
:1051A000E82E80E50E94D339882339F00E944139E6
:1051B0008B0177FF04C00C94E3320DE010E0902FD8
:1051C000E7E1F6E08BE28E0F2491921729F03196F9
:1051D0008E13FACF0C94F432E1E6F8E084918F015B
:1051E0000F5F1F4F882321F00E94593AF801F6CF34
:1051F000EAEBF2E084918F010F5F1F4F882311F4D7
:105200000C94E3320E94593AF801F4CF0E947F795E
:105210000C94E33280918D0C90918E0C019711F0DB
:105220000C94E33282E090E090938E0C80938D0C8E
:105230000E94FB696093970C7093980C8093990C73
:1052400090939A0C0C94E3320E94D1760C94E33242
:1052500088E690E00E94C63A81110C94E332809176
:10526000BB0E83FF02C00C94E33283E50E94D33966
:10527000882309F440C00E9471390E9438CF70938E
:1052800041066093400680E00E94BC960E947139FE
:1052900020E030E04AEA52E40E94DDC918163CF0F2
:1052A0000E94D17660E080ED92E00E9494640E94BA
:1052B00071392091120630911306409114065091D5
:1052C00015060E941AD01816B4F485E193E09F9356
:1052D0008F938091CC0390E001969F938F9389ECFC
:1052E00092E09F938F931F920E9462790FB6F89479
:1052F000DEBF0FBECDBF0E9455C20C94E3328EE4D8
:105300000E94D339882311F40C94E3320E9441396E
:105310006093440F7093450F8093460F9093470F0F
:105320000C94E33283E50E94A439882359F083E585
:105330000E94D339882319F00E94513901C080E0BE
:105340008093BB0EEFE7F9E084918F010F5F1F4F51
:10535000882321F00E94593AF801F6CFEDEEF2E0F1
:1053600084918F010F5F1F4F882321F00E94593ACB
:10537000F801F6CF8091BB0E8823A1F1FFEDCF2E6F
:10538000F2E0DF2EE12CF12C20E08091BB0E90E0CA
:105390000E2C02C0959587950A94E2F780FF17C0FE
:1053A000BB24B394B20E222319F08CE20E94593A26
:1053B000F60125913491F901849189010F5F1F4F06
:1053C000882321F00E94593A9801F5CF2B2DFFEF49
:1053D000EF1AFF0A32E0C30ED11C45E0E416F104D7
:1053E000A1F60CC0E9EEF2E084918F010F5F1F4F30
:1053F000882321F00E94593AF801F6CF8AE00E94F2
:10540000593A0C94E332109204020C94E3320E9455
:1054100042A70C94E33283E50E94D339882369F0D4
:105420000E94513980939B028D3310F40C94E33227
:105430008CE380939B020C94E332EFE7F9E08491D4
:105440008F010F5F1F4F882321F00E94593AF80106
:10545000F6CF40919B0250E060E070E08DEF92E06B
:105460000E941B758AE00E94593A0C94E3328091A5
:10547000BB0E83FF02C00C94E33283E50E94D33954
:10548000882311F40C94E3320E9471390E9438CFC2
:1054900070931C0D60931B0D0C94E33289E690E031
:1054A0000E94C63A811111C0E4E0F3E084918F01BB
:1054B0000F5F1F4F882321F00E94593AF801F6CF61
:1054C0000E94B73D8AE00E94593A10927F061092DE
:1054D0007E060C94D13483E50E94D339882311F4DD
:1054E0000C94E3320E94513980934C0F8D3318F0A5
:1054F0008CE380934C0F0E94FB696B017C0120912F
:105500004C0F30E0A8EEB3E00E94E4CDDC01CB010B
:105510008C0D9D1DAE1DBF1D8093480F9093490FAC
:10552000A0934A0FB0934B0F0C94E3328DE690E0BA
:105530000E94C63A81110C94E3328091BB0E83FF26
:1055400002C00C94E33283E50E94D3398AAF811103
:105550000C94093382E50E94D33981110C940933EC
:105560000C94E33283E50E94D339882339F00E94FA
:1055700041398B016F3F710519F010F00FEF10E00A
:1055800080E50E94D339811106C010933F06009335
:105590003E060C94E3320E94513981110C94E3329F
:1055A000F4CF80E50E94D339811106C010923F06E6
:1055B00010923E060C94E3320E944139672B11F0A1
:1055C0000C94E332F3CF8CE40E94A439882319F0C1
:1055D0000E94713904C060E070E080E090EC6EA33E
:1055E0007FA388A799A78AE50E94D339882319F059
:1055F0000E94713903C060E070E0CB0120E030E030
:1056000040E251E40E94F4CD6AA37BA38CA39DA346
:1056100088E50E94D339882319F00E94713903C0AC
:1056200060E070E0CB0120E030E040E450E40E9414
:10563000F4CD6E8F7F8F88A399A389E50E94D3391B
:10564000882319F00E94713903C060E070E0CB013B
:1056500020E030E040E450E40E94F4CD6A8F7B8F7C
:105660008C8F9D8FA0908D0CB0908E0C19821A8219
:105670001B821C8280916D068111A5C7C12CE12C73
:105680008E010F5F1F4F9E01265E3F4FAE01425EAF
:105690005F4FBE016E5D7F4FCE0186960E94515BCB
:1056A000882309F490C780E00E94413619821A824B
:1056B0001B821C821E8A1F8A188E198E80916D068D
:1056C000882331F040E0B801CE0146960E9495C093
:1056D000AA94AB2809F077C70E947F7974C710920B
:1056E000D00371C781E08093D0036DC783E50E942A
:1056F000D339882399F00E94713920E030E04AE7DD
:1057000054E40E9442CA0E943DCF60939C02709371
:105710009D0280939E0290939F0255C788E50E9448
:10572000A43981110C94823489E50E94A439811135
:105730000C9482348AE50E94A43981110C9482343D
:1057400085E40E94A43981110C9482340E94A19AAC
:105750000E944BB738C783E50E94A439882309F417
:1057600032C70E94713920E030E04AE754E40E94D9
:1057700042CA0E943DCF6093530F7093540F8093A1
:10578000550F9093560F1FC750EAC52E52E0D52EE5
:1057900066EFE62E6BE0F62E10E0F60181916F01C8
:1057A0000E94A439882309F46EC0133009F063C045
:1057B0000E9471394B015C0120E030E040EA51E485
:1057C0000E94DDC987FF4EC0A50194016091020CC3
:1057D0007091030C8091040C9091050C0E94D0CE26
:1057E0002B013C019B01AC016091AF0C7091B00C9E
:1057F0008091B10C9091B20C0E9442CA6093AF0CA0
:105800007093B00C8093B10C9093B20CA3019201F1
:105810006091930E7091940E8091950E9091960EDA
:105820000E9442CA6093930E7093940E8093950EDB
:105830009093960E6091D30C7091D40C8091D50CFE
:105840009091D60C0E94E1C9A30192010E9442CA24
:105850000E943DCF6093D30C7093D40C8093D50CF1
:105860009093D60C8092020C9092030CA092040CA0
:10587000B092050C08C00E947139D7016D937D93D9
:105880008D939C9313971F5FB4E0EB0EF11C1430C3
:1058900009F083CF0E944A8396C60E94A19A0E9473
:1058A000073D91C6E7E1F4E084918F010F5F1F4F40
:1058B000882321F00E94593AF801F6CFE9E0F4E09C
:1058C00084918F010F5F1F4F882321F00E94593A66
:1058D000F801F6CFE2EFF3E084918F010F5F1F4FE5
:1058E000882321F00E94593AF801F6CFE2EEF3E066
:1058F00084918F010F5F1F4F882321F00E94593A36
:10590000F801F6CFE1EDF3E084918F010F5F1F4FB7
:10591000882321F00E94593AF801F6CFE0ECF3E039
:1059200084918F010F5F1F4F882321F00E94593A05
:10593000F801F6CFE1EBF3E084918F010F5F1F4F89
:10594000882321F00E94593AF801F6CFECE9F3E000
:1059500084918F010F5F1F4F882321F00E94593AD5
:10596000F801F6CFE6E8F3E084918F010F5F1F4F57
:10597000882321F00E94593AF801F6CFE1E7F3E0DD
:1059800084918F010F5F1F4F882321F00E94593AA5
:10599000F801F6CFE4E5F3E084918F010F5F1F4F2C
:1059A000882321F00E94593AF801F6CFECE3F3E0A6
:1059B00084918F010F5F1F4F882309F404C60E9452
:1059C000593AF801F5CF85E40E94A439882381F083
:1059D0000E946239882361F0EFE7F9E084918F013A
:1059E0000F5F1F4F882321F00E94593AF801F6CF2C
:1059F00081E40E94A439882381F00E9462398823BF
:105A000061F0EAEDF4E084918F010F5F1F4F88236E
:105A100021F00E94593AF801F6CF009158051091F3
:105A20005905F80181918F01882309F4E7CC0E9480
:105A3000593AF7CFEFEFF4E084918F010F5F1F4FDA
:105A4000882321F00E94593AF801F6CFE7EFF4E0FD
:105A500084918F010F5F1F4F882321F00E94593AD4
:105A6000F801F6CF659903C006E013E002C00BE031
:105A700013E0D8018D918D01882319F00E94593AC5
:105A8000F8CF8AE00E94593AEFEEF4E084918F015A
:105A90000F5F1F4F882321F00E94593AF801F6CF7B
:105AA0008091030181FD03C006E013E002C00BE01A
:105AB00013E0F80181918F01882319F00E94593A6F
:105AC000F8CF8AE00E94593AE7EEF4E084918F0122
:105AD0000F5F1F4F882321F00E94593AF801F6CF3B
:105AE0004B9903C006E013E002C00BE013E0D801BD
:105AF0008D918D01882319F00E94593AF8CF8AE0E0
:105B00000E94593AEEEDF4E084918F010F5F1F4F30
:105B1000882321F00E94593AF801F6CF4A9903C030
:105B200006E013E002C00BE013E0F80181918F0161
:105B3000882309F463CC0E94593AF7CF81E080931F
:105B4000D0058093720E3FC51092D0051092720E50
:105B50003AC583E50E94D339882319F00E94413960
:105B600002C060E070E08B01112702301105CCF01B
:105B7000E1E6F8E084918F010F5F1F4F882321F049
:105B80000E94593AF801F6CFE9E1F5E084918F01DE
:105B90000F5F1F4F882309F416C50E94593AF80178
:105BA000F5CF88E40E94D3398823A9F00E944139B7
:105BB0006A3A71053CF06530F1E07F072CF064E053
:105BC00071E002C06AEA70E0F801EE0FFF1FEE5BC1
:105BD000F94F7183608386E40E94D339882309F4E6
:105BE000F2C40E944139000F111FF801EA5BF94F1E
:105BF000718360836F3F710519F014F06FEF70E0EF
:105C000077FF02C060E070E071836083DCC488ECE1
:105C100090E00E94C63A8111D6C484E40E94A4395F
:105C20008823D1F10E94713911E020E030E0A90110
:105C30000E94DDC9811101C010E01093B70C11233F
:105C400059F10091CC0310E00E947139000F111F2F
:105C5000000F111FF801ED54F34F608371838283AD
:105C6000938320E030E0A9016091B30C7091B40CF3
:105C70008091B50C9091B60C0E94DDC981110CC0C9
:105C800080E090E0A0EEBFE38093B30C9093B40C5F
:105C9000A093B50CB093B60C0E9456B494C4A7E977
:105CA000EA2EAEE0FA2E00EA12E0B4E0DB2ED00ECF
:105CB000D8018D918D010E94A439882349F00E945A
:105CC00071390E943DCFF701608371838283938392
:105CD000F4E0EF0EF11CD012EBCF0E941D8273C4D2
:105CE000F4E0EF0EF11CD01609F46DC4D8018D91CB
:105CF0008D010E94A439882399F30E947139F7011C
:105D00006083718382839383EBCF83E50E94A43900
:105D10008823D9F00E947139AB01BC014093AF0ECA
:105D20005093B00E6093B10E7093B20E4093A70ED5
:105D30005093A80E6093A90E7093AA0E85E995E082
:105D40000E9455758AE00E94593A80E50E94A43964
:105D5000882399F00E947139AB01BC014093AF0ECA
:105D60005093B00E6093B10E7093B20E88E795E039
:105D70000E9455758AE00E94593A82E50E94A43932
:105D8000882399F00E947139AB01BC014093AB0E9E
:105D90005093AC0E6093AD0E7093AE0E89E595E016
:105DA0000E9455758AE00E94593A84E50E94A43900
:105DB000882309F408C40E947139AB01BC014093E7
:105DC000A70E5093A80E6093A90E7093AA0E8BE3B2
:105DD00095E00E9455758AE00E94593AF4C383E524
:105DE0000E94A439882351F00E9471396093830E78
:105DF0007093840E8093850E9093860E84E50E94A6
:105E0000A439882351F00E94713960937F0E7093FA
:105E1000800E8093810E9093820E82E40E94A439BA
:105E2000882351F00E9431396093BF0C7093C00CED
:105E30008093C10C9093C20C88E50E94A4398823FA
:105E400051F00E9471396093A30C7093A40C80935D
:105E5000A50C9093A60C89E50E94A439882351F0E3
:105E60000E9471396093A70C7093A80C8093A90CC1
:105E70009093AA0C8AE50E94A439882351F00E94CD
:105E800071396093AB0C7093AC0C8093AD0C909314
:105E9000AE0C85E40E94A439882309F494C30E94BF
:105EA00071396093AF0C7093B00C8093B10C9093E8
:105EB000B20C89C350EAA52E52E0B52E66EEC62E6E
:105EC0006BE0D62E74EDE72E75E0F72E00E010E0C3
:105ED000D5018D915D010E94A439882311F10E94A2
:105EE00071392B013C01F7012081318142815381BD
:105EF0000E94F3CD9B01AC01D6016D917D918D91F6
:105F00009C910E94F4CDF601608371838283938318
:105F1000D7014D925D926D927C921397C8010E94B9
:105F2000A9370F5F1F4FB4E0CB0ED11CE4E0EE0E9B
:105F3000F11C0330110561F60E9493380E94073D61
:105F400042C38AE50E94A439882351F00E94713926
:105F500060936D0D70936E0D80936F0D9093700D27
:105F600040916D0D50916E0D60916F0D7091700D9F
:105F70008DEB95E00E9455758AE00E94593A23C343
:105F800084918F010F5F1F4F882321F00E94593A9F
:105F9000F801F6CF83E50E94A439882321F00E94FE
:105FA000623980932702E7E0F6E084918F010F5F6A
:105FB0001F4F882321F00E94593AF801F6CF8091B3
:105FC0002702811103C0E3E0F6E002C0EFEFF5E045
:105FD00084918F010F5F1F4F882321F00E94593A4F
:105FE000F801F6CFE7EFF5E084918F010F5F1F4FC7
:105FF000882321F00E94593AF801F6CF40911A0601
:1060000050911B0660911C0670911D0685EF95E06E
:106010000E94557540911E0650911F066091200602
:106020007091210682EF95E00E94557540912206FD
:106030005091230660912406709125068FEE95E01D
:106040000E945575E7EEF5E084918F010F5F1F4FB9
:10605000882321F00E94593AF801F6CF40911B02A3
:1060600050911C0260911D0270911E0285EE95E018
:106070000E94557540911F025091200260912102AB
:106080007091220282EE95E00E94557540912302A4
:106090005091240260912502709126028FED95E0C7
:1060A0000E9455758AE00E94593A8DC283E50E948C
:1060B000D339882309F487C20E94413970939A0228
:1060C0006093990280C28DED90E00E94C63A8111E2
:1060D0007AC283E50E94D339882309F474C20091FF
:1060E000CC0310E00E944139000F111FF801E9565E
:1060F000FD4F7183608367C280E50E94A4398823C5
:1061000009F461C20E944139F62EC62ED72E83E5CE
:106110000E94D339882321F00E9441398B0102C0AB
:106120000FEF1FEFC8010196039708F04CC2D7FC90
:106130004AC2E7E1F6E08BE28E0F9491F91609F47A
:1061400042C231968E13F9CF04C483E50E94D3393D
:10615000882319F00E94413902C064E071E07F8B0E
:106160006E8B80E50E94D339882339F00E94413933
:106170006938F3E17F0730F402C068EE73E07A8398
:10618000698304C088E893E19A838983BE016A5ECB
:106190007F4FCE0101960E942E7915C20E94B6ABA8
:1061A00012C20E9460AB0FC20E949BA70CC20E9449
:1061B000A19A09C294EDC92E95E0D92E26EEE22EC1
:1061C0002BE0F22E37E1232E36E0332E00E010E0F4
:1061D0009101275136403FA72EA7D1018D911D0176
:1061E000882309F4A0C0F701408051806280738049
:1061F000F801E55EFD4F2081318142815381F80134
:10620000E65EF94F60817181828193810E94F4CDB5
:1062100020E030E040E05FE30E9442CA9B01AC0115
:10622000C301B2010E941AD0181644F4F801E959CA
:10623000F14F85909590A590B49003C0812C912C3E
:106240005401F801EC5FF94F208131814281538183
:10625000C301B2010E94F3CD9B01AC01C501B401A1
:106260000E94F3CD4B015C0120E030E040EA51ECAC
:106270000E941AD087FD28C020E030E040EA51E4B7
:10628000C501B4010E94DDC91816F4F0D6012D91A4
:106290003D914D915C91C501B4010E94F3CD9B01EC
:1062A000AC01C301B2010E94F4CDF7016083718398
:1062B00082839383D6018D929D92AD92BC92139767
:1062C0008EA59FA546D62FC0E1E6F8E084918F0108
:1062D0000F5F1F4F882321F00E94593AF801F6CF33
:1062E000E0E6F6E084918F010F5F1F4F882321F0D5
:1062F0000E94593AF801F6CF61E082E596E00E94EB
:1063000094640E94E29388E290E09A83898388EC07
:1063100090E09F8B8E8BBE016F5F7F4FCE014696C4
:106320000E942E7950C1B4E0CB0ED11C0C5F1F4FE0
:10633000E4E0EE0EF11C0C30110509F049CFF3D664
:106340000E94073D60E082E496E00E94946483E945
:1063500092E09F8B8E8B04E610E01A830983BE01C6
:106360006A5E7F4FCE0101960E942E798AEB92E001
:106370009F8B8E8B1A830983BE016A5E7F4FCE018D
:1063800001960E942E791FC10E947BA21CC10E940F
:106390005EA119C183E5D8D7882311F093D701C036
:1063A00081E091E089270E94AC9A0DC185E4CCD7A9
:1063B000882311F096D704C060E070E080E090EC94
:1063C0006AA77BA78CA79DA78AE5EDD7882311F044
:1063D00088D704C060E070E080E291E46EA37FA300
:1063E00088A799A788E5DFD7882311F07AD704C05A
:1063F00060E070E080E490E46AA37BA38CA39DA39B
:1064000089E5D1D7882311F06CD704C060E070E033
:1064100080E490E46E8F7F8F88A399A385E594D75D
:10642000882311F05ED704C060E070E088EC92EC45
:106430006A8F7B8F8C8F9D8F8CE486D7882311F099
:1064400050D703C060E070E0CB016E8B7F8B888FEC
:10645000998F82E4A8D7882319F013D7F62E02C0AB
:1064600085E0F82EA0908D0CB0908E0C80916D067A
:1064700081112BC0CC24C394EF2C8E01065E1F4FDC
:106480009E01225E3F4FAE014E5D5F4FBE016A5DD1
:106490007F4FCE018A960E94515B8823B1F08F2DE9
:1064A000F0D380E090E0A8E4B2E489839A83AB83E0
:1064B000BC8380916D06882341F04F2DBE016F5F34
:1064C0007F4FCE0146960E9495C0AA94AB2809F052
:1064D0007AC00E947F7977C084918F010F5F1F4F30
:1064E000882319F0E6D7F801F7CFEEE7F6E08491BC
:1064F0008F010F5F1F4F882309F465C0DAD7F801B9
:10650000F6CF81E080937F021092070C83E51CD7C1
:10651000811103C00E9412B856C0D4D6811153C055
:10652000F9CFF0905A05FF2001F1EFE7F9E08491EF
:106530008F010F5F1F4F882319F0BBD7F801F7CFEA
:1065400084E5B7D76F2D70E080E090E04AE0B8D7DF
:1065500080E2AFD700E213E0D8018D918D0188234E
:1065600011F40C94FE29A5D7F7CF10920306EFE79C
:10657000F9E084918F010F5F1F4F882319F099D79D
:10658000F801F7CF6091030670E08DE896E00E9475
:1065900072758AE08ED717C0EFE7F9E084918F011A
:1065A0000F5F1F4F882319F084D7F801F7CF609150
:1065B0004D0F70914E0F8FE996E00E948B7582E22D
:1065C00078D78AE076D710927F0610927E060E94D6
:1065D000F3B7E7C16115710519F4BC016150710988
:1065E000A0E0B0E00C94271961E0802F0E94C06801
:1065F0006E2D802F0E949168F12CB701802F0E9490
:10660000FC6809301105F9F6F0923F06E0923E066B
:10661000DACF67D60E9438CF709341066093400668
:1066200080E00E94BC965DD620E030E04AEA52E469
:106630000E94DDC9181644F00E94D17660E080E225
:1066400093E00E94946402C00E947F7960914006AA
:1066500070914106072E000C880B990B0E94E3C92C
:1066600020911206309113064091140650911506A0
:106670000E941AD01816B4F485E193E09F938F938B
:106680008091CC0390E001969F938F9389E193E0F2
:106690009F938F931F920E9462790FB6F894DEBF8A
:1066A0000FBECDBF0E9455C281E0809304021AAA9A
:1066B0001BAA1CAA1DAA1EAA1FAA18AE19AE1EA6A6
:1066C0001EAE9CE323969FAF2397ACE12796AFAF16
:1066D0002797B6E42B96BFAF2B97C12CD12C70E82F
:1066E000E72EEFEBFE2E812C912C54016091400699
:1066F00070914106072E000C880B990B0E94E3C98C
:10670000162F072F782E692E262F372F482F592F17
:10671000B601C7010E94DDC9882311F1209112063C
:10672000309113064091140650911506612F702F79
:10673000872D962D0E94DDC9881F8827881F8EA768
:10674000CAACCC2089F0882379F080910402882398
:1067500009F439CF60E087E093E00E94946433CF7E
:106760001C2D0D2D7E2C6F2C0E94FB696B017C0172
:10677000DC01CB012EA93FA948AD59AD821B930B7B
:10678000A40BB50BB7FD37C0D701C60188519C4F8C
:10679000AF4FBF4F8EAB9FABA8AFB9AF0E94B73D15
:1067A000E5E1F3E084912F019FEF491A590A88230C
:1067B00019F07FD6F201F6CF81149104A104B1043F
:1067C000B1F0D501C401805F984DAF4FBF4FBC0100
:1067D000CD016C197D098E099F0928EE33E040E058
:1067E00050E00E94B8CDCA01B9010CD702C08FE3B6
:1067F00060D68AE05ED680E00E949DB44FD620909D
:106800001206309013064090140650901506910120
:10681000A201612F702F872D962D0E94F3CD9F77B7
:1068200081149104A104B10449F420E030E040E86F
:106830005FE30E94DDC987FF0BC008C020E030E0A5
:1068400040E450E40E941AD0181614F4460157018F
:10685000AEA5AA23D9F12AA93BA94CA95DA9211566
:1068600031054105510541F0D701C601821B930B4B
:10687000A40BB50BB7FD2AC09101A2016EAD239602
:106880007FAD239727968FAD27972B969FAD2B979C
:106890000E94F3CD20E030E040EC5FE30E94DDC9D0
:1068A00087FD53CFD701C601805A9541AF4FBF4FE7
:1068B0008AAB9BABACABBDAB2EAE23963FAE239762
:1068C00027964FAE27972B965FAE2B9780910402A9
:1068D000882309F43ACF81149104A104B10429F466
:1068E000C12ED02EE72CF62C01CF90E1C91A97E2E9
:1068F000D90AE108F108C818D908EA08FB08F7FE28
:1069000024CFEECF0E94A19A88E51ED5882319F0E6
:106910005F9A1092D10589E517D5882319F08A9AD4
:106920001092D2058AE510D5882359F09FB7F894C4
:10693000809108018160809308019FBF479A10925F
:10694000D30585E401D5882309F43DCE0E949BB48C
:106950003ACE0E94A19A60E08F2D0E94C0680F3F3E
:10696000BFEF1B0759F48F2D0E94696831E020E0CA
:10697000892B09F030E0032F122F05C001301105DB
:1069800069F000E010E08F2D0E9469688017910780
:1069900009F419CE80E00E949DB4F5CF01E010E02B
:1069A000F2CFC956DF4F0FB6F894DEBF0FBECDBF92
:1069B000DF91CF911F910F91FF90EF90DF90CF90DB
:1069C000BF90AF909F908F907F906F905F904F900F
:1069D0003F902F90089582E08093220D08958FB705
:1069E000F8949091430F2091420F291759F0E92F05
:1069F000F0E0EE53F14F208130E09F5F9F7790935E
:106A0000430F02C02FEF3FEF8FBFC90108950F93CF
:106A10001F93CF93DF93EC010E94FB690E811F81CE
:106A200028853985011511052105310559F52C8574
:106A30002223A9F13A8521502C8721E0230F2A87B0
:106A40004D85241301C01A86FE0124E0329FE00D1B
:106A5000F11D112406851785208931890A831B833E
:106A60002C833D83DC01CB01800F911FA11DB11D43
:106A70008E839F83A887B9878C819D81892B79F02C
:106A8000409A0DC0DC01CB01801B910BA20BB30B14
:106A9000B7FD05C040981E821F8218861986DF91B7
:106AA000CF911F910F910895CF92EF92FF920F9384
:106AB0001F93E0900002F0900102009102021091F9
:106AC0000302C090030622EF3BE04EEE5BE06AEE6D
:106AD0007BE086EE9BE00E9474831F910F91FF90F4
:106AE000EF90CF900895CF92DF92EF92FF92CF93E5
:106AF00081E080930402C1E080910402882309F4BC
:106B000044C0CC2309F441C080E00E949DB4609150
:106B1000400670914106C0E06115710569F3072ECA
:106B2000000C880B990B0E94E3C99B01AC0160919A
:106B300012067091130680911406909115060E941A
:106B4000F3CD6B017C0120E030E0A9010E941AD056
:106B500018165CF020E030E040E450ECC701B601CC
:106B60000E94DDC987FFC8CF0BC020E030E040E4C1
:106B700050E4C701B6010E941AD018160CF0BCCF21
:106B800089E090E00E940556B6CFCF91FF90EF903C
:106B9000DF90CF900895CF92DF92EF92FF920F9304
:106BA0001F93CF93DF9300D01F92CDB7DEB7182F7E
:106BB000662351F01092CB051092C7051092C805BC
:106BC0001092C9051092CA050E94FB69C090C705C2
:106BD000D090C805E090C905F090CA059B01AC01B2
:106BE0002C193D094E095F0957FD3EC017FD16C01F
:106BF0004091CB05212F012E000C330B2C5F3F4F12
:106C0000E42F042E000CFF0B2E173F076CF14117E9
:106C10002CF000E911E020E030E004C004EC19E0C1
:106C200020E030E0DC01CB01800F911FA21FB31FD9
:106C30008093C7059093C805A093C905B093CA0572
:106C400080ED97E09C838B838CE291E09A8389832B
:106C5000BE016D5F7F4FCE0101960E942E7980911B
:106C6000CB058F5F8093CB050F900F900F900F9007
:106C7000DF91CF911F910F91FF90EF90DF90CF9018
:106C80000895CF93DF93C82F83E090E090937F0621
:106C900080937E0681E08093A006D1E08091A006DB
:106CA000882309F43FC060E08C2F75DF8091080CC9
:106CB0008823A1F188E090E00E9405568091A0060B
:106CC000882321F081E00E949DB4F8CF1092170D27
:106CD0001092180D1092190D10921A0D1092080CA6
:106CE0000E94BC9600DF82E090E00E9405560E9460
:106CF000FB69DC01CB0188539045AF4FBF4F8093B8
:106D0000170D9093180DA093190DB0931A0D1092B2
:106D1000080CD093A00661E08C2F3DDF81E00E943B
:106D20009DB4BCCF81E090E090937F0680937E0677
:106D3000DF91CF9108954F925F926F927F928F92E1
:106D40009F92AF92BF92CF92DF92EF92FF920F93FA
:106D50001F93CF93DF935C014B01EA0189014090BF
:106D6000000250900102609002027090030228819C
:106D700039814A815B816091EE0B7091EF0B8091BC
:106D8000F00B9091F10B0E94DDC987FF29C0F8013B
:106D9000C080D180E280F38020E030E0A901C7010B
:106DA000B6010E94DDC9811106C0EBE7FEE0C59087
:106DB000D590E590F490C0920002D0920102E0924A
:106DC0000202F092030288819981AA81BB8180939B
:106DD000EE0B9093EF0BA093F00BB093F10B64DEEE
:106DE000F801C080D180E280F38020E030E0A9018A
:106DF000C701B6010E94DDC9811107C085E5C82E13
:106E0000DC2C85E0E82E83E4F82EC0920002D092BC
:106E10000102E0920202F0920302F5018081918169
:106E2000A281B3818093E60B9093E70BA093E80BCC
:106E3000B093E90BF40180819181A281B3818093A9
:106E4000EA0B9093EB0BA093EC0BB093ED0B2CDEC5
:106E5000288139814A815B816091EE0B7091EF0B43
:106E60008091F00B9091F10B0E941AD018164CF5FE
:106E7000F801C080D180E280F38020E030E0A901F9
:106E8000C701B6010E94DDC9811106C0EBE7FEE033
:106E9000C590D590E590F490C0920002D092010286
:106EA000E0920202F092030288819981AA81BB815B
:106EB0008093EE0B9093EF0BA093F00BB093F10B3C
:106EC000F3DD0E94A19A409200025092010260926A
:106ED000020270920302DF91CF911F910F91FF90F8
:106EE000EF90DF90CF90BF90AF909F908F907F906A
:106EF0006F905F904F90089580E1E6EEFBE0AEE684
:106F0000B6E001900D928A95E1F7089580E1EEE6F2
:106F1000F6E0A6EEBBE001900D928A95E1F70895A8
:106F2000CF92EF92FF920F931F93C09003067B01C5
:106F30008C012AE736E046E756E062E776E08EE627
:106F400096E00E9474831F910F91FF90EF90CF9075
:106F50000895CF92DF92EF92FF920F931F93CF93FA
:106F6000DF93EC01CC0FDD1FCC0FDD1FFE01EC52D7
:106F7000FA4F20E030E0A901608171818281938124
:106F80000E94F4CDFE01EF59F94F208131814281F9
:106F900053810E94F4CD6B017C01FE01EC5FF94F3F
:106FA0006083718382839383FE01E650F84F65917D
:106FB0007591859194918E01065E194FA7019601F6
:106FC0000E94F4CDF8016083718382839383FE0174
:106FD000EA5FF74F6591759185919491C55EDD4F9C
:106FE000A70196010E94F4CD688379838A839B83ED
:106FF000DF91CF911F910F91FF90EF90DF90CF9095
:107000000895FF920F931F93CF93DF93FC0120818C
:107010002B3319F1D0910206D430F8F4F62EBC01CE
:10702000C0915F050C2F10E0F0E6CF9FC001112446
:107030008E529C4F0E9421D1F801E052FA4FF0820B
:10704000CF5FC43018F4C0935F0502C010925F0593
:10705000DF5FD093020681E001C080E0DF91CF9135
:107060001F910F91FF900895DF92EF92FF920F937F
:107070001F93CF93DF93CDB7DEB76E970FB6F8941B
:10708000DEBF0FBECDBF6091100670911106611575
:10709000710501F14DE150E0CE0101967C010E94A5
:1070A0004DC91E8EF7018F010E191F09D190DD20E9
:1070B00019F09AE0D912F7CFF701E00FF11F108213
:1070C00060E0C7019EDF882329F0C7010E94EB5DC5
:1070D000811109C081E02091100630911106232B07
:1070E000A1F480E012C0DD2049F00F5F1F4F8091B6
:1070F000100690911106080F191F02C000E010E061
:107100001093110600931006E5CF6E960FB6F89413
:10711000DEBF0FBECDBFDF91CF911F910F91FF90CA
:10712000EF90DF90089522EF3BE04EEE5BE06AEED9
:107130007BE086EE9BE00C9487829F92AF92BF9299
:10714000CF92DF92EF92FF920F931F93CF93DF9333
:1071500000D01F92CDB7DEB7902EA12EB22ED32E27
:107160007C01EE0CFF1CEE0CFF1C87010A51144F32
:10717000F801108211821282138249835A836B8331
:107180007C83D1DF49815A816B817C81F801408306
:10719000518362837383C090030620E030E0A9012D
:1071A000692D7A2D8B2D9D2D0E94DDC9811108C07E
:1071B000F701ED58F14FE590F5900591149106C057
:1071C000892D9A2DAB2DBD2D7C018D0122EF3BE049
:1071D0004EEE5BE06AEE7BE086EE9BE00E947483FD
:1071E0000E94A19A109200060F900F900F900F909E
:1071F000DF91CF911F910F91FF90EF90DF90CF9093
:10720000BF90AF909F9008951F920F920FB60F926C
:1072100011248F9382E08093220D8F910F900FBEE7
:107220000F901F9018951F920F920FB60F92112476
:107230008F9382E08093220D8F910F900FBE0F905D
:107240001F9018951F920F920FB60F9211248F93D3
:1072500082E08093220D8F910F900FBE0F901F90B0
:10726000189580915D0590915E05009731F04AE098
:1072700050E060E070E00C94F9C760E070E0CB0192
:10728000089580915D0590915E05009731F04AE088
:1072900050E060E070E00C94D1C660E070E0CB019B
:1072A0000895EFDF97FD0AC0ECDF6F3F71058105A0
:1072B000910509F02CF4E5DF862F089580E008950C
:1072C0008FEF089580915D0590915E05892B31F0D7
:1072D000E8DF91E0811103C090E001C091E0892FC7
:1072E00008950F931F93CF9380915D0590915E0554
:1072F0000097F1F0FC018F01C1912C2F2F7D89F0B7
:10730000C53411F0C536B9F7F801108260E070E0BD
:107310000E946BC5F801C083562F472F382F292FA5
:107320000BC060E070E0CF911F910F910C946BC582
:1073300050E040E030E020E0652F742F832F922F43
:10734000CF911F910F91089581548A3150F5482FA4
:1073500050E0FA0193E0F595E7959A95E1F7E85347
:10736000FC4F208130E08770B90102C075956795A8
:107370008A95E2F760FF15C0FA01E255FC4F2081C3
:10738000222339F080914D0F90914E0F820F911D65
:1073900002C080E090E090935E0580935D0581E0FF
:1073A000089580E00895D0DF882341F081E02091A6
:1073B0005D0530915E05232B09F480E00895BF92AE
:1073C000CF92DF92EF92FF920F931F93CF93DF93B1
:1073D0008EE6E82E86E0F82E06EE1BE09DECC92E28
:1073E00093E0D92EC0EAD2E0BC2E84E0B80E899199
:1073F000ABDF8823D1F075DFF6012081211104C0B5
:107400002091D103222331F0F80120813181428182
:10741000538103C020E030E0A9010E94F4CDF701C0
:1074200060837183828393830AC0F8018081918194
:10743000A281B381F70180839183A283B383F4E0B7
:10744000EF0EF11C0C5F1F4F8FEFC81AD80ABC1249
:10745000CECF86E4A8DF8823B9F043DF20E030E018
:10746000A9010E941AD018167CF43BDF20E030E01E
:1074700040E752E40E94D0CE609300027093010274
:107480008093020290930302DF91CF911F910F919D
:10749000FF90EF90DF90CF90BF9008950E94FB691E
:1074A00060934F0F7093500F8093510F9093520F32
:1074B00008959091C00095FFFCCF8093C600089579
:1074C0008F929F92AF92BF92EF92FF921F93CF93B2
:1074D000DF93CDB7DEB7A0970FB6F894DEBF0FBE2F
:1074E000CDBF611571058105910579F110E0842EFC
:1074F000912CA12CB12CEE24E394F12CEC0EFD1E6A
:10750000E10EF11C17FDFA94A50194010E94B8CD7B
:10751000F7016083B901CA011F5F6115710581051B
:10752000910549F7115010F1E1E0F0E0EC0FFD1F7B
:10753000E10FF11D17FDFA9580818A3010F097E375
:1075400001C090E3890FB5DFEDCF80E3A0960FB6C1
:10755000F894DEBF0FBECDBFDF91CF911F91FF909A
:10756000EF90BF90AF909F908F90A3CFA0960FB653
:10757000F894DEBF0FBECDBFDF91CF911F91FF907A
:10758000EF90BF90AF909F908F900895EF92FF92F1
:107590000F931F93CF93DF937C0184E504DFD82FF3
:1075A000882321F17EDEC82F1816E4F4EFE7F9E016
:1075B00084918F010F5F1F4F882319F07ADFF80144
:1075C000F7CF8DE476DFB70180E090E04AE078DF26
:1075D0006C2FCC0F770B87EE97E00E9472758AE0D4
:1075E00068DF08C08093CC03D0E004C0809103061C
:1075F0008093CC038D2FDF91CF911F910F91FF903E
:10760000EF900895CF92DF92EF92FF926B017C0191
:1076100097FF0AC08DE24DDFF094E094D094C094BF
:10762000C11CD11CE11CF11C4AE0C701B601FF904E
:10763000EF90DF90CF9044CFEF92FF920F931F9384
:10764000CF93DF931F92CDB7DEB7082F162FE1E659
:10765000F8E084917F012FEFE21AF20A882329F0E3
:10766000998327DFF7019981F4CFE02FF92F8491D7
:107670007F019FEFE91AF90A882319F01ADFF70151
:10768000F6CF6091440F7091450F8091460F909115
:10769000470FB8DF8AE00DDF11110E9412B8109277
:1076A000C5051092C4050F90DF91CF911F910F91E6
:1076B000FF90EF900895DF92EF92FF920F931F9348
:1076C000CF93DF93D1DC811129C1809102068430F0
:1076D00008F024C184D99C0197FD20C1982FC09146
:1076E000C405D091C5058A3019F09D3009F0EBC072
:1076F0001092C605209749F3CC59DA4F18821092A0
:10770000C5051092C40524E635E0E90188812F5FA4
:107710003F4F8032D1F38E018E3411F000E010E043
:107720006AE270E0CE010E940DD17C0101151105C5
:1077300009F473C062EE77E0CE010E945CC9DD24DB
:10774000D394892B11F4D12C09C06EE470E0CE01E2
:1077500004960E940DD1009709F08C014AE050E098
:1077600060E070E0C80101960E94D1C66093600598
:107770007093610580936205909363050091440FB7
:107780001091450F2091460F3091470F0F5F1F4F0B
:107790002F4F3F4F601771078207930731F0D110C9
:1077A00004C061E08FEA97E03DC0E114F10401F10B
:1077B00080E010E0FE01E80FF11D90819A3219F08F
:1077C0008F5F1927F7CF4AE050E060E070E0C70113
:1077D00001960E94D1C6012F10E020E030E0601732
:1077E00071078207930741F061E080E997E01AC0D2
:1077F00061E086E697E016C0809160059091610592
:10780000A0916205B09163058093440F9093450F5A
:10781000A093460FB093470F0DC0892B59F060E03D
:1078200082EB96E0DF91CF911F910F91FF90EF9047
:10783000DF9002CF80917F02811121C067E470E068
:10784000CE010E940DD10097D1F04AE050E060E0F7
:1078500070E001960E94D1C66430710580F4EFEEAD
:10786000F6E084918F010F5F1F4F882319F021DE0E
:10787000F801F7CF60E085EE96E00E94946461E342
:1078800073E0CE010E9418D1892B21F410920402DA
:107890001092A00666E373E0CE010E9418D1892BF6
:1078A00021F48CED96E00E940C5E6BE373E0CE0158
:1078B0000E9418D1892B11F40E9442A761E084E64E
:1078C00095E09FDB02CFCF35D1050CF0FECE9C3585
:1078D00091F485D897FDF9CE2091C6052111F5CEFA
:1078E0009E012F5F3F4F3093C5052093C405CC59AF
:1078F000DA4F8883EACE9B3319F481E08093C60582
:107900008091C6058111E1CECE0101969093C50507
:107910008093C405CC59DA4F2883D7CEDF91CF911D
:107920001F910F91FF90EF90DF9008958F929F929B
:10793000AF92BF92CF92DF92EF92FF92CF936B0103
:107940007C01B42E20E030E0A9010E94DDC987FF50
:1079500006C08DE2AEDDF7FAF094F7F8F094C0E0DF
:1079600060E070E080E09FE3CB1541F02DEC3CEC53
:107970004CEC5DE30E9442CACF5FF6CF9B01AC01A5
:10798000C701B6010E94F4CD6B017C010E943DCF7E
:107990004B015C014AE094DDCC2379F1C501B401CF
:1079A0000E94E1C99B01AC01C701B6010E94F3CD61
:1079B0006B017C018EE27DDD20E030E040E251E4AD
:1079C000C701B6010E9442CA4B015C010E9438CF38
:1079D0006B01770FEE08FF08C701B60113DEC70180
:1079E000B6010E94E3C99B01AC01C501B4010E942C
:1079F000F3CD6B017C01C150F9F6CF91FF90EF9070
:107A0000DF90CF90BF90AF909F908F9008954F924E
:107A10005F926F927F928F929F92AF92BF92CF921E
:107A2000DF92EF92FF92CF93DF93E7E3F8E0849148
:107A3000EF012196882319F03CDDFE01F8CF60911B
:107A4000E60B7091E70B8091E80B9091E90B42E017
:107A50006DDFE3E3F8E08491EF012196882319F0CC
:107A600028DDFE01F8CF6091EA0B7091EB0B80915D
:107A7000EC0B9091ED0B42E059DFEFE2F8E08491DE
:107A8000EF012196882319F014DDFE01F8CF6091F3
:107A9000EE0B7091EF0B8091F00B9091F10B42E0A7
:107AA00045DFEBE2F8E08491EF012196882319F09D
:107AB00000DDFE01F8CF6091F20B7091F30B809125
:107AC000F40B9091F50B42E031DF8FB7F8944090C2
:107AD000D60B5090D70B6090D80B7090D90B80903C
:107AE000DA0B9090DB0BA090DC0BB090DD0BC0901C
:107AF000DE0BD090DF0BE090E00BF090E10B8FBF3E
:107B0000E1E2F8E08491EF012196882319F0D1DCBD
:107B1000FE01F8CFC301B20175DDEDE1F8E084911B
:107B2000EF012196882319F0C4DCFE01F8CFC501CE
:107B3000B40168DDE9E1F8E08491EF012196882342
:107B400019F0B7DCFE01F8CFC701B6015BDD8AE0B2
:107B5000DF91CF91FF90EF90DF90CF90BF90AF90EB
:107B60009F908F907F906F905F904F90A2CC8F925C
:107B70009F92AF92BF92CF92DF92EF92FF92CF93FC
:107B8000DF936091400670914106072E000C880B30
:107B9000990B0E94E3C96B017C01809012069090C2
:107BA0001306A0901406B090150680E282DC84E5EE
:107BB00080DC8AE37EDC42E0C501B401B7DEB701B8
:107BC000A60182E198E00E945575E5E1F8E0849114
:107BD000EF012196882319F06CDCFE01F8CFE091CB
:107BE000CC03F0E0EB5DF24F608170E080E090E06C
:107BF000DF91CF91FF90EF90DF90CF90BF90AF904B
:107C00009F908F90FFCC1F920F920FB60F9211246E
:107C10000BB60F922F938F939F93EF93FF93E09167
:107C2000420F81E08E0F8F779091C6002091430F15
:107C3000821731F0F0E0EE53F14F90838093420FC2
:107C4000FF91EF919F918F912F910F900BBE0F900D
:107C50000FBE0F901F901895CF92DF92EF92FF9278
:107C60000F931F93CF93DF936C017A018B01C0E0D8
:107C7000D0E0CE15DF0589F0D8016D918D01D601D8
:107C8000ED91FC910190F081E02DC6011995892BB1
:107C900011F47E0102C02196ECCFC701DF91CF9194
:107CA0001F910F91FF90EF90DF90CF9008950E9469
:107CB00009D11F93CF93DF9310929D068091BC0B47
:107CC0009091BD0BA091BE0BB091BF0B813090483D
:107CD000A105B10540F01092BC0B1092BD0B1092A3
:107CE000BE0B1092BF0BC091BC0B809130061816D2
:107CF000DCF4282F082E000C330B215031094C2FB7
:107D00000C2E000C550B4217530774F0CFEFC80F21
:107D10008C2F90E0A0E0B0E08093BC0B9093BD0B63
:107D2000A093BE0BB093BF0B1092B80C8091560677
:107D3000C81714F4C093560680915606082E000CFE
:107D4000990B04962C2F0C2E000C330B82179307E3
:107D500024F48CEF8C0F8093560610915606D0E0D9
:107D600011111AC080919F06811106C080913B02BB
:107D7000882309F48DC009C0C111F8CF0E94E8938F
:107D80008091B80C882391F38AC081E0C11180E012
:107D900024E046EC5AE079C01130E9F480919F0666
:107DA000811106C080913B02882309F471C00BC089
:107DB000C130C1F78BED90E40E94BEC18091B80C38
:107DC000882381F36CC081E0C13009F080E023E0BA
:107DD0004FEB5AE05AC01230E9F480919F068111AE
:107DE00006C080913B02882309F452C00BC0C23008
:107DF000C1F780EE90E40E94BEC18091B80C882348
:107E000081F34DC081E0C23009F080E023E048EB0F
:107E10005AE03BC01330E1F480919F06811105C008
:107E200080913B028823A1F10BC0C330C9F785EED6
:107E300090E40E94BEC18091B80C882389F32FC0C2
:107E400081E0C33009F080E023E041EB5AE01DC03F
:107E50001430F1F480919F06811105C080913B029E
:107E60008823B1F00BC0C430C9F78AEE90E40E94B9
:107E7000BEC18091B80C882389F311C081E0C43061
:107E800009F080E023E048EA5AE06D2F0E94DE63AB
:107E9000DF5F1F5FD53009F063CFD0933006DF91ED
:107EA000CF911F910895EF92FF921F93CF93DF938D
:107EB0007C0170932F0660932E0610929D06809190
:107EC000BC0B9091BD0BA091BE0BB091BF0B81304C
:107ED0009048A105B10540F01092BC0B1092BD0B6B
:107EE0001092BE0B1092BF0BC091BC0B80912D065F
:107EF0001816DCF4282F082E000C330B2150310902
:107F00004C2F0C2E000C550B4217530774F0CFEF7B
:107F1000C80F8C2F90E0A0E0B0E08093BC0B909352
:107F2000BD0BA093BE0BB093BF0B1092B80C809109
:107F30005606C81714F4C093560620915606022E12
:107F4000000C330B2C5F3F4F8C2F0C2E000C990B29
:107F50002817390724F48CEF8C0F80935606109164
:107F60005606D0E091E081E0E816F10469F122E0E4
:107F7000E216F10409F44CC0E114F10409F06CC0FC
:107F8000111191C09923B1F01C16A4F08091BC0B83
:107F90009091BD0BA091BE0BB091BF0B0196A11D9E
:107FA000B11D8093BC0B9093BD0BA093BE0BB093FF
:107FB000BF0BCF5F80913B02882309F4EEC021E024
:107FC00041E061EA7AE06BC011116DC09923B1F014
:107FD0001C16A4F08091BC0B9091BD0BA091BE0B20
:107FE000B091BF0B0196A11DB11D8093BC0B909366
:107FF000BD0BA093BE0BB093BF0BCF5F80913B0234
:10800000882309F4CAC021E041E06AE97AE047C068
:10801000111149C09923B1F01C16A4F08091BC0B3A
:108020009091BD0BA091BE0BB091BF0B0196A11D0D
:10803000B11D8093BC0B9093BD0BA093BE0BB0936E
:10804000BF0BCF5F80913B02882309F4A6C021E0DB
:1080500041E063E97AE023C0111125C09923B1F012
:108060001C16A4F08091BC0B9091BD0BA091BE0B8F
:10807000B091BF0B0196A11DB11D8093BC0B9093D5
:10808000BD0BA093BE0BB093BF0BCF5F80913B02A3
:10809000882309F482C021E041E06AE87AE08D2F6C
:1080A0000E94D0C27AC01130D9F480919F0681110C
:1080B00006C080913B02882309F46FC009C0C1301B
:1080C000C1F70E94E8938091B80C882391F36DC0AA
:1080D00081E0C13009F080E024E040E85AE05AC075
:1080E0001230E9F480919F06811106C080913B0215
:1080F000882309F452C00BC0C230C1F783E091E479
:108100000E94BEC18091B80C882381F34EC081E0EB
:10811000C23009F080E023E046E75AE03BC013306C
:10812000E1F480919F06811105C080913B02882374
:10813000A1F10BC0C330C9F788E091E40E94BEC131
:108140008091B80C882389F330C081E0C33009F0F6
:1081500080E023E04DE65AE01DC01430F1F4809138
:108160009F06811105C080913B028823B1F00BC0AE
:10817000C430C9F78DE091E40E94BEC18091B80C73
:10818000882389F312C081E0C43009F080E023E045
:1081900042E65AE06D2F0E94DE63DF5F1F5F90E0D2
:1081A000D53009F0E0CED0932D06DF91CF911F910D
:1081B000FF90EF9008956BEA72E480E090E073CE58
:1081C00066EA72E481E090E06ECE61EA72E482E0F9
:1081D00090E069CE68E471E483E090E064CE21E051
:1081E000209398066093290670932A0680932B06A5
:1081F00090932C0640E050E0BA0180912E069091B9
:108200002F060C944D9060E070E080E291E4E7CF9F
:1082100060E070E080E89FE3E2CF6DEC7CEC8CECFA
:108220009DE3DDCFCF92DF92EF92FF92CF93C82FE5
:108230000E94FB696B017C0124EA30E74DE75FE3B4
:108240006091290670912A0680912B0690912C0648
:108250000E94DDC987FD05C04AEF50E060E070E094
:1082600003C040E050E0BA01C40ED51EE61EF71E62
:10827000C0929006D0929106E0929206F0929306F8
:10828000C0933602CF91FF90EF90DF90CF9008958A
:1082900080919F0681110C94E8936091BC0B7091C2
:1082A000BD0B8091BE0B9091BF0B611571058105CF
:1082B000910571F10E94E3C92091290630912A06A7
:1082C00040912B0650912C060E9442CA9B01AC01A2
:1082D0006091F20B7091F30B8091F40B9091F50B80
:1082E0000E94F4CD6093F20B7093F30B8093F40B28
:1082F0009093F50B83E090E095DF81E080933B0263
:108300001092BC0B1092BD0B1092BE0B1092BF0BC3
:1083100080913B02882349F082EF9BE00E944962F2
:10832000BC0189E59AE00C94FD9308952F923F9249
:108330004F925F926F927F928F929F92AF92BF9275
:10834000CF92DF92EF92FF920F931F93CF93DF9321
:10835000CDB7DEB72A970FB6F894DEBF0FBECDBFFC
:108360009A8789871B0180919F06882319F00E94B4
:10837000E893CEC08091BC0B9091BD0BA091BE0B39
:10838000B091BF0B892B8A2B8B2B09F490C086D818
:108390008101000F111F000F111FF801EA51F44F66
:1083A000408051806280738080912702811115C0C6
:1083B00020E030E04AE754E4C301B2010E94F3CD6B
:1083C0004B015C0120E030E04AE754E4C301B20114
:1083D0000E94F4CD6B017C010EC0F801E65EF94FFE
:1083E00080809180A280B380F801E55EFD4FC0805F
:1083F000D180E280F3802091BC0B3091BD0B409185
:10840000BE0B5091BF0B2D833E834F835887CA010B
:10841000B9010E94E3C92091290630912A064091B2
:108420002B0650912C060E9442CA9B01AC01C3014D
:10843000B2010E94F4CD0A51144FD8016D937D937F
:108440008D939C9313972D813E814F81588557FFC3
:108450000DC0A50194010E94DDC987FF1BC0D80192
:108460008D929D92AD92BC92139714C02D813E8146
:108470004F815885232B242B252B61F0A7019601D2
:108480000E941AD0181634F4D801CD92DD92ED92E4
:10849000FC9213971092BC0B1092BD0B1092BE0B66
:1084A0001092BF0BC101BEDE81E080933B02809140
:1084B0003B02882369F1F101EE0FFF1FEE0FFF1F52
:1084C000EA51F44F80819181A281B38189839A839B
:1084D000AB83BC832DEC3CEC4CEC5DE36091290656
:1084E00070912A0680912B0690912C060E941AD03A
:1084F00087FD05C0CE0101960E94496204C0CE01ED
:1085000001960E94597ABC0189859A850E94FD9343
:108510002A960FB6F894DEBF0FBECDBFDF91CF9184
:108520001F910F91FF90EF90DF90CF90BF90AF9091
:108530009F908F907F906F905F904F903F902F9083
:10854000089562E070E082E59AE0F0CE61E070E0CC
:108550008BE49AE0EBCE60E070E084E49AE0E6CE53
:108560002F923F924F925F926F927F928F929F9243
:10857000AF92BF92CF92DF92EF92FF920F931F9331
:10858000CF93DF9310929D068091BC0B9091BD0B11
:10859000A091BE0BB091BF0B81309048A105B105F1
:1085A00040F01092BC0B1092BD0B1092BE0B1092BB
:1085B000BF0BC091BC0B809128061816DCF4282F45
:1085C000082E000C330B215031094C2F0C2E000CBF
:1085D000550B4217530774F0CFEFC80F8C2F90E064
:1085E000A0E0B0E08093BC0B9093BD0BA093BE0BBA
:1085F000B093BF0B1092B80C80915606C81714F4B4
:10860000C093560680915606082E000C990B0496CE
:108610002C2F0C2E000C330B8217930724F48CEFB5
:108620008C0F809356061091560600E047E0642EAA
:108630004AE0742E54E1452E5AE0552E61E2E62EB2
:108640006AE0F62E71E3C72E7AE0D72EE6E9AE2E69
:10865000E9E0BE2EF1ED8F2EF9E09F2E11111AC028
:1086600080919F06811106C080913B02882309F406
:10867000B4C009C0C111F8CF0E94E8938091B80C32
:10868000882391F318C281E0C11180E024E04FE318
:108690005AE0A0C01130E9F480919F06811106C014
:1086A00080913B02882309F498C00BC0C130C1F708
:1086B00089E59EE30E94BEC18091B80C882381F3B6
:1086C000FAC181E0C13009F080E023E045E35AE0DF
:1086D00081C01230F9F480919F06811106C080910B
:1086E0003B02882309F479C00DC0C230C1F7D09293
:1086F0001106C09210060E9434388091B80C88236D
:1087000071F3D9C181E0C23009F080E020E247E294
:108710005AE060C01330F9F480919F06811106C0C1
:1087200080913B02882309F458C00DC0C330C1F7C3
:10873000F0921106E09210060E9434388091B80C35
:10874000882371F3B8C181E0C33009F080E020E2F2
:108750004AE15AE03FC01430F1F480919F06811144
:1087600005C080913B028823C1F10DC0C430C9F718
:1087700050921106409210060E9434388091B80C35
:10878000882379F398C181E0C43009F080E020E2C9
:108790004DE05AE01FC0153001F580919F06811110
:1087A00005C080913B028823C1F00DC0C530C9F7D8
:1087B00070921106609210060E9434388091B80CB5
:1087C000882379F378C181E0C53009F080E020E2A8
:1087D00040E05AE0602F0E94DE63809117068823F4
:1087E000A1F180911806882381F1809119068823D0
:1087F00061F1163069F580919F06811106C0809164
:108800003B02882309F43AC115C0C630C1F781E0A4
:108810008093980640E050E0BA018EE695E40E940D
:108820004D90109227060E9432BF8091B80C882389
:1088300031F341C181E0C63009F080E020E242EF2F
:1088400059E0602F0E94DE6319C136E0332E02C06A
:1088500027E0322E131122C080919F06811105C09E
:1088600080913B028823C9F00FC0C113F9CFB092A9
:108870001106A09210060E9434380E94E293809163
:10888000B80C882369F317C181E0C11380E020E2AE
:1088900045ED59E0602F0E94DE63312E81E0830DAB
:1088A00018131FC080919F06811105C080913B0263
:1088B0008823B9F00DC0C113F9CF909211068092B0
:1088C00010060E9434388091B80C882379F3F3C0E5
:1088D00081E0C11380E020E240EC59E0602F0E946B
:1088E000DE63D2E0D30D80911606811118C060912D
:1088F000190270911A02072E000C880B990B0E9426
:10890000E3C99B01AC01609112067091130680913E
:108910001406909115060E94DDC987FD1FC01D1326
:108920001BC080919F06811105C080913B02882366
:1089300099F009C0C113F9CF0E9412B28091B80C0E
:10894000882399F3B8C081E0C11380E020E240EBB6
:1089500059E0602F0E94DE63D3E0D30D8091400682
:1089600090914106892B59F01D1308C080919F06F4
:10897000811187C080913B02811193C0DF5F1D137D
:1089800037C080919F06811105C080913B028823EA
:1089900079F125C0C113F9CF2090460630904706E3
:1089A0008091420690914306181619066CF48431A2
:1089B00021E0920714F083E191E0909341068093C7
:1089C000400680E00E94BC9630923F0620923E0610
:1089D0000E94E2938091B80C8823B9F26CC081E0C8
:1089E000C11380E020E24BE959E0602F0E94DE6372
:1089F00081E08D0F181337C080919F06811105C04B
:108A000080913B02882379F125C0C113F9CF2090D2
:108A10004806309049068091440690914506181604
:108A200019066CF4843121E0920714F083E191E09F
:108A3000909341068093400680E00E94BC9630925D
:108A40003F0620923E060E94E2938091B80C882354
:108A5000B9F231C081E0C11380E020E246EE59E076
:108A6000602F0E94DE630F5F1F5F053009F0F6CDB7
:108A700092E0492E4D0E409228061DC087E0382E08
:108A80000DCFC11377CF10923F0610923E060E9481
:108A900007970E94E2938091B80C882309F46ACF6B
:108AA0000AC081E0C11380E020E247EA59E0602F6C
:108AB0000E94DE6363CFDF91CF911F910F91FF90F2
:108AC000EF90DF90CF90BF90AF909F908F907F906E
:108AD0006F905F904F903F902F9008951F93CF938A
:108AE000DF9310929D068091BC0B9091BD0BA091DD
:108AF000BE0BB091BF0B81309048A105B10540F08D
:108B00001092BC0B1092BD0B1092BE0B1092BF0BBB
:108B1000C091BC0B809126061816DCF4282F082E75
:108B2000000C330B215031094C2F0C2E000C550B2F
:108B30004217530774F0CFEFC80F8C2F90E0A0E0DE
:108B4000B0E08093BC0B9093BD0BA093BE0BB09391
:108B5000BF0B1092B80C80915606C81714F4C0933E
:108B6000560680915606082E000C990B04962C2F61
:108B70000C2E000C330B8217930724F48CEF8C0F10
:108B80008093560610915606D0E08D2F810FC9F4C0
:108B900080919F06811105C080913B02882389F155
:108BA00009C0C111F9CF0E9432BF8091B80C88234F
:108BB00099F32EC081E0C11180E020E24AE859E03B
:108BC0001DC08130F1F480919F06811105C0809114
:108BD0003B028823B1F00BC0C130C9F71092980650
:108BE0000E94E8938091B80C882389F311C081E03A
:108BF000C13009F080E020E245E859E06D2F0E9485
:108C0000DE63DF5FD53009F0C0CF82E080932606B7
:108C1000DF91CF911F9108952CEA35EC47E25EE396
:108C200060914C0670914D0680914E0690914F06D2
:108C30000E94D0CE60933506709336068093370637
:108C40009093380608952CEA35EC47E25EE3609194
:108C500050067091510680915206909153060E94E1
:108C600042CA6093390670933A0680933B0690930C
:108C70003C0608952F923F924F925F926F927F929F
:108C80008F929F92AF92BF92DF92EF92FF920F93DB
:108C90001F93CF93DF9310929D068091BC0B909110
:108CA000BD0BA091BE0BB091BF0B81309048A105C8
:108CB000B10540F01092BC0B1092BD0B1092BE0B90
:108CC0001092BF0BC091BC0B809154061816DCF4B7
:108CD000282F082E000C330B215031094C2F0C2E5D
:108CE000000C550B4217530774F0CFEFC80F8C2FB1
:108CF00090E0A0E0B0E08093BC0B9093BD0BA093FC
:108D0000BE0BB093BF0B1092B80C80915606C817DB
:108D100014F4C093560680915606082E000C990B49
:108D200004962C2F0C2E000C330B8217930724F47F
:108D30008CEF8C0F80935606D0905606D0E055EEFF
:108D4000252E5BE0352E66E9862E912CA12CB12CC8
:108D50007EE6472E512C612C712CD1101DC08091C4
:108D60009F06811106C080913B02882309F4D6C179
:108D700009C0C111F8CF0E94E8938091B80C8823F4
:108D800091F367C381E0C11180E024E046E25CE03A
:108D90006D2F0E94DE63C2C181E0D8126EC0809147
:108DA0009F06811106C080913B02882309F4B6C159
:108DB00055C0C130C1F7C0939D061092990610921C
:108DC0009A0610929B0610929C060E942D9083E0BA
:108DD00080933B028FE19CE09093CB0B8093CA0B76
:108DE00080E496E09093C90B8093C80B1092C40B5B
:108DF0001092C50B1092C60B1092C70B84E091E045
:108E0000A0E0B0E08093C00B9093C10BA093C20B85
:108E1000B093C30B8091400690914106092E000C3F
:108E2000AA0BBB0B8093BC0B9093BD0BA093BE0B06
:108E3000B093BF0B86ED90E590933A028093390290
:108E40008BE791EB9093BB0B8093BA0B1092B90B0D
:108E50008091B80C882309F4A6CFFBC2809140060C
:108E6000909141060E9476639C0181E0C13009F037
:108E700080E000E048E15CE04EC192E0D91235C0EC
:108E800080919F06811106C080913B02882309F4DE
:108E900045C11CC0C230C1F781E080939D0610928D
:108EA000990610929A0610929B0610929C062FEF3C
:108EB00030E040E050E06EE376E08EE09CE00E941F
:108EC0003FC08091B80C8823F9F2C3C280913E065E
:108ED00090913F060E9476639C0181E0C23009F0C8
:108EE00080E000E044E05CE016C1A3E0DA1229C0B3
:108EF00080919F06811105C080913B02811110C0B5
:108F00000DC1C330C9F790913D0681E08927809358
:108F10003D06C0933B028091B80C882369F399C247
:108F200080913D06811103C023EF3BE002C027EF93
:108F30003BE081E0C33009F080E001E04BEF5BE013
:108F4000EAC0B4E0DB123FC080919F06811106C0E9
:108F500080913B02882309F4E1C014C0C430C1F7FA
:108F6000E12CF12C02E813E420E030E0A90162E3F7
:108F700072E08CEE9BE00E94C8BF8091B80C882301
:108F800039F367C281E08F9384E08F931F921F9221
:108F900082E392E09F938F93AEEDBBE0BF93AF93DC
:108FA0003F922F92DF9381E0C43009F080E08F93ED
:108FB0000E94E6C48DB79EB70C960FB6F8949EBF7C
:108FC0000FBE8DBFABC095E0D91241C080919F0606
:108FD000811106C080913B02882309F49FC014C010
:108FE000C530C1F7E12CF12C02E813E420E030E0B9
:108FF000A9016EE272E087ED9BE00E94C8BF8091FC
:10900000B80C882339F325C281E08F9384E08F93D5
:109010001F921F928EE292E09F938F93A9ECBBE088
:10902000BF93AF93A0EDBBE0BF93AF93DF9381E01D
:10903000C53009F080E08F930E94E6C48DB79EB7DB
:109040000C960FB6F8949EBF0FBE8DBF67C096E01A
:10905000D91264C080919F06811106C080913B02A5
:10906000882309F45BC04BC0C630C1F70E942D9025
:1090700083E080933B02A1ECBBE0B093CB0BA093C9
:10908000CA0B8AE292E09093C90B8093C80B1092AE
:10909000C40B1092C50B1092C60B1092C70B84E63E
:1090A00090E0A0E0B0E08093C00B9093C10BA09340
:1090B000C20BB093C30B20E030E048EC52E4609167
:1090C0002A0270912B0280912C0290912D020E9415
:1090D00042CA0E943DCF6093BC0B7093BD0B80933E
:1090E000BE0B9093BF0BA5E0BFE4B0933A02A093F0
:1090F00039028091B80C882309F4B0CFAAC18AE262
:1091000092E00E9491629C0181E0C63009F080E00B
:1091100000E049EB5BE06D2F0E9476C42CEA35EC51
:1091200047E25EE36091390670913A0680913B0612
:1091300090913C060E94D0CE6093500670935106E9
:1091400080935206909353062CEA35EC47E25EE397
:1091500060913506709136068091370690913806F9
:109160000E9442CA60934C0670934D0680934E064F
:1091700090934F06B7E0DB1233C080919F068111B8
:1091800006C080913B02882309F45BC11CC0C73034
:10919000C1F7E12C18E1F12E0CE116E420E030E0FB
:1091A00040E85FE361E376E083EB9BE00E94D3C19C
:1091B0008EE99EE590933A02809339028091B80C33
:1091C0008823F9F246C181E396E00E945F609C012A
:1091D00081E0C73009F080E000E04DEA5BE07BC051
:1091E00028E0D2123BC080919F06811106C0809179
:1091F0003B02882309F425C124C0C830C1F7E12C03
:1092000018E1F12E0CE116E42AE037ED43E25CE3CD
:1092100060E576E087EA9BE00E94D3C184E99EE5A1
:1092200090933A028093390283E296E49093BB0BC9
:109230008093BA0B1092B90B8091B80C8823B9F2C5
:1092400008C180E596E00E945F609C0181E0C83023
:1092500009F080E000E041EA5BE03DC089E0D8121F
:109260003EC080919F06811106C080913B028823F9
:1092700009F4E7C024C0C930C1F7E12C18E1F12E90
:109280000CE116E420E030E040E85FE36CE476E0D7
:109290008BE99BE00E94D3C184E99EE590933A025A
:1092A000809339028CE096E49093BB0B8093BA0BC9
:1092B0001092B90B8091B80C8823B9F2CAC08CE423
:1092C00096E00E945F609C0181E0C93009F080E077
:1092D00000E045E95BE06D2F0E9476C4B2C09AE0E1
:1092E000D9126FC080919F06811106C080913B0208
:1092F000882309F4A6C056C0CA30C1F781E0809324
:109300009D061092990610929A0610929B06109252
:109310009C060E942D9083E080933B0288E89BE0AE
:109320009093CB0B8093CA0B88E292E09093C90B89
:109330008093C80B8092C40B9092C50BA092C60B71
:10934000B092C70B4092C00B5092C10B6092C20BFF
:109350007092C30B8091280290912902092E000C73
:10936000AA0BBB0B86599109A109B1098093BC0BCB
:109370009093BD0BA093BE0BB093BF0B86ED90E511
:1093800090933A02809339028BE39AE49093BB0B5B
:109390008093BA0B1092B90B8091B80C882309F412
:1093A000A5CF57C080912802909129020E94766330
:1093B0009C0181E0CA3009F080E000E04BE75BE00F
:1093C0008ACFABE0DA121CC080919F06811105C0E4
:1093D00080913B028823A9F10BC0CB30C9F784E907
:1093E00090EB0E94BEC18091B80C882389F331C0F4
:1093F00081E0CB3009F080E023E04AE65BE01EC06C
:10940000BCE0DB121EC080919F06811105C08091D7
:109410003B028823B1F00BC0CC30C9F781E990EB57
:109420000E94BEC18091B80C882389F312C081E0EC
:10943000CC3009F080E023E049E55BE06D2F0E942D
:10944000DE63DF5FD394D53009F087CC8DE0809365
:109450005406DF91CF911F910F91FF90EF90DF9015
:10946000BF90AF909F908F907F906F905F904F9044
:109470003F902F9008950F931F93CF93DF93CDB715
:10948000DEB76E970FB6F894DEBF0FBECDBF8091EA
:1094900029028F93809128028F931F921F9289E453
:1094A0009BE09F938F938E010F5F1F4F1F930F932E
:1094B0000E9476C960E0C8010E9401380FB6F89496
:1094C000DEBF0FBECDBF882319F0C8010E94EB5D3F
:1094D0006E960FB6F894DEBF0FBECDBFDF91CF9171
:1094E0001F910F9108951F93CF93DF9310929D06C4
:1094F0008091BC0B9091BD0BA091BE0BB091BF0BA6
:1095000081309048A105B10540F01092BC0B10923B
:10951000BD0B1092BE0B1092BF0BC091BC0B809183
:109520004B061816DCF4282F082E000C330B2150A4
:1095300031094C2F0C2E000C550B4217530774F0B9
:10954000CFEFC80F8C2F90E0A0E0B0E08093BC0B71
:109550009093BD0BA093BE0BB093BF0B1092B80CB1
:1095600080915606C81714F4C0935606809156068B
:10957000082E000C990B04962C2F0C2E000C330B8C
:109580008217930724F48CEF8C0F8093560610916A
:109590005606D0E011111AC080919F06811106C0B5
:1095A00080913B02882309F4F3C009C0C111F8CFB0
:1095B0000E94E8938091B80C882391F3F1C081E078
:1095C000C11180E024E044E45BE0DFC01130E9F445
:1095D00080919F06811106C080913B02882309F487
:1095E000D7C00BC0C130C1F78AE396E40E94BEC168
:1095F0008091B80C882381F3D3C081E0C13009F099
:1096000080E023E048E35BE0C0C01230E9F48091E1
:109610009F06811106C080913B02882309F4B8C0DF
:109620000BC0C230C1F78BE29EE70E94BEC18091A1
:10963000B80C882381F3B4C081E0C23009F080E027
:1096400023E041E35BE0A1C01330E9F480919F0681
:10965000811106C080913B02882309F499C00BC098
:10966000C330C1F788EC9CE70E94BEC18091B80C62
:10967000882381F395C081E0C33009F080E023E0C6
:1096800048E25BE082C01430D9F480919F068111DA
:1096900006C080913B02882309F47AC009C0C43017
:1096A000C1F70E94BBBF8091B80C882391F378C0AA
:1096B00081E0C43009F080E020E249E15BE065C070
:1096C000153041F580919F06811106C080913B02C3
:1096D000882309F45DC016C0C530C1F70E947BA283
:1096E000882319F00E94CE6308C048EB51E064E182
:1096F00070E080E090E00E943EB48091B80C882336
:1097000029F34EC081E0C53009F080E020E249EF46
:109710005AE03BC01630E1F480919F06811105C0EC
:1097200080913B028823A1F10BC0C630C9F70E948B
:109730005EA10E94CE638091B80C882389F330C06B
:1097400081E0C63009F080E020E248EE5AE01DC01A
:109750001730F1F480919F06811105C080913B0282
:109760008823B1F00BC0C730C9F784ED9BE40E9499
:10977000BEC18091B80C882389F312C081E0C73044
:1097800009F080E023E047E05BE06D2F0E94DE639C
:10979000DF5F1F5FD53009F0FDCE88E080934B0678
:1097A000DF91CF911F9108951F93CF93DF93109274
:1097B0009D068091BC0B9091BD0BA091BE0BB0910A
:1097C000BF0B81309048A105B10540F01092BC0B51
:1097D0001092BD0B1092BE0B1092BF0BC091BC0B30
:1097E00080914A061816DCF4282F082E000C330B43
:1097F000215031094C2F0C2E000C550B42175307EA
:1098000074F0CFEFC80F8C2F90E0A0E0B0E0809311
:10981000BC0B9093BD0BA093BE0BB093BF0B1092EB
:10982000B80C80915606C81714F4C0935606809160
:109830005606082E000C990B04962C2F0C2E000CAB
:10984000330B8217930724F48CEF8C0F809356060A
:1098500010915606D0E08D2F810FC9F480919F069C
:10986000811105C080913B028823A9F109C0C11173
:10987000F9CF0E94E8938091B80C882399F332C005
:1098800081E0C11180E024E040EE5AE021C0813047
:1098900011F580919F06811105C080913B028823BC
:1098A000D1F00FC0C130C9F70E945EA10E94CE6303
:1098B0000E94D6560E94E8938091B80C882369F3E1
:1098C00011C081E0C13009F080E020E24EEC5AE0A6
:1098D0006D2F0E94DE63DF5FD53009F0BCCF82E0E0
:1098E00080934A06DF91CF911F910895CF92DF9226
:1098F000EF92FF920F931F93CF93DF9310929D06E9
:109900004091BC0B5091BD0B6091BE0B7091BF0B91
:10991000413050486105710540F01092BC0B109227
:10992000BD0B1092BE0B1092BF0BC091BC0B90915F
:1099300055061916DCF4292F092E000C330B215083
:1099400031094C2F0C2E000C550B4217530774F0A5
:10995000CFEFC90F4C2F50E060E070E04093BC0B9C
:109960005093BD0B6093BE0B7093BF0B1092B80C5D
:1099700090915606C91714F4C093560620915606C6
:10998000022E000C330B2C5F3F4F4C2F0C2E000C83
:10999000550B2417350724F49CEF9C0F9093560623
:1099A00010915606D0E0E82EF12CC701880F991FC0
:1099B000FC01EE5BF94F6F019C012A5B394F790185
:1099C00011111AC080919F06811106C080913B023F
:1099D000882309F486C009C0C111F8CF0E94E8931A
:1099E0008091B80C882391F384C081E0C11180E09C
:1099F00024E04FE55CE072C0113041F580919F0694
:109A0000811106C080913B02882309F46AC010C00E
:109A1000C130C1F72FEF30E040E050E0B70185E5FD
:109A20009CE00E943FC08091B80C882359F361C02C
:109A3000F701808191810E9476639C0181E0C130B1
:109A400009F080E000E04BE45CE029C0123059F5F9
:109A500080919F06811106C080913B02882309F402
:109A600040C010C0C230C1F724E031E045E050E012
:109A7000B60184E49CE00E943FC08091B80C88232A
:109A800059F337C0F601808191810E9476639C0171
:109A900081E0C23009F080E000E04DE35CE06D2F32
:109AA0000E9476C41EC01330E1F480919F0681119C
:109AB00005C080913B028823A1F009C0C330C9F7DB
:109AC0000E94BBBF8091B80C882399F312C081E03B
:109AD000C33009F080E020E24EE25CE06D2F0E948E
:109AE000DE63DF5F1F5FD53009F06ACF84E08093CB
:109AF0005506DF91CF911F910F91FF90EF90DF906E
:109B0000CF900895CF92DF92EF92FF920F931F9321
:109B1000CF93DF9300D01F92CDB7DEB78091BC0BFF
:109B20009091BD0BA091BE0BB091BF0BB7FF08C0C9
:109B30001092BC0B1092BD0B1092BE0B1092BF0B7B
:109B40008091C00B9091C10BA091C20BB091C30B3F
:109B50004091BC0B5091BD0B6091BE0B7091BF0B3F
:109B600084179507A607B70744F48093BC0B90931E
:109B7000BD0BA093BE0BB093BF0B80913B0288231B
:109B800079F14091BC0B5091BD0B6091BE0B70916F
:109B9000BF0B8091C40B9091C50BA091C60BB091E7
:109BA000C70B6A017B01C80ED91EEA1EFB1EC70146
:109BB000B6010E94E3C920E030E048EC52E40E9484
:109BC00042CA69837A838B839C83CE0101960E946B
:109BD000E060BC018091CA0B9091CB0B0E94FD9379
:109BE00080919F061091B90B811106C01123D1F10C
:109BF00080913B028823B1F14091BC0B5091BD0B89
:109C00006091BE0B7091BF0B8091C40B9091C50BFE
:109C1000A091C60BB091C70B6A017B01C80ED91E7B
:109C2000EA1EFB1EC701B6010E94E3C920E030E036
:109C300048EC52E40E9442CAE091C80BF091C90B73
:109C4000309721F06083718382839383112329F0FD
:109C5000E091BA0BF091BB0B199580919F06811191
:109C60000E94E8930F900F900F900F90DF91CF918B
:109C70001F910F91FF90EF90DF90CF900895CF92BA
:109C8000DF92EF92FF920F931F93CF93DF9300D059
:109C90001F92CDB7DEB78091BC0B9091BD0BA09108
:109CA000BE0BB091BF0BB7FF08C01092BC0B109257
:109CB000BD0B1092BE0B1092BF0B8091C00B909108
:109CC000C10BA091C20BB091C30B4091BC0B509142
:109CD000BD0B6091BE0B7091BF0B84179507A60753
:109CE000B70744F48093BC0B9093BD0BA093BE0BBD
:109CF000B093BF0B80913B02882379F14091BC0B5C
:109D00005091BD0B6091BE0B7091BF0B8091C40B45
:109D10009091C50BA091C60BB091C70B6A017B0156
:109D2000C80ED91EEA1EFB1EC701B6010E94E3C978
:109D30002FE632E143E85AE30E9442CA69837A83FC
:109D40008B839C83CE0101960E94597ABC0180913D
:109D5000CA0B9091CB0B0E94FD9380919F061091AE
:109D6000B90B811106C01123D1F180913B028823E8
:109D7000B1F14091BC0B5091BD0B6091BE0B709145
:109D8000BF0B8091C40B9091C50BA091C60BB091F5
:109D9000C70B6A017B01C80ED91EEA1EFB1EC70154
:109DA000B6010E94E3C92FE632E143E85AE30E947C
:109DB00042CAE091C80BF091C90B309721F0608343
:109DC000718382839383112329F0E091BA0BF09180
:109DD000BB0B199580919F0681110E94E893809199
:109DE0009F06882329F0E091BA0BF091BB0B1995DF
:109DF0000F900F900F900F90DF91CF911F910F91C7
:109E0000FF90EF90DF90CF900895CF92DF92EF9286
:109E1000FF920F931F93CF93DF9300D01F92CDB784
:109E2000DEB78091BC0B9091BD0BA091BE0BB091A1
:109E3000BF0BB7FF08C01092BC0B1092BD0B109265
:109E4000BE0B1092BF0B8091C00B9091C10BA091E3
:109E5000C20BB091C30B4091BC0B5091BD0B6091F4
:109E6000BE0B7091BF0B84179507A607B70744F484
:109E70008093BC0B9093BD0BA093BE0BB093BF0B14
:109E800080913B02882379F14091BC0B5091BD0B2E
:109E90006091BE0B7091BF0B8091C40B9091C50B6C
:109EA000A091C60BB091C70B6A017B01C80ED91EE9
:109EB000EA1EFB1EC701B6010E94E3C92AE037ED86
:109EC00043E25CE30E9442CA69837A838B839C836A
:109ED000CE0101960E949162BC018091CA0B9091C3
:109EE000CB0B0E94FD9380919F061091B90B8111BD
:109EF00006C01123D1F180913B028823B1F140913A
:109F0000BC0B5091BD0B6091BE0B7091BF0B80914B
:109F1000C40B9091C50BA091C60BB091C70B6A0101
:109F20007B01C80ED91EEA1EFB1EC701B6010E94A6
:109F3000E3C92AE037ED43E25CE30E9442CAE091C4
:109F4000C80BF091C90B309721F060837183828335
:109F50009383112329F0E091BA0BF091BB0B199573
:109F600080919F0681110E94E8930F900F900F90AF
:109F70000F90DF91CF911F910F91FF90EF90DF90A5
:109F8000CF9008950F931F93CF938091BC0B909126
:109F9000BD0BA091BE0BB091BF0BB7FF08C01092D4
:109FA000BC0B1092BD0B1092BE0B1092BF0B809198
:109FB000C00B9091C10BA091C20BB091C30B40910B
:109FC000BC0B5091BD0B6091BE0B7091BF0B841701
:109FD0009507A607B70744F48093BC0B9093BD0B7D
:109FE000A093BE0BB093BF0B80913B02882331F14D
:109FF0004091BC0B5091BD0B6091BE0B7091BF0B9B
:10A000008091C40B9091C50BA091C60BB091C70B6A
:10A010008A019B01080F191F2A1F3B1FC901B801A4
:10A020000E94E3C90E9438CFCB010E947663BC0135
:10A030008091CA0B9091CB0B0E94FD9380919F065B
:10A04000C091B90B811106C0CC23C1F180913B02B4
:10A050008823A1F14091BC0B5091BD0B6091BE0BC8
:10A060007091BF0B8091C40B9091C50BA091C60B52
:10A07000B091C70B8A019B01080F191F2A1F3B1FB4
:10A08000C901B8010E94E3C9E091C80BF091C90B66
:10A09000309721F06083718382839383CC2329F0EE
:10A0A000E091BA0BF091BB0B199580919F06882324
:10A0B00029F0CF911F910F910C94E893CF911F91AC
:10A0C0000F9108958091BC0B9091BD0BA091BE0B98
:10A0D000B091BF0BB7FF08C01092BC0B1092BD0B24
:10A0E0001092BE0B1092BF0B8091C00B9091C10BD0
:10A0F000A091C20BB091C30B4091BC0B5091BD0B12
:10A100006091BE0B7091BF0B84179507A607B70728
:10A1100044F48093BC0B9093BD0BA093BE0BB09303
:10A12000BF0B80913B02882399F02091C40B3091A2
:10A13000C50B8091BC0B9091BD0B820F931F0E94A9
:10A140007663BC018091CA0B9091CB0B0E94FD936A
:10A1500080919F062091B90B811106C0222311F135
:10A1600080913B028823F1F04091C40B5091C50BC4
:10A170008091BC0B9091BD0B840F951FE091C80B93
:10A18000F091C90B309711F091838083222329F03D
:10A19000E091BA0BF091BB0B199580919F0681114C
:10A1A0000E94E89380919F0608958CCF8BDF8823CF
:10A1B00029F0E091BA0BF091BB0B199408951F930D
:10A1C000CF93DF9310929D068091BC0B9091BD0BB5
:10A1D000A091BE0BB091BF0B81309048A105B10595
:10A1E00040F01092BC0B1092BD0B1092BE0B10925F
:10A1F000BF0BC091BC0B8091590618160CF5282F87
:10A20000082E000C330B255031094C2F0C2E000C5E
:10A21000550B42175307A4F085301CF0CBEFC80F45
:10A2200001C0C0E08C2F0C2E000C990BAA0BBB0BAD
:10A230008093BC0B9093BD0BA093BE0BB093BF0B50
:10A24000C0935606D0E012E0C11109C080913B02D4
:10A250008823D9F121E041E06CE97CE015C0C130F0
:10A2600049F480913B02882381F120E041E06DE8D0
:10A270007CE00AC0C23061F480913B02882329F15E
:10A2800020E041E06DE77CE08D2F0E94D0C21DC030
:10A29000C33049F480913B028823B9F020E041E0CB
:10A2A00066E77CE0F1CFC43081F480913B028823E3
:10A2B00051F021E040E06BE67CE08D2F0E94D0C29F
:10A2C0008D2F0E9401C510933B02DF5FCF5FD53019
:10A2D00009F0BACFD0935906DF91CF911F9108951D
:10A2E0001F93CF93DF9310929D068091BC0B9091AA
:10A2F000BD0BA091BE0BB091BF0B81309048A10562
:10A30000B10540F01092BC0B1092BD0B1092BE0B29
:10A310001092BF0BC091BC0B80915A0618160CF519
:10A32000282F082E000C330B255031094C2F0C2EF2
:10A33000000C550B42175307A4F085301CF0CBEFEF
:10A34000C80F01C0C0E08C2F0C2E000C990BAA0B7B
:10A35000BB0B8093BC0B9093BD0BA093BE0BB09333
:10A36000BF0BC0935606D0E012E0C11109C0809126
:10A370003B028823D9F121E041E06FEC7CE015C07D
:10A38000C13049F480913B02882381F120E041E013
:10A3900066EC7CE00AC0C23061F480913B02882305
:10A3A00029F120E041E066EB7CE08D2F0E94D0C2D5
:10A3B0001DC0C33049F480913B028823B9F020E0EE
:10A3C00041E064EB7CE0F1CFC43081F480913B024A
:10A3D000882351F021E040E069EA7CE08D2F0E9463
:10A3E000D0C28D2F0E9401C510933B02DF5FCF5F6B
:10A3F000D53009F0BACFD0935A06DF91CF911F9193
:10A4000008951F93CF93DF9310929D068091BC0B0C
:10A410009091BD0BA091BE0BB091BF0B81309048C5
:10A42000A105B10540F01092BC0B1092BD0B10922B
:10A43000BE0B1092BF0BC091BC0B80915D0618162D
:10A440000CF5282F082E000C330B255031094C2F0A
:10A450000C2E000C550B42175307A4F085301CF04E
:10A46000CBEFC80F01C0C0E08C2F0C2E000C990B55
:10A47000AA0BBB0B8093BC0B9093BD0BA093BE0BA0
:10A48000B093BF0BC0935606D0E012E0C11109C0D3
:10A4900080913B028823D9F121E041E066E87DE02C
:10A4A00015C0C13049F480913B02882381F120E03E
:10A4B00041E066E77DE00AC0C23061F480913B0272
:10A4C000882329F120E041E065E67DE08D2F0E94A0
:10A4D000D0C21DC0C33049F480913B028823B9F03B
:10A4E00020E041E066E57DE0F1CFC43081F4809169
:10A4F0003B02882351F021E040E06BE47DE08D2FAA
:10A500000E94D0C28D2F0E9401C510933B02DF5FD5
:10A51000CF5FD53009F0BACFD0935D06DF91CF91F0
:10A520001F9108951F93CF93DF9310929D06809102
:10A53000BC0B9091BD0BA091BE0BB091BF0B8130B5
:10A540009048A105B10540F01092BC0B1092BD0BD4
:10A550001092BE0B1092BF0BC091BC0B80915E0697
:10A5600018160CF5282F082E000C330B2550310936
:10A570004C2F0C2E000C550B42175307A4F08530BE
:10A580001CF0CBEFC80F01C0C0E08C2F0C2E000CCC
:10A59000990BAA0BBB0B8093BC0B9093BD0BA093A4
:10A5A000BE0BB093BF0BC0935606D0E012E0C111B2
:10A5B00009C080913B028823D9F121E041E067EB9B
:10A5C0007DE015C0C13049F480913B02882381F1C0
:10A5D00020E041E06EEA7DE00AC0C23061F4809183
:10A5E0003B02882329F120E041E060EA7DE08D2FE5
:10A5F0000E94D0C21DC0C33049F480913B02882321
:10A60000B9F020E041E06EE97DE0F1CFC43081F4A3
:10A6100080913B02882351F021E040E063E97DE036
:10A620008D2F0E94D0C28D2F0E9401C510933B0236
:10A63000DF5FCF5FD53009F0BACFD0935E06DF91F0
:10A64000CF911F9108951F93CF93DF9310929D0692
:10A650008091BC0B9091BD0BA091BE0BB091BF0B34
:10A6600081309048A105B10540F01092BC0B1092CA
:10A67000BD0B1092BE0B1092BF0BC091BC0B809112
:10A680005F0618160CF5282F082E000C330B2550EA
:10A6900031094C2F0C2E000C550B42175307A4F018
:10A6A00085301CF0CBEFC80F01C0C0E08C2F0C2E02
:10A6B000000C990BAA0BBB0B8093BC0B9093BD0BAA
:10A6C000A093BE0BB093BF0BC0935606D0E012E030
:10A6D000C11109C080913B028823D9F121E041E0FA
:10A6E0006BEE7DE015C0C13049F480913B028823B8
:10A6F00081F120E041E062EE7DE00AC0C23061F409
:10A7000080913B02882329F120E041E061ED7DE06A
:10A710008D2F0E94D0C21DC0C33049F480913B02EE
:10A720008823B9F020E041E06FEC7DE0F1CFC43048
:10A7300081F480913B02882351F021E040E064ECF9
:10A740007DE08D2F0E94D0C28D2F0E9401C51093F5
:10A750003B02DF5FCF5FD53009F0BACFD0935F0601
:10A76000DF91CF911F9108951F93CF93DF931092A4
:10A770009D068091BC0B9091BD0BA091BE0BB0913A
:10A78000BF0B81309048A105B10540F01092BC0B81
:10A790001092BD0B1092BE0B1092BF0BC091BC0B60
:10A7A00080915C0618160CF5282F082E000C330B30
:10A7B000255031094C2F0C2E000C550B4217530716
:10A7C000A4F085301CF0CBEFC80F01C0C0E08C2F87
:10A7D0000C2E000C990BAA0BBB0B8093BC0B909317
:10A7E000BD0BA093BE0BB093BF0BC0935606D0E039
:10A7F00012E0C11109C080913B028823D9F121E008
:10A8000041E06EE37DE015C0C13049F480913B0228
:10A81000882381F120E041E06EE27DE00AC0C23091
:10A8200061F480913B02882329F120E041E061E25C
:10A830007DE08D2F0E94D0C21DC0C33049F48091AD
:10A840003B028823B9F020E041E06FE17DE0F1CFE9
:10A85000C43081F480913B02882351F021E040E034
:10A8600064E17DE08D2F0E94D0C28D2F0E9401C532
:10A8700010933B02DF5FCF5FD53009F0BACFD093A2
:10A880005C06DF91CF911F9108951F93CF93DF93C3
:10A8900010929D068091BC0B9091BD0BA091BE0BB8
:10A8A000B091BF0B81309048A105B10540F01092E6
:10A8B000BC0B1092BD0B1092BE0B1092BF0BC0913F
:10A8C000BC0B80915B0618160CF5282F082E000C87
:10A8D000330B255031094C2F0C2E000C550B421711
:10A8E0005307A4F085301CF0CBEFC80F01C0C0E0C7
:10A8F0008C2F0C2E000C990BAA0BBB0B8093BC0B5E
:10A900009093BD0BA093BE0BB093BF0BC0935606A4
:10A91000D0E012E0C11109C080913B028823D9F137
:10A9200021E041E067E07DE015C0C13049F480914D
:10A930003B02882381F120E041E068EF7CE00AC01F
:10A94000C23061F480913B02882329F120E041E08C
:10A9500069EE7CE08D2F0E94D0C21DC0C33049F447
:10A9600080913B028823B9F020E041E067EE7CE073
:10A97000F1CFC43081F480913B02882351F021E073
:10A9800040E06CED7CE08D2F0E94D0C28D2F0E94A4
:10A9900001C510933B02DF5FCF5FD53009F0BACF1E
:10A9A000D0935B06DF91CF911F910895CF93DF93F2
:10A9B00010929D068091BC0B9091BD0BA091BE0B97
:10A9C000B091BF0B81309048A105B10540F01092C5
:10A9D000BC0B1092BD0B1092BE0B1092BF0BC0911E
:10A9E000BC0B8091600618160CF5282F082E000C61
:10A9F000330B255031094C2F0C2E000C550B4217F0
:10AA00005307A4F085301CF0CBEFC80F01C0C0E0A5
:10AA10008C2F0C2E000C990BAA0BBB0B8093BC0B3C
:10AA20009093BD0BA093BE0BB093BF0BC093560683
:10AA3000D0E0C11109C080913B028823E9F021E0F8
:10AA400041E061E17EE015C0C13049F480913B02F4
:10AA5000882391F020E041E062E07EE00AC0C2304D
:10AA600059F480913B02882339F020E041E068EFFF
:10AA70007DE08D2F0E94D0C2DF5FCF5FD530C9F659
:10AA800083E080936006DF91CF910895CF92DF92AB
:10AA9000EF92FF920F931F93CF93DF9300D01F92FB
:10AAA000CDB7DEB78091BC0B9091BD0BA091BE0BD2
:10AAB000B091BF0BB7FF08C01092BC0B1092BD0B3A
:10AAC0001092BE0B1092BF0B8091C00B9091C10BE6
:10AAD000A091C20BB091C30B4091BC0B5091BD0B28
:10AAE0006091BE0B7091BF0B84179507A607B7073F
:10AAF00044F48093BC0B9093BD0BA093BE0BB0931A
:10AB0000BF0B80913B02882379F14091BC0B50919F
:10AB1000BD0B6091BE0B7091BF0B8091C40B9091E7
:10AB2000C50BA091C60BB091C70B6A017B01C80E83
:10AB3000D91EEA1EFB1EC701B6010E94E3C92AE026
:10AB400037ED43E25CE30E9442CA69837A838B83D8
:10AB50009C83CE0101960E945F60BC018091CA0B6C
:10AB60009091CB0B0E94FD9380919F061091B90BA1
:10AB7000811106C01123D1F180913B028823B1F1EC
:10AB80004091BC0B5091BD0B6091BE0B7091BF0BFF
:10AB90008091C40B9091C50BA091C60BB091C70BCF
:10ABA0006A017B01C80ED91EEA1EFB1EC701B60151
:10ABB0000E94E3C92AE037ED43E25CE30E9442CA07
:10ABC000E091C80BF091C90B309721F0608371833D
:10ABD00082839383112329F0E091BA0BF091BB0B90
:10ABE000199580919F0681110E94E89380919F069C
:10ABF0000F900F900F900F90DF91CF911F910F91B9
:10AC0000FF90EF90DF90CF9008958A30910508F083
:10AC10005FC0FC018827EE58FF4F8F4F0C94FBD08C
:10AC200081E08093980640E050E0BA018FED90E516
:10AC300008C081E08093980640E050E0BA0180E7C8
:10AC400091E50C944D9081E08093980640E050E0AF
:10AC5000BA0181E092E5F5CF81E08093980640E06B
:10AC600050E0BA0182E992E5ECCF81E0809398064A
:10AC700040E050E0BA0183E293E5E3CF81E08093C6
:10AC8000980640E050E0BA0184EB93E5DACF81E02A
:10AC90008093980640E050E0BA0185E494E5D1CF76
:10ACA00081E080939806109258061092570640E073
:10ACB00050E0BA0182E09BE7C4CF81E08093980620
:10ACC00040E050E0BA0186ED94E5BBCF0C94E293EE
:10ACD00008958F929F92AF92BF92CF92DF92EF92A0
:10ACE000FF920F931F93CF93DF931F921F92CDB7C5
:10ACF000DEB7E091710EE1114AC059016C018B0180
:10AD00007B01E40EF51E0E151F0509F440C0F60187
:10AD100080809180F80161918F016983C4016A8309
:10AD20000E9493CD6A81681729F1C4010E949BCDCE
:10AD3000C4010E9493CD99818917E1F0EFE7F9E012
:10AD400084918F010F5F1F4F882321F00E94593A91
:10AD5000F801F6CFECEEFEE084918F010F5F1F4FFC
:10AD6000882321F00E94593AF801F6CF81E08093C0
:10AD7000710E0DC0BE016F5F7F4FC5010E94287A22
:10AD8000F60180819181019691838083BCCF0F90E1
:10AD90000F90DF91CF911F910F91FF90EF90DF9077
:10ADA000CF90BF90AF909F908F9008958F929F9279
:10ADB000AF92BF92CF92DF92EF92FF920F931F93C9
:10ADC000CF93DF93CDB7DEB7C155D1090FB6F89455
:10ADD000DEBF0FBECDBF19AE1AAE1BAE1CAE80E3F8
:10ADE00090E3A0E3B0E08DAB9EABAFABB8AF2996DC
:10ADF0001FAE1EAE299784E690E027969FAF8EAFD8
:10AE000027971092710E9E01295B3F4F44E050E05E
:10AE1000BE016B5C7F4FCE018B5B9F4F5ADF279645
:10AE20008EAD9FAD2797029627969FAF8EAF27973F
:10AE300029961FAE1EAE299781E062968FAF62976A
:10AE40009E01295B3F4F41E050E0BE016F5A7F4FAA
:10AE5000CE018B5B9F4F3DDF9E01295B3F4F40E161
:10AE600050E066EF7BE0CE018B5B9F4F32DF9E01AF
:10AE7000295B3F4F40E150E067E87EE0CE018B5B0D
:10AE80009F4F27DF9E01295B3F4F40E150E067E97C
:10AE90007EE0CE018B5B9F4F1CDF9E01295B3F4F05
:10AEA00044E050E06FEA7EE0CE018B5B9F4F11DF04
:10AEB0009E01295B3F4F44E050E06BEA7EE0CE010B
:10AEC0008B5B9F4F06DF9E01295B3F4F44E050E0C4
:10AED00067EA7EE0CE018B5B9F4FFBDE9E01295B24
:10AEE0003F4F44E050E063E87EE0CE018B5B9F4F34
:10AEF000F0DE9E01295B3F4F44E050E06FE77EE0CB
:10AF0000CE018B5B9F4FE5DE9E01295B3F4F44E006
:10AF100050E06FEB7CE0CE018B5B9F4FDADE9E0151
:10AF2000295B3F4F40E150E063EA7CE0CE018B5B60
:10AF30009F4FCFDE9E01295B3F4F4CE050E064ED18
:10AF400075E0CE018B5B9F4FC4DE80E090E0A0E215
:10AF5000B1E489AB9AABABABBCAB9E01295B3F4F75
:10AF600044E050E0BE016F5C7F4FCE018B5B9F4F92
:10AF7000B0DE61961FAE619719AE1AAE1BAE1CAE65
:10AF800083E060968FAF60972F968FAF2F979E01CB
:10AF9000295B3F4F41E050E0BE01605B7F4FCE0137
:10AFA0008B5B9F4F96DE9E01295B3F4F44E050E054
:10AFB000BE01675C7F4FCE018B5B9F4F8ADE9E0197
:10AFC000295B3F4F41E050E0BE01615B7F4FCE0106
:10AFD0008B5B9F4F7EDE9E01295B3F4F41E050E03F
:10AFE000BE01625B7F4FCE018B5B9F4F72DE1AE02A
:10AFF000115069F09E01295B3F4F44E050E0BE01D3
:10B00000675C7F4FCE018B5B9F4F63DEF1CF1DA648
:10B010001EA61FA618AA9E01295B3F4F44E050E0E0
:10B02000BE01635D7F4FCE018B5B9F4F52DE19AE39
:10B030001AAE1BAE1CAE1AE0115069F09E01295BDE
:10B040003F4F44E050E0BE01675C7F4FCE018B5B19
:10B050009F4F3FDEF1CF83E02E968FAF2E972D9638
:10B060008FAF2D9719A61AA61BA61CA61DA21EA25D
:10B070001FA218A619AE1AAE1BAE1CAE9E01295B0C
:10B080003F4F41E050E0BE01635B7F4FCE018B5BE1
:10B090009F4F1FDE9E01295B3F4F41E050E0BE0104
:10B0A000645B7F4FCE018B5B9F4F13DE9E01295B5C
:10B0B0003F4F44E050E0BE016B5D7F4FCE018B5BA4
:10B0C0009F4F07DE9E01295B3F4F44E050E0BE01E9
:10B0D000675D7F4FCE018B5B9F4FFBDD0AE010E089
:10B0E0000150110969F09E01295B3F4F44E050E097
:10B0F000BE01675C7F4FCE018B5B9F4FEADDF0CFD7
:10B100002C961FAE2C9719AE1AAE1BAE1CAE8FEF4D
:10B110002B968FAF2B979E01295B3F4F41E050E06C
:10B12000BE01655B7F4FCE018B5B9F4FD2DD9E01E1
:10B13000295B3F4F44E050E0BE01675C7F4FCE018A
:10B140008B5B9F4FC6DD9E01295B3F4F41E050E086
:10B15000BE01665B7F4FCE018B5B9F4FBADD9E01C8
:10B16000295B3F4F44E050E06DE67DE0CE018B5B14
:10B170009F4FAFDD19AE1AAE1BAE1CAE1CE01150D6
:10B180009E01295B3F4F44E050E0112341F0BE0196
:10B19000675C7F4FCE018B5B9F4F9BDDF0CF62E4FE
:10B1A00076E0CE018B5B9F4F94DD9E01295B3F4F84
:10B1B00044E050E069E67DE0CE018B5B9F4F89DD86
:10B1C0009E01295B3F4F44E050E066E476E0CE010B
:10B1D0008B5B9F4F7EDDC12C80E8D82E8BE3E82E61
:10B1E00085E4F82E812C912C90E8A92E9FE3B92EAE
:10B1F000111132C09E01295B3F4F44E050E061E3F2
:10B2000076E0CE018B5B9F4F64DD9E01295B3F4F53
:10B2100044E050E069E376E0CE018B5B9F4F59DD5F
:10B220009E01295B3F4F44E050E065E376E0CE01AC
:10B230008B5B9F4F4EDD89AE9AAEABAEBCAE9E012E
:10B24000295B3F4F44E050E0BE01675C7F4FCE0179
:10B250008B5B9F4F3EDD24C0C9AEDAAEEBAEFCAED9
:10B260009E01295B3F4F44E050E0BE01675C7F4F89
:10B27000CE018B5B9F4F2DDD19AE1AAE1BAE1CAEFF
:10B2800004E0015069F09E01295B3F4F44E050E02B
:10B29000BE01675C7F4FCE018B5B9F4F1ADDF1CF04
:10B2A0001F5F153009F0A4CF84E190E025969FAF91
:10B2B0008EAF25979E01295B3F4F42E050E0BE01D3
:10B2C0006D5B7F4FCE018B5B9F4F03DD80E090E88D
:10B2D000ABE3B5E489AF9AAFABAFBCAF14E01150AC
:10B2E00069F09E01295B3F4F44E050E0BE01675C7E
:10B2F0007F4FCE018B5B9F4FECDCF1CF80E290E083
:10B3000023969FAF8EAF23979E01295B3F4F42E06C
:10B3100050E0BE016F5B7F4FCE018B5B9F4FD9DC4E
:10B320002A961FAE2A9780E090E0A0E4B0E489A3BB
:10B330009AA3ABA3BCA380E090E0A4E3B2E48D8F1A
:10B340009E8FAF8FB8A3198E1A8E1B8E1C8E1D8AEE
:10B350001E8A1F8A188E198A1A8A1B8A1C8A80E004
:10B3600090E0A0E5B1E48D879E87AF87B88B198602
:10B370001A861B861C8680E090E0A0E0B1E48D83F5
:10B380009E83AF83B8879E01295B3F4F41E050E029
:10B39000BE01675B7F4FCE018B5B9F4F9ADC9E01A6
:10B3A000295B3F4F44E050E0BE016F5D7F4FCE010F
:10B3B0008B5B9F4F8EDC9E01295B3F4F44E050E04A
:10B3C000BE01635E7F4FCE018B5B9F4F82DC9E018F
:10B3D000295B3F4F44E050E0BE01675E7F4FCE01E6
:10B3E0008B5B9F4F76DC9E01295B3F4F44E050E032
:10B3F000BE016B5E7F4FCE018B5B9F4F6ADC9E016F
:10B40000295B3F4F44E050E0BE016F5E7F4FCE01AD
:10B410008B5B9F4F5EDC9E01295B3F4F44E050E019
:10B42000BE01635F7F4FCE018B5B9F4F52DC9E015D
:10B43000295B3F4F44E050E0BE01675F7F4FCE0184
:10B440008B5B9F4F46DC9E01295B3F4F44E050E001
:10B45000BE016B5F7F4FCE018B5B9F4F3ADC9E013D
:10B46000295B3F4F41E050E067EB7CE0CE018B5B16
:10B470009F4F2FDC11110CC08091B30C9091B40C34
:10B48000A091B50CB091B60C89AF9AAFABAFBCAF81
:10B490009E01295B3F4F44E050E0BE01675C7F4F57
:10B4A000CE018B5B9F4F15DC1F5F153019F721967E
:10B4B0001FAE1EAE21971CE0115069F09E01295B62
:10B4C0003F4F42E050E0BE01615C7F4FCE018B5B9D
:10B4D0009F4FFFDBF1CF19AE1AAE1BAE1CAE9E0123
:10B4E000295B3F4F44E050E0BE01675C7F4FCE01D7
:10B4F0008B5B9F4FEEDB9E01295B3F4F44E050E0AA
:10B50000BE01675C7F4FCE018B5B9F4FE2DB1982F0
:10B510001A821B821C8214E0115069F09E01295B83
:10B520003F4F44E050E0BE016F5F7F4FCE018B5B29
:10B530009F4FCFDBF1CF8091710E81114EC02796C6
:10B54000EEACFFAC279729968EAD9FAD29979EAFA5
:10B550008DAF84E690E027969FAF8EAF27979E0130
:10B56000295B3F4F44E050E062E073E0CE018B5B2B
:10B570009F4FAFDB9E01295B3F4F42E050E0BE0191
:10B58000635C7F4FCE018B5B9F4FA3DBEFE7F9E05E
:10B5900084918F010F5F1F4F882321F00E94593A39
:10B5A000F801F6CFB7016456710986E19FE00E9469
:10B5B00072754DAD5EAD60E070E089E09FE00E9485
:10B5C0001B75E6E0FFE084918F010F5F1F4F88231A
:10B5D00021F00E94593AF801F6CF9091710E81E066
:10B5E0008927CF5ADF4F0FB6F894DEBF0FBECDBF0D
:10B5F000DF91CF911F910F91FF90EF90DF90CF904F
:10B60000BF90AF909F908F900895AF92BF92CF92CE
:10B61000DF92EF92FF920F931F93CF93DF931F92CE
:10B62000CDB7DEB77C016B018A0159018091710EA3
:10B63000811119C0F701808191810E9493CD898386
:10B64000F60181936F01BE016F5F7F4FC5010E94BC
:10B65000287AF701408151814F5F5F4F51834083CA
:10B660000150110939F70F90DF91CF911F910F9180
:10B67000FF90EF90DF90CF90BF90AF9008950E9421
:10B680001D820E944A830E9456B480E090E00E948E
:10B69000A93781E090E00E94A93782E090E00C9405
:10B6A000A9374F925F926F927F928F929F92AF9243
:10B6B000BF92CF92EF92FF920F931F93CF93DF939E
:10B6C000CDB7DEB728970FB6F894DEBF0FBECDBF5B
:10B6D0005C014B013A0129018091BB0E83FD42C000
:10B6E00020E030E0A901F8016081718182819381BD
:10B6F0000E94DDC981110CC020E030E0A901F501F4
:10B7000060817181828193810E94DDC9882351F11A
:10B71000F0901606F11024C02091400630914106A9
:10B720008091190290911A0228173907CCF4E1E6AA
:10B73000F8E084918F010F5F1F4F882321F00E9452
:10B74000593AF801F6CFE3ECFEE084918F010F5FE8
:10B750001F4F882309F4FBC00E94593AF801F5CF26
:10B760000E94733581E080936D0680918D0C9091DD
:10B770008E0C019781F482E090E090938E0C809380
:10B780008D0C0E94FB696093970C7093980C8093CA
:10B79000990C90939A0CCC2019F080E090E035DA67
:10B7A0000E94A19A80E1E6EEFBE0A0E8B6E00190FD
:10B7B0000D928A95E1F720E030E0A901F501608162
:10B7C0007181828193810E94DDC9882309F10E94E1
:10B7D0007C37F501208131814281538160917A0665
:10B7E00070917B0680917C0690917D060E94F4CD3D
:10B7F00060937A0670937B0680937C0690937D0617
:10B8000060E070E080EF91E40E9490370E94A19A7E
:10B81000F40180809180A280B38020E030E0A90113
:10B82000C501B4010E941AD0181624F580E090E0FA
:10B83000A0EAB0E489839A83AB83BC83A501940119
:10B840006091EE0B7091EF0B8091F00B9091F10BEA
:10B850000E94F4CD6D837E838F8398879E012F5F36
:10B860003F4FAE014B5F5F4F6AEE7BE086EE9BE0A1
:10B870000E949B3680E090E0A8ECB2E489839A8332
:10B88000AB83BC839E012F5F3F4F4EEE5BE0B20166
:10B89000C3010E949B3620E030E0A901F8016081DD
:10B8A0007181828193810E94DDC9882349F1CC2076
:10B8B00031F081E090E0A9D980E00E949DB40E941F
:10B8C0007C37F801208131814281538160917A0671
:10B8D00070917B0680917C0690917D060E94F4CD4C
:10B8E00060937A0670937B0680937C0690937D0626
:10B8F00060E070E080E291E40E9490370E94A19A9B
:10B90000CC2019F082E090E080D961E08E2D0E9479
:10B91000CB3580E00E949DB40E949BB464E670E049
:10B9200080E090E019D70E94FB69DC01CB018853CD
:10B930009045AF4FBF4F8093170D9093180DA09374
:10B94000190DB0931A0D1092080CFF24F3948F2D4B
:10B9500028960FB6F894DEBF0FBECDBFDF91CF9112
:10B960001F910F91FF90EF90CF90BF90AF909F905D
:10B970008F907F906F905F904F9008954F925F925D
:10B980006F927F928F929F92AF92BF92DF92EF92CF
:10B99000FF920F931F93CF93DF93EC01FC01E054D0
:10B9A000F14FD490029719F481E08093210D7E012C
:10B9B000EE0CFF1CEE0CFF1CF701EC54F14F459010
:10B9C0005590659074906D2D0D2C000C770B880BA5
:10B9D000990B0E94E3C94B015C0120E030E040EC90
:10B9E0005FE3C301B2010E9442CAA50194010E9413
:10B9F00042CAAB01BC0100E010E09801CE010E94F8
:10BA00009D38F701E855F14F2591359145915491B5
:10BA1000C501B4010E9442CA4B015C0120E030E044
:10BA2000A9010E94DDC9882309F44BC000E010E0A1
:10BA30009801B501A4017058CE010E949D38FE0105
:10BA4000EB55F14F649161111BC0EFE7F9E0849170
:10BA50003F019FEF691A790A882321F00E94593A21
:10BA6000F301F5CFE3E8FEE084913F019FEF691A0F
:10BA7000790A882321F00E94593AF301F5CF6AE050
:10BA8000F701ED58F14F459055906590749070E036
:10BA900080E090E00E94E3C99B01AC01C301B201C8
:10BAA0000E94D0CE2B013C01A5019401C501B40137
:10BAB0000E94F4CDAB01BC0193018201CE010E9432
:10BAC0009D38C230D10509F03FC060916D0D709175
:10BAD0006E0D80916F0D9091700D4B015C01E8949B
:10BAE000B7F81D1474F4B7FAB094B7F8B094DD2425
:10BAF000D39420E030E0A9010E941AD018167CF0FF
:10BB000009C0DD24D39420E030E0A9010E94DDC902
:10BB100087FD05C0D12C81E080931D0D03C081E01D
:10BB200080931E0D00E010E09801B501A40182E0B1
:10BB300090E00E949D38DD2019F010921E0D02C089
:10BB400010921D0D1092210DFE01E95EF94F81E06A
:10BB50008083FE01EF52FA4F8083F701EF59F94FCE
:10BB60001082118212821382CE010E94A937F7013E
:10BB7000E959F14F6591759185919491E701CA5109
:10BB8000D44FF701EC5FF94F20813181428153811D
:10BB90000E94F4CD688379838A839B830E949338C3
:10BBA000F701E259F94F88819981AA81BB8180838D
:10BBB0009183A283B383DF91CF911F910F91FF9067
:10BBC000EF90DF90BF90AF909F908F907F906F909D
:10BBD0005F904F9008950F931F93CF93DF938C0145
:10BBE000EFE7F9E08491EF012196882321F00E948C
:10BBF000593AFE01F7CFB8018AE59EE00E948B75A5
:10BC000082E20E94593A8AE00E94593A81E0DF912B
:10BC1000CF911F910F9108958C01E1E6F8E0849196
:10BC2000EF012196882321F00E94593AFE01F7CFB7
:10BC3000EAE3FEE08491EF012196882321F00E943F
:10BC4000593AFE01F7CF0E9407970E944BB70E9416
:10BC50007B6761E0C80168D60E94E2938091480C3E
:10BC6000811107C081E08093480C8FE09CE00E9426
:10BC7000D76C8091110C9091120C0E947C7784E01B
:10BC80000E948FA08091100C869586951092460C8C
:10BC90008093470C66E18CE392E00E947BA0809148
:10BCA000100C86958695880F1092460C8093470C51
:10BCB0008BE29EE00E9439A18091100C86958695BA
:10BCC000982F990F890F1092460C8093470C8EE1A4
:10BCD0009EE00E9439A10E94EA768111D0CF2FEF19
:10BCE0008BE49DE1215080409040E1F700C00000CE
:10BCF000F8942FEF84E39CE0215080409040E1F7DE
:10BD000000C000000E940797A895FECFFC01E60F37
:10BD1000F11D849190E0982F88273196E4918E0F41
:10BD2000911D089581E008950E944655882329F0C9
:10BD3000E091BA0BF091BB0B199408950C94465501
:10BD40000A96FC018491089568E0E0CF66E0DECFBA
:10BD5000FC0184910895FCDF882321F0823011F0EA
:10BD600083E0089586E0089588E290E00197F1F776
:10BD700008952EE93FE0009729F0F9013197F1F796
:10BD80000197F9CF08950F93FC010150040F84A986
:10BD900096A9941718F0081728F402C0081750F055
:10BDA000041740F42150260F83A995A9961720F473
:10BDB000281720F480E007C0281720F481E0261718
:10BDC00010F0F8CF81E00F9108958F929F92AF927B
:10BDD000BF92CF92DF92EF92FF92CF93FC01C0808F
:10BDE000D180E280F38020E030E0A901C701B601F4
:10BDF0000E94DDC987FF08C0C701B601905820E046
:10BE000030E048EC52E406C020E030E048EC52E478
:10BE1000C701B6010E9442CA0E9438CF6B017C0163
:10BE2000603AF6E87F07F1E08F07910584F020EA99
:10BE300036E841E050E00E94DFD0CA01B9012AE0B3
:10BE400030E040E050E00E94DFD0605D01C060E281
:10BE50006093CE0B80E1C81687E2D806E104F104B6
:10BE600094F0C701B60120E137E240E050E00E94C3
:10BE7000DFD0CA01B9012AE030E040E050E00E9482
:10BE8000DFD0605D01C060E26093CF0BE8EECE16BC
:10BE9000E3E0DE06E104F10494F0C701B60128EE08
:10BEA00033E040E050E00E94DFD0CA01B9012AE04F
:10BEB00030E040E050E00E94DFD0605D01C060E211
:10BEC0006093D00BC701B60124E630E040E050E0BB
:10BED0000E94DFD08AE0882E912CA12CB12CCA01BF
:10BEE000B901A50194010E94DFD0605D6093D10B80
:10BEF0008EE28093D20BC701B601A50194010E9486
:10BF0000DFD0C62FCA01B901A50194010E94DFD07C
:10BF1000605D6093D30BC05DC093D40B8EEC9BE04F
:10BF2000CF91FF90EF90DF90CF90BF90AF909F9018
:10BF30008F900895CF92DF92EF92FF920F931F930D
:10BF4000CF93DF9300D01F92CDB7DEB78091BC0BAB
:10BF50009091BD0BA091BE0BB091BF0BB7FF08C075
:10BF60001092BC0B1092BD0B1092BE0B1092BF0B27
:10BF70008091C00B9091C10BA091C20BB091C30BEB
:10BF80004091BC0B5091BD0B6091BE0B7091BF0BEB
:10BF900084179507A607B70744F48093BC0B9093CA
:10BFA000BD0BA093BE0BB093BF0B80913B028823C7
:10BFB00071F14091BC0B5091BD0B6091BE0B709123
:10BFC000BF0B8091C40B9091C50BA091C60BB09193
:10BFD000C70B6A017B01C80ED91EEA1EFB1EC701F2
:10BFE000B6010E94E3C92AE037ED43E25CE30E9418
:10BFF00042CA69837A838B839C83CE010196E5DEF6
:10C00000BC018091CA0B9091CB0B0E94FD93809153
:10C010009F061091B90B811106C01123D1F18091B7
:10C020003B028823B1F14091BC0B5091BD0B609154
:10C03000BE0B7091BF0B8091C40B9091C50BA0916A
:10C04000C60BB091C70B6A017B01C80ED91EEA1E50
:10C05000FB1EC701B6010E94E3C92AE037ED43E2A7
:10C060005CE30E9442CAE091C80BF091C90B309783
:10C0700021F06083718382839383112329F0E091FF
:10C08000BA0BF091BB0B199580919F0681110E940C
:10C09000E89380919F06882329F0E091BA0BF091F4
:10C0A000BB0B19950F900F900F900F90DF91CF91D0
:10C0B0001F910F91FF90EF90DF90CF9008958F9296
:10C0C0009F92AF92BF92CF92DF92EF92FF92CF9367
:10C0D00020E030E048EC52E4FC0160817181828113
:10C0E00093810E9442CA0E9438CF6B017C0197FF66
:10C0F0000AC0F094E094D094C094C11CD11CE11CFF
:10C10000F11C8DE201C08BE28093CE0BC701B6011A
:10C1100020E137E240E050E00E94DFD08AE0882E44
:10C12000912CA12CB12CCA01B901A50194010E9446
:10C13000DFD0605D6093CF0BC701B60128EE33E01E
:10C1400040E050E00E94DFD0CA01B901A50194018E
:10C150000E94DFD0605D6093D00BC701B60124E67A
:10C1600030E040E050E00E94DFD0CA01B901A501F3
:10C1700094010E94DFD0605D6093D10B8EE28093CA
:10C18000D20BC701B601A50194010E94DFD0C62FD2
:10C19000CA01B901A50194010E94DFD0605D6093DE
:10C1A000D30BC05DC093D40B8EEC9BE0CF91FF907E
:10C1B000EF90DF90CF90BF90AF909F908F900895B9
:10C1C0008F929F92AF92BF92CF92DF92EF92FF92A7
:10C1D000FC01C080D180E280F38020E030E0A90142
:10C1E000C701B6010E94DDC987FF04C0C701B601BF
:10C1F000905802C0C701B6010E9438CF6B017C0184
:10C200006031F7E27F078105910584F020E137E294
:10C2100040E050E00E94DFD0CA01B9012AE030E0DE
:10C2200040E050E00E94DFD0605D01C060E26093BA
:10C23000D00B88EEC81683E0D806E104F10494F030
:10C24000C701B60128EE33E040E050E00E94DFD0A5
:10C25000CA01B9012AE030E040E050E00E94DFD09E
:10C26000605D01C060E26093D10BE4E6CE16D104BC
:10C27000E104F10494F0C701B60124E630E040E0A7
:10C2800050E00E94DFD0CA01B9012AE030E040E06E
:10C2900050E00E94DFD0605D01C060E26093D20B8D
:10C2A000FAE0CF16D104E104F1049CF08AE0882E74
:10C2B000912CA12CB12CC701B601A50194010E94BB
:10C2C000DFD0CA01B901A50194010E94DFD0605DF1
:10C2D00001C060E26093D30BC701B6012AE030E0F1
:10C2E00040E050E00E94DFD0605D6093D40B80EDB1
:10C2F0009BE0FF90EF90DF90CF90BF90AF909F902A
:10C300008F900895CF92DF92EF92FF920F931F9339
:10C31000CF93DF9300D01F92CDB7DEB78091BC0BD7
:10C320009091BD0BA091BE0BB091BF0BB7FF08C0A1
:10C330001092BC0B1092BD0B1092BE0B1092BF0B53
:10C340008091C00B9091C10BA091C20BB091C30B17
:10C350004091BC0B5091BD0B6091BE0B7091BF0B17
:10C3600084179507A607B70744F48093BC0B9093F6
:10C37000BD0BA093BE0BB093BF0B80913B028823F3
:10C3800071F14091BC0B5091BD0B6091BE0B70914F
:10C39000BF0B8091C40B9091C50BA091C60BB091BF
:10C3A000C70B6A017B01C80ED91EEA1EFB1EC7011E
:10C3B000B6010E94E1C920E030E048EC52E40E945E
:10C3C00042CA69837A838B839C83CE010196F8DE0F
:10C3D000BC018091CA0B9091CB0B0E94FD93809180
:10C3E0009F061091B90B811106C01123E1F18091D4
:10C3F0003B028823C1F14091BC0B5091BD0B609171
:10C40000BE0B7091BF0B8091C40B9091C50BA09196
:10C41000C60BB091C70B6A017B01C80ED91EEA1E7C
:10C42000FB1EC701B6010E94E1C920E030E048ECE4
:10C4300052E40E9442CA0E943DCFE091C80BF091A5
:10C44000C90B309721F0608371838283938311231A
:10C4500029F0E091BA0BF091BB0B199580919F06E2
:10C4600081110E94E89380919F06882329F0E09132
:10C47000BA0BF091BB0B19950F900F900F900F9086
:10C48000DF91CF911F910F91FF90EF90DF90CF90B0
:10C49000089520E030E040E251E4FC0160817181C8
:10C4A000828193810E9442CA0E9438CF9B0177FF0C
:10C4B00006C022273327261B370B8DE201C08BE2F3
:10C4C0008093CF0BC90168EE73E00E94CCD0CB0102
:10C4D000EAE0F0E0BF010E94CCD0805D8093D00BF9
:10C4E000C90164E670E00E94CCD0CB01BF010E947C
:10C4F000CCD0805D8093D10BC901BF010E94CCD00C
:10C50000282FCB01BF010E94CCD0805D8093D20B3D
:10C510008EE28093D30B205D2093D40B8FEC9BE0B5
:10C5200008958F929F92AF92BF92CF92DF92EF9237
:10C53000FF92CF9320E030E048EC52E4FC016081B0
:10C540007181828193810E9442CA0E9438CF6B011F
:10C550007C0197FD10C020E137E240E050E00E94EE
:10C56000DFD0CA01B9012AE030E040E050E00E948B
:10C57000DFD0605D09C0F094E094D094C094C11CF9
:10C58000D11CE11CF11C6DE26093CF0BC701B60119
:10C5900028EE33E040E050E00E94DFD08AE0882EB1
:10C5A000912CA12CB12CCA01B901A50194010E94C2
:10C5B000DFD0605D6093D00BC701B60124E630E0A8
:10C5C00040E050E00E94DFD0CA01B901A50194010A
:10C5D0000E94DFD0605D6093D10B8EE28093D20B1E
:10C5E000C701B601A50194010E94DFD0C62FCA0180
:10C5F000B901A50194010E94DFD0605D6093D30B67
:10C60000C05DC093D40B8FEC9BE0CF91FF90EF9077
:10C61000DF90CF90BF90AF909F908F900895AC0126
:10C62000952F991F9927991F29F022273327241B1B
:10C63000350B01C09A01483E5340ACF0C90168EE89
:10C6400073E00E94CCD0CB01EAE0F0E0BF010E9491
:10C65000CCD0805D8093D10BC90164E670E00E946C
:10C66000CCD0CB0112C024363105B4F0911102C0F8
:10C6700080E201C08DE28093D10BC90164E670E0D5
:10C680000E94CCD0CB01EAE0F0E0BF010E94CCD008
:10C69000805D8093D20B0EC080E28093D10B80939B
:10C6A000D20B2A30310584F091118DE28093D20BA8
:10C6B000EAE0F0E0C901BF010E94CCD0CB01BF018C
:10C6C0000E94CCD0805D05C0911102C080E201C003
:10C6D0008DE28093D30BC9016AE070E00E94CCD058
:10C6E000805D8093D40B81ED9BE008959C0197FDC4
:10C6F0000EC08436910584F064E670E00E94CCD0D0
:10C70000CB016AE070E00E94CCD0805D06C031951C
:10C71000219531098DE201C080E28093D20B2A304D
:10C72000310564F0EAE0F0E0C901BF010E94CCD01D
:10C73000CB01BF010E94CCD0805D01C080E280931C
:10C74000D30BC9016AE070E00E94CCD0805D809379
:10C75000D40B82ED9BE00895CF92DF92EF92FF928F
:10C760006B017C0183E3C816D104E104F10468F095
:10C7700082E3C81AD108E108F10862E370E080E0C2
:10C7800090E001D60E94A899EDCFC701B601FBD574
:10C79000FF90EF90DF90CF900C94A89943E952E07E
:10C7A00064E670E080E090E00E943EB44AEB52E024
:10C7B00064E670E080E090E00C943EB40F931F9329
:10C7C000CF93DF93982F862F8A01D22F692F0E9453
:10C7D00089949091430C8091CD0B891748F19091E9
:10C7E000450C8091CC0B981718F1C4E1F8018491A5
:10C7F000882331F00E940EA1C81B0F5F1F4FF6CF98
:10C80000CC2329F080E20E942477C150F9CF809197
:10C81000CD0B9AE79093460C8093470C8D2F0E9486
:10C8200025A180E2DF91CF911F910F910C94247785
:10C83000DF91CF911F910F91089588E29FE00E94B0
:10C840002F7781E08093A10608950F931F93D3D58E
:10C850000091B5061091B6062091B7063091B80642
:10C86000DC01CB01801B910BA20BB30BB7FD0CC0FD
:10C8700086B186FB992790F981E08927349B8260F5
:10C88000329B84608093B4068091B406817090914D
:10C89000B40691FD82609091B306891731F1813021
:10C8A000A9F028F0823041F0833059F01CC091305B
:10C8B00089F0923099F017C0992361F0933071F0AC
:10C8C00012C0913059F0923071F404C0992331F0C4
:10C8D000933049F49091B206915003C09091B20602
:10C8E0009F5F9093B2068093B3061F910F910895B6
:10C8F000ECE3F2E080E09191992329F0863111F088
:10C900008F5FF9CF0895982F863169F080E2E92F83
:10C910009F5F973129F0F0E0E45CFD4F8083F7CF13
:10C920001092520208950895FC0167FF03C010920F
:10C93000070C60E02091070C30E0462F062E000C1B
:10C94000550B421753077CF06093070C42E450E00C
:10C95000BF018CE392E00E944DC9CADF83E080935F
:10C960003B021092060C08952091070C21110DC076
:10C97000BC0142E450E08CE392E00E9436D1B8DF83
:10C9800083E080933B021092060C08954F925F92D1
:10C990006F927F928F929F92AF92BF92CF92DF92CF
:10C9A000EF92FF920F931F93CF93C0913602CF3F28
:10C9B000F1F021D5C0909006D0909106E0909206BB
:10C9C000F0909306DC01CB018C199D09AE09BF09DB
:10C9D000B7FD0DC020916E0C80916D0C30E090E0A1
:10C9E00001968F7099272817390709F0EEC12DDFBE
:10C9F0008091B40682FF37C08091B106811135C0A5
:10CA000081E08093B1069091A006892780939F06CC
:10CA10001092A00683E080933B021092B406EBD400
:10CA2000DC01CB018C509E4FAF4FBF4F8093B506BA
:10CA30009093B606A093B706B093B80648E853E1C2
:10CA400062E070E080E090E00E943EB4C6E0C15039
:10CA500061F08FE69CE00E94073562E070E080E0C4
:10CA600090E091D4F4CF1092B106C5D46B017C0153
:10CA70008091AD069091AE06A091AF06B091B00640
:10CA8000A7019601281B390B4A0B5B0B57FF05C00A
:10CA900080919E06882309F4E7C1D701C6018C590D
:10CAA0009F4FAF4FBF4F8093AD069093AE06A093BC
:10CAB000AF06B093B0068091B20618162CF48091A0
:10CAC000B206843074F408C08091B206992781952B
:10CAD0000CF4909504972CF480919F0681119FC0CF
:10CAE000AFC080919D06882309F472C08091B20680
:10CAF000181664F48091B206082E000C990B97FD6D
:10CB0000039695958795959587950EC08091B20669
:10CB1000082E000C990B97FD039695958795959592
:10CB200087959195819591098090990690909A06A4
:10CB3000A0909B06B0909C0681149104A104B104BE
:10CB4000D1F1BC01990F880B990B0E94E3C92B010D
:10CB50003C01C701B601681979098A099B090E943D
:10CB6000E1C99B01AC01C301B2010E94D0CE20E01B
:10CB700030E04AE754E40E9442CA4B015C0120E0E5
:10CB800030E040E253E40E941AD087FF0FC020E05B
:10CB900030E046E952E4C501B4010E941AD087FD95
:10CBA0000AC02AE030E040E050E009C024E630E06E
:10CBB00040E050E004C021E030E040E050E0C092AE
:10CBC0009906D0929A06E0929B06F0929C0604C0C9
:10CBD00021E030E040E050E0A091B2060A2E000CC7
:10CBE000BB0B0E9403D124E030E040E050E00E9403
:10CBF000DFD08091BC0B9091BD0BA091BE0BB0918A
:10CC0000BF0B820F931FA41FB51F8093BC0B909383
:10CC1000BD0BA093BE0BB093BF0B1092B206D70111
:10CC2000C6018856954CAF4FBF4F8093A90690938D
:10CC3000AA06A093AB06B093AC0681E080933B02BA
:10CC40008091390290913A028057904941F4809145
:10CC50003702882309F4DAC08150809337022FB756
:10CC6000F8948091940690919506A0919606B091C3
:10CC700097062FBF3AE0B695A795979587953A9571
:10CC8000D1F7009741E0A407B10520F08FEF9FEFA7
:10CC9000A0E0B0E09695879520913B02211105C058
:10CCA00030919E063111DCC053C0009741F0409195
:10CCB000A7065091A8064817590708F049C0809167
:10CCC0009E06811111C0223050F0243028F024300B
:10CCD00031F410923B0203C081E080933B020E943A
:10CCE000A37781E080939E0684E00E948FA081E07C
:10CCF00080932F0CE0913902F0913A02199510922D
:10CD00009F0680919E06882351F00E94EA7691E06A
:10CD1000811101C090E090939E06911187C0809090
:10CD2000A7069090A806A12CB12C65D3DC01CB01FD
:10CD30008C199D09AE09BF0988169906AA06BB067B
:10CD400038F459D36C197D097093A8066093A7062F
:10CD50008091390290913A028057904921F0809158
:10CD60009806882379F088E9C80E8AE3D81EE11C6A
:10CD7000F11CC092A906D092AA06E092AB06F092EE
:10CD8000AC060FC08091A9069091AA06A091AB06AF
:10CD9000B091AC06C81AD90AEA0AFB0AF7FE0E944B
:10CDA000E29380919E0681115FC080913B028130A9
:10CDB00049F008F459C0843008F056C081E08093EF
:10CDC0003B0252C010923B024FC024E0C202F0016D
:10CDD0001124EC55FD4F20E030E040E752E4608143
:10CDE0007181828193810E94D0CEC12C7B018C0104
:10CDF00022EF3BE04EEE5BE06AEE7BE086EE9BE0EE
:10CE00000E9474838FEF80933602F1CD8CE0809383
:10CE100037028091A7069091A80601979093A806E3
:10CE20008093A70681E080933B0219CF8090A706EC
:10CE30009090A806A12CB12CDED2DC01CB018C197C
:10CE40009D09AE09BF0988169906AA06BB0660F4BB
:10CE5000D2D26C197D097093A8066093A70604C00E
:10CE6000009709F441CF23CFCF911F910F91FF90ED
:10CE7000EF90DF90CF90BF90AF909F908F907F907A
:10CE80006F905F904F900895CF92DF92EF92FF9254
:10CE90000F931F93B0D20091A3061091A406209186
:10CEA000A5063091A6066B017C01C01AD10AE20AE0
:10CEB000F30AF7FC13C02091A20620952093A20646
:10CEC000DC01CB018A549C4FAF4FBF4F8093A30628
:10CED0009093A406A093A506B093A60681E0909136
:10CEE000A206911101C080E01F910F91FF90EF9079
:10CEF000DF90CF9008950E94A9A03E98469A3C9852
:10CF0000449A3A98429AA1DC1092B206089590E0B1
:10CF1000FC013197E231F10508F04EC08827E45852
:10CF2000FF4F8F4F0C94FBD0809180008F7703C010
:10CF3000809180008F7D8093800008958091800093
:10CF4000877FF9CF84B58F7702C084B58F7D84BD8C
:10CF500008958091B0008F7703C08091B0008F7DDD
:10CF60008093B0000895809190008F7707C08091E2
:10CF700090008F7D03C080919000877F8093900008
:10CF800008958091A0008F7707C08091A0008F7DC9
:10CF900003C08091A000877F8093A00008958091B6
:10CFA00020018F7707C0809120018F7D03C0809181
:10CFB0002001877F8093200108953FB7F8948091E6
:10CFC000BE069091BF06A091C006B091C10626B5DD
:10CFD000A89B05C02F3F19F00196A11DB11D3FBFB1
:10CFE000BA2FA92F982F8827820F911DA11DB11D3F
:10CFF000BC01CD0142E0660F771F881F991F4A953B
:10D00000D1F7089508950895FC01A681B781828122
:10D01000481B8581483018F0A80FB11D4770382F84
:10D02000369536953695562F577080E890E002C0B9
:10D03000959587955A95E2F7439F402D1124669563
:10D0400066956695E62FF0E0E40FF11DEA0FFB1FF1
:10D050003081222311F0832B02C0809583238083AB
:10D060000895FB014181DC0112962C911297421721
:10D0700060F013962C911397241738F06081159661
:10D080002C91621710F42481BFCF0895FC01808198
:10D090009281980F92832181921760F494819F5F0F
:10D0A00094839381890F821710F08FEF820F83830F
:10D0B00081E0089580E00895FC0112828081815012
:10D0C00083831482089580E008950B96FC01849177
:10D0D0000895CF93DF93282F30E0F901EE5DF54EF0
:10D0E0008491F901E452F64ED491F901EA56F64ED4
:10D0F000C491CC2389F081110ADFEC2FF0E0EE0F10
:10D10000FF1FE458F64EA591B491EC91ED2381E018
:10D1100090E021F480E002C080E090E0DF91CF91C8
:10D1200008951F93CF93DF93282F30E0F901EE5D30
:10D13000F54E8491F901E452F64ED491F901EA5684
:10D14000F64EC491CC23C1F0162F8111E0DEEC2FF6
:10D15000F0E0EE0FFF1FEE59F64EA591B4918FB798
:10D16000F894111105C09C91ED2FE095E92302C0C0
:10D17000EC91ED2BEC938FBFDF91CF911F91089530
:10D18000CF93DF9390E0FC01E452F64E2491FC0132
:10D19000EA56F64E8491882361F190E0880F991F3A
:10D1A000FC01E85BF64EC591D491FC01EE59F64EB8
:10D1B000A591B491611109C09FB7F8948881209519
:10D1C00082238883EC912E230BC0623061F49FB7D9
:10D1D000F8943881822F809583238883EC912E2BBD
:10D1E0002C939FBF06C08FB7F894E8812E2B28831D
:10D1F0008FBFDF91CF9108951F93CF93DF93182FA7
:10D20000EB0161E0BDDF209711F460E004C0CF3F87
:10D21000D10531F461E0812FDF91CF911F9181CF52
:10D22000E12FF0E0EE5DF54EE4914E2F50E0FA0173
:10D230003197E231F10508F09DC08827E257FF4F92
:10D240008F4F0C94FBD084B5806884BDC7BD97C058
:10D2500084B5806284BDC8BD92C080918000806822
:10D2600080938000D0938900C093880088C080910B
:10D270008000806280938000D0938B00C0938A00EE
:10D280007EC080918000886080938000D0938D0064
:10D29000C0938C0074C08091B00080688093B0000F
:10D2A000C093B3006CC08091B00080628093B000E6
:10D2B000C093B40064C08091900080688093900017
:10D2C000D0939900C09398005AC0809190008062DA
:10D2D00080939000D0939B00C0939A0050C080919F
:10D2E0009000886080939000D0939D00C0939C0034
:10D2F00046C08091A00080688093A0008091A0002B
:10D300008F7B8093A000D093A900C093A80037C062
:10D310008091A00080628093A000D093AB00C09366
:10D32000AA002DC08091A00088608093A000D093B7
:10D33000AD00C093AC0023C0809120018068809331
:10D340002001D0932901C093280119C080912001A8
:10D35000806280932001D0932B01C0932A010FC0DB
:10D3600080912001886080932001D0932D01C0938B
:10D370002C0105C0C038D1050CF04CCF46CFDF9151
:10D38000CF911F9108958F929F92AF92BF92CF92AB
:10D39000DF92EF92FF926B017C010FDE4B015C018B
:10D3A000C114D104E104F104E9F007DEDC01CB0192
:10D3B00088199909AA09BB09883E9340A105B105BE
:10D3C00078F321E0C21AD108E108F10888EE880E4E
:10D3D00083E0981EA11CB11CC114D104E104F10426
:10D3E00021F7DECFFF90EF90DF90CF90BF90AF900E
:10D3F0009F908F9008952FB7F8946091BA0670911E
:10D40000BB068091BC069091BD062FBF08951F9268
:10D410000F920FB60F9211242F933F938F939F93E8
:10D42000AF93BF938091BA069091BB06A091BC06C2
:10D43000B091BD063091B90623E0230F2D3720F4BB
:10D440000196A11DB11D05C026E8230F0296A11D5E
:10D45000B11D2093B9068093BA069093BB06A093A2
:10D46000BC06B093BD068091BE069091BF06A09108
:10D47000C006B091C1060196A11DB11D8093BE06E4
:10D480009093BF06A093C006B093C106BF91AF9121
:10D490009F918F913F912F910F900FBE0F901F90F2
:10D4A00018951F920F920FB60F9211240BB60F9280
:10D4B0002F933F934F935F936F937F938F939F939C
:10D4C000AF93BF93EF93FF93E0911702F09118028F
:10D4D0001995FF91EF91BF91AF919F918F917F919E
:10D4E0006F915F914F913F912F910F900BBE0F90D5
:10D4F0000FBE0F901F9018951F920F920FB60F92AC
:10D5000011240BB60F922F933F934F935F936F931A
:10D510007F938F939F93AF93BF93EF93FF93E0918C
:10D520001502F09116021995FF91EF91BF91AF91FD
:10D530009F918F917F916F915F914F913F912F912B
:10D540000F900BBE0F900FBE0F901F9018951F925B
:10D550000F920FB60F9211240BB60F922F933F9399
:10D560004F935F936F937F938F939F93AF93BF93EB
:10D57000EF93FF93E0910B02F0910C021995FF914C
:10D58000EF91BF91AF919F918F917F916F915F913B
:10D590004F913F912F910F900BBE0F900FBE0F90A8
:10D5A0001F9018951F920F920FB60F9211240BB671
:10D5B0000F922F933F934F935F936F937F938F932C
:10D5C0009F93AF93BF93EF93FF93E0910902F09184
:10D5D0000A021995FF91EF91BF91AF919F918F91A1
:10D5E0007F916F915F914F913F912F910F900BBE63
:10D5F0000F900FBE0F901F9018951F920F920FB6AD
:10D600000F9211240BB60F922F933F934F935F937A
:10D610006F937F938F939F93AF93BF93EF93FF93FA
:10D62000E0911302F09114021995FF91EF91BF91CF
:10D63000AF919F918F917F916F915F914F913F91AA
:10D640002F910F900BBE0F900FBE0F901F9018954B
:10D650001F920F920FB60F9211240BB60F922F93B9
:10D660003F934F935F936F937F938F939F93AF936A
:10D67000BF93EF93FF93E0911102F091120219957D
:10D68000FF91EF91BF91AF919F918F917F916F919A
:10D690005F914F913F912F910F900BBE0F900FBE56
:10D6A0000F901F9018951F920F920FB60F92112492
:10D6B0000BB60F922F933F934F935F936F937F938C
:10D6C0008F939F93AF93BF93EF93FF93E0910F02DC
:10D6D000F09110021995FF91EF91BF91AF919F9139
:10D6E0008F917F916F915F914F913F912F910F900B
:10D6F0000BBE0F900FBE0F901F9018951F920F92A8
:10D700000FB60F9211240BB60F922F933F934F93A6
:10D710005F936F937F938F939F93AF93BF93EF9399
:10D72000FF93E0910D02F0910E021995FF91EF9198
:10D73000BF91AF919F918F917F916F915F914F9129
:10D740003F912F910F900BBE0F900FBE0F901F9027
:10D750001895CF92DF92FF920F931F93CF93DF9391
:10D760001F921F92CDB7DEB76901DB0112960D91B2
:10D770001C911397423309F470C0B8F4453109F491
:10D7800077C0473109F487C0443109F09DC0D80102
:10D7900015962C9115971696ED91FC911797CF0140
:10D7A000820F911D820F911D5CC0463409F483C025
:10D7B000473409F484C04B3309F086C0F9018181F4
:10D7C0009381913029F0933031F4482F885004C070
:10D7D00048E0480F01C0482F21E0D80113963C9142
:10D7E000381708F420E031E0F8015281451708F4B9
:10D7F00030E051E0481708F050E0822F852B3823A5
:10D8000019F4252309F460C0D6011296FC909130DA
:10D8100051F030F0923049F0933051F42FEF09C0BD
:10D8200020E031E007C021E004C020E03FEF02C06B
:10D8300020E030E0F7FE07C0B601C8012A83398333
:10D8400010DC39812A81F6018081830F80838181F8
:10D85000820F8183FF0C71F737C0B901C80101DC69
:10D8600033C01192E817F907E1F7C80125DC2CC095
:10D87000C8010CDC882349F1F80125810680F78175
:10D88000E02DCF01820F911D820F911D1192E8179B
:10D89000F907E1F719C0D9011C92F80182811196AC
:10D8A0008C9311978581815012968C931297838166
:10D8B00013968C9309C0D80115968C9103C0D8019A
:10D8C00011968C91F601808381E00F900F90DF918B
:10D8D000CF911F910F91FF90DF90CF900895DB01C2
:10D8E000ED91FC9119948F929F92BF92CF92DF920B
:10D8F000EF92FF920F931F93CF93DF931F92CDB7B9
:10D90000DEB74C01062FF42E122F522FE62EE20E18
:10D91000BB24BA946C018CE1C80ED11C8E2D851BE2
:10D92000583078F0F40162817381848FF58E178E00
:10D93000B68E96014BE3C4015983D1DF598158500B
:10D94000EDCF812F887F080F212F277019F187E0F5
:10D950002827F40162817381048FF58E178E2F5F63
:10D9600027708FEF90E001C0880F2A95EAF7868F25
:10D970009401245E3F4F4BE3C4010F90DF91CF91A0
:10D980001F910F91FF90EF90DF90CF90BF909F90ED
:10D990008F90A5CF0F90DF91CF911F910F91FF90A6
:10D9A000EF90DF90CF90BF909F908F900895EF926F
:10D9B000FF920F931F93CF93DF931F92CDB7DEB7E4
:10D9C0008C01DC011296ED90FC901397D196ED91AD
:10D9D000FC91D29782E0199520E030E04AE0B7014F
:10D9E000C8017DDFF82ED801D196ED91FC91D29738
:10D9F00083E01995D801D196ED91FC91D29780E002
:10DA00001995FF2081F1F801628173819E012F5FDA
:10DA10003F4F46E4C80163DF8981D8018C93129699
:10DA20006D917C9113979E012F5F3F4F47E4C80192
:10DA300056DF8981F80181836281738120E030E0C3
:10DA400048E4C8014CDFD8011B968C931B979801C2
:10DA50002D5C3F4F12966D917C91139747E1C80161
:10DA60003EDF81E001C080E00F90DF91CF911F91F8
:10DA70000F91FF90EF9008952F923F925F926F92D7
:10DA80007F928F929F92AF92BF92CF92DF92EF924E
:10DA9000FF920F931F93CF93DF931F92CDB7DEB703
:10DAA0001C01C62E142FD22EDC011496ED90FC9092
:10DAB0001597C7010E94A85E082FF1018481958106
:10DAC0000E94AB5E982E013019F48FE0A82E02C0A0
:10DAD000AA24AA94D10114968D919C9115970E9425
:10DAE000A05E082FF10184819581EFDAB82ED10173
:10DAF00014968D919C9115970E94A45EB0E6BD1579
:10DB000030F4009721F0E80EF91E01E611C0F10192
:10DB1000848195810E94A65EF0E4FD1530F40097A3
:10DB200021F0E80EF91E01E403C021E1E20EF11C30
:10DB3000BD1480F4D10150961C92509753961C92BC
:10DB4000539754961C92549751961C925197529603
:10DB50001C92C6C0B01670F3892D90E0F701249195
:10DB60002F3F21F4FFEFEF1AFF0A5AC00D114FC0EB
:10DB7000D10114968D919C9115970E94A85E9701F2
:10DB80002F5F3F4FF701882311F08230E1F4849139
:10DB9000D10153968C935397F901249154962C9369
:10DBA0005497F7013396E4915096EC935097F70110
:10DBB0003496E4915196EC935197F7013596E491A0
:10DBC0005296EC9320C08491982F9F709250D1016F
:10DBD00052969C93529782958F7051968C93519741
:10DBE000F9012491822F8F7054968C93549722952B
:10DBF0002F7053962C935397F7013296E491E29548
:10DC0000EF705096EC93E114F10479F469C0F701D8
:10DC10003296E491EA219C012E0F311DE20EF31E93
:10DC20000B1509F487CF0F5F99CFF101848195819E
:10DC30000E94AB5EB82ED10153969C905397549698
:10DC4000DC90549751968C915197C80E52969C91A6
:10DC50009D0D512E591A0D2D292D452D6C2DC101CB
:10DC60000E94C35E8823C9F1C7018B0D911D5C0121
:10DC700087E0890DF82EF694F694F694D50C4101C0
:10DC80009CE1890E911C6F2C712C5D1431F15C2D7F
:10DC90008501802F8A198F15E0F4F8018491D10154
:10DCA00012966D917C9113975C965C935C975D9650
:10DCB0005C925D975F961C925F975E968C93940141
:10DCC0004BE3C10159830BDE0F5F1F4F5981585F32
:10DCD000E0CFA60CB71C5394D8CFF101808901C0C6
:10DCE00080E00F90DF91CF911F910F91FF90EF9007
:10DCF000DF90CF90BF90AF909F908F907F906F906C
:10DD00005F903F902F9008958091960B80FF03C005
:10DD100089988FEF02C0899A81E080938002809178
:10DD2000960B81FF03C08F988FEF02C08F9A81E01E
:10DD3000809381028091960B9FB782FF0AC0F8946E
:10DD400080910B01826080930B019FBF439A8FEFFC
:10DD500009C0F89480910B018D7F80930B019FBFC8
:10DD6000439881E0809382028091960B83FF03C0E9
:10DD7000169A8FEF02C0169881E08093830208956F
:10DD800090916D0C80916E0C981731F080916E0C13
:10DD90008F5F8F7080936E0C08951F920F920FB655
:10DDA0000F9211240BB60F92BF92CF92DF92EF9297
:10DDB000FF920F931F932F933F934F935F936F9314
:10DDC0007F938F939F93AF93BF93EF93FF93CF93E3
:10DDD000DF9300D01F92CDB7DEB780916E008B7FAE
:10DDE00080936E0080916F008D7F80936F00789498
:10DDF0008091990B90919A0B009769F001979093FD
:10DE00009A0B8093990B1092980B1092970BB8DF96
:10DE100088EC90E0B5C1C090970BD090980BC114DE
:10DE2000D10409F0B2C190916D0C80916E0C9817DD
:10DE300049F190916E0C0DE4909F900111242E53A6
:10DE4000394F8091940690919506A0919606B091D5
:10DE50009706F901E75BFF4F408151816281738131
:10DE6000841B950BA60BB70B809394069093950695
:10DE7000A0939606B0939706D9018C9188608C93F5
:10DE800069010BC08FB7F894109294061092950612
:10DE900010929606109297068FBFD092980BC09260
:10DEA000970BC114D10409F469C1F60152A1809104
:10DEB000960B418158130AC0242F30E0809138021C
:10DEC000082E000C990B2817390729F05093960B50
:10DED0004093380219DF1092B50B1092B60B1092D6
:10DEE000B70B1092B80BD601D7968D919C91D8970D
:10DEF0008134BCE99B0728F48132EEE49E0748F0A8
:10DF000002C080E49CE9969587959695879524E0D4
:10DF100007C08131F7E29F0730F09695879522E0A0
:10DF20002093B40B08C021E02093B40B80329105FC
:10DF300010F480E290E08C0100521109011528E0F4
:10DF40001207D8F0E12FFF27EE0FFF1FEE0FFF1F84
:10DF5000CF018859914EFC01329645915491AA27E0
:10DF6000059F9001049F210D3A1F06942A1F3A1F16
:10DF70001124FC01859194911CC098013695279538
:10DF80002C7F2859354EF90185919491F9013296EB
:10DF900065917491A80147705527649F9001659F12
:10DFA000300D749F300D112443E0369527954A9526
:10DFB000E1F7821B930B8436910580F480E4E82E10
:10DFC00083E0F82ED7018D917D01882319F00E94FE
:10DFD000593AF8CFC801D9D684E690E09093B30BB4
:10DFE0008093B20B8091B40B8093B10BF60183AD9B
:10DFF00094AD9093B00B8093AF0B8134FCE99F07F5
:10E0000028F481320EE4900748F002C080E49CE9D5
:10E01000969587959695879524E007C0813117E2FC
:10E02000910730F09695879522E02093B40B08C0B5
:10E0300021E02093B40B8032910510F480E290E04F
:10E040008C0100521109011528E01207D8F0E12FC8
:10E05000FF27EE0FFF1FEE0FFF1FCF018859914ED4
:10E06000FC01329645915491AA27059F9001049F87
:10E07000210D3A1F06942A1F3A1F1124FC01859195
:10E0800094911CC09801369527952C7F2859354EC0
:10E09000F90185919491F901329665917491A801E5
:10E0A00047705527649F9001659F300D749F300D18
:10E0B000112473E0369527957A95E1F7821B930B2F
:10E0C0008436910580F450E4E52E53E0F52ED70117
:10E0D0008D917D01882319F00E94593AF8CFC8012B
:10E0E00054D684E690E0AC0160E070E04093AB0B66
:10E0F0005093AC0B6093AD0B7093AE0B9093890073
:10E1000080938800F60182899389A489B589B695A0
:10E11000A79597958795B095A095909581959F4FD8
:10E12000AF4FBF4F8093A70B9093A80BA093A90B61
:10E13000B093AA0B8093A30B9093A40BA093A50B71
:10E14000B093A60B80939F0B9093A00BA093A10B71
:10E15000B093A20B80939B0B90939C0BA0939D0B71
:10E16000B0939E0B1092920B1092930B1092940B03
:10E170001092950B82E08093220D07C080ED97E00E
:10E18000909389008093880009C48091220D882390
:10E1900021F08091D005811134C42091B40B222349
:10E1A00009F4EEC1E091970BF091980B40919B0B15
:10E1B00050919C0B60919D0B70919E0B828193817D
:10E1C000A481B581840F951FA61FB71F80939B0B59
:10E1D00090939C0BA0939D0BB0939E0B1816190661
:10E1E0001A061B060CF4889AE091970BF091980B95
:10E1F00040919F0B5091A00B6091A10B7091A20BCD
:10E2000086819781A085B185840F951FA61FB71FB2
:10E2100080939F0B9093A00BA093A10BB093A20BA4
:10E22000181619061A061B060CF48E9AE091970B25
:10E23000F091980B4091A30B5091A40B6091A50B0A
:10E240007091A60B82859385A485B585840F951F53
:10E25000A61FB71F8093A30B9093A40BA093A50BAD
:10E26000B093A60B181619061A061B063CF58091EA
:10E27000210D8823D1F080911F0D82FF04C0809171
:10E28000820287FD05C080911E0D882309F4C1C359
:10E2900080911F0D87FF04C08091820287FD0EC010
:10E2A00080911D0D81110AC008C09FB7F89480911C
:10E2B0000B01886080930B019FBF419AE091970BFF
:10E2C000F091980B4091A70B5091A80B6091A90B6E
:10E2D0007091AA0B86859785A089B189840F951FB7
:10E2E000A61FB71F8093A70B9093A80BA093A90B11
:10E2F000B093AA0B181619061A061B060CF4149AEA
:10E3000080919B0B90919C0BA0919D0BB0919E0BCB
:10E31000181619061A061B0684F5E091970BF09162
:10E32000980B4289538964897589841B950BA60BC8
:10E33000B70B80939B0B90939C0BA0939D0BB0937A
:10E340009E0B809180024091D60B5091D70B60912B
:10E35000D80B7091D90B082E000C990BAA0BBB0B94
:10E36000840F951FA61FB71F8093D60B9093D70BD2
:10E37000A093D80BB093D90B889880919F0B909164
:10E38000A00BA091A10BB091A20B181619061A06AA
:10E390001B0684F5E091970BF091980B4289538905
:10E3A00064897589841B950BA60BB70B80939F0B13
:10E3B0009093A00BA093A10BB093A20B809181022C
:10E3C0004091DA0B5091DB0B6091DC0B7091DD0B0F
:10E3D000082E000C990BAA0BBB0B840F951FA61FD0
:10E3E000B71F8093DA0B9093DB0BA093DC0BB093F9
:10E3F000DD0B8E988091A30B9091A40BA091A50B9F
:10E40000B091A60B181619061A061B060CF056C07A
:10E41000E091970BF091980B428953896489758933
:10E42000841B950BA60BB70B8093A30B9093A40BA7
:10E43000A093A50BB093A60B809182024091DE0BB6
:10E440005091DF0B6091E00B7091E10B082E000CF6
:10E45000990BAA0BBB0B840F951FA61FB71F8093A8
:10E46000DE0B9093DF0BA093E00BB093E10B809158
:10E47000210D8823D1F080911F0D82FF04C080916F
:10E48000820287FD05C080911E0D882309F4CAC24F
:10E4900080911F0D87FF04C08091820287FD0EC00E
:10E4A00080911D0D81110AC008C09FB7F89480911A
:10E4B0000B01877F80930B019FBF41988091A70B31
:10E4C0009091A80BA091A90BB091AA0B1816190650
:10E4D0001A061B0684F5E091970BF091980B428980
:10E4E000538964897589841B950BA60BB70B8093A0
:10E4F000A70B9093A80BA093A90BB093AA0B8091A4
:10E5000083024091E20B5091E30B6091E40B709118
:10E51000E50B082E000C990BAA0BBB0B840F951F63
:10E52000A61FB71F8093E20B9093E30BA093E40B1D
:10E53000B093E50B14988091920B9091930BA0915E
:10E54000940BB091950B0196A11DB11D8093920B78
:10E550009093930BA093940BB093950B2150E09163
:10E56000970BF091980B42895389648975898417B8
:10E570009507A607B70708F412CEBB24B39401C0D1
:10E58000B12C4091920B5091930B6091940B709130
:10E59000950BE090970BF090980BF701868997897F
:10E5A000A08DB18D84179507A607B70708F4DBC0C7
:10E5B0004091AB0B5091AC0B6091AD0B7091AE0BD9
:10E5C000068D178D20A131A1AA27419FB12D529F01
:10E5D000C001629F900D619F800D911D429FB00D03
:10E5E000811D9A1F519FB00D811D9A1F609FB00D14
:10E5F000811D9A1F509FB10D8A1F9A1FB6958A1FC1
:10E600009A1F349F800D911D359F900D112423ADCD
:10E6100034AD820F931F9093B00B8093AF0B47A93B
:10E6200050AD61AD72ADA0E0B0E0481759076A0780
:10E630007B0720F45093B00B4093AF0B8091AF0B4E
:10E640009091B00B8134BCE99B0728F48132EEE451
:10E650009E0748F002C080E49CE9969587959695C0
:10E66000879524E007C08131F7E29F0730F0969547
:10E67000879522E02093B40B08C021E02093B40BCF
:10E680008032910510F480E290E08C010052110973
:10E69000011528E01207D8F0E12FFF27EE0FFF1F2A
:10E6A000EE0FFF1FCF018859914EFC013296459124
:10E6B0005491AA27059F9001049F210D3A1F0694AB
:10E6C0002A1F3A1F1124FC01859194911CC09801C6
:10E6D000369527952C7F2859354EF90185919491CF
:10E6E000F901329665917491A80147705527649F8E
:10E6F0009001659F300D749F300D1124B3E0369565
:10E700002795BA95E1F7821B930B8436910580F427
:10E71000F0E4EF2EF3E0FF2ED7018D917D018823E9
:10E7200019F00E94593AF8CFC8012FD384E690E03F
:10E7300090938900809388004091AB0B5091AC0B73
:10E740006091AD0B7091AE0B8A019B01080F191FF0
:10E75000211D311D0093AB0B1093AC0B2093AD0B1F
:10E760003093AE0BFFC04091920B5091930B609190
:10E77000940B7091950BF701828D938DA48DB58DBF
:10E7800084179507A607B70708F0E0C02091B50BDE
:10E790003091B60B4091B70B5091B80B29833A8357
:10E7A0004B835C83468D578D60A171A109811A81CD
:10E7B0002B813C81AA27059FB12D169F6001269FC2
:10E7C000D00C259FC00CD11C069FB00DC11CDA1EB9
:10E7D000159FB00DC11CDA1E249FB00DC11CDA1E9E
:10E7E000149FB10DCA1EDA1EB695CA1EDA1E709F9E
:10E7F000C00CD11C719FD00C11248091AF0B909153
:10E80000B00BFF96C816D90680F48C199D0940817B
:10E810005181628173816C01E12CF12CC416D50603
:10E82000E606F70620F4CA0102C080819181813496
:10E830001CE9910728F481322EE4920748F002C0C7
:10E8400080E49CE9969587959695879524E007C086
:10E85000813137E2930730F09695879522E0209337
:10E86000B40B08C021E02093B40B8032910510F462
:10E8700080E290E08C0100521109011548E0140774
:10E88000E8F0E12FFF27EE0FFF1FEE0FFF1FCF0174
:10E890008859914EFC01329645915491AA27059FC3
:10E8A0009001049F210D3A1F06942A1F3A1F11243C
:10E8B000FC0185919491821B930B20C0C801969511
:10E8C00087958C7F8859954EFC0125913491FC01E8
:10E8D000329665917491A80147705527649FC001D5
:10E8E000659F900D749F900D112443E09695879538
:10E8F0004A95E1F7D901A81BB90BCD0184369105E2
:10E9000080F480E4E82E83E0F82EF70181917F0106
:10E91000882319F00E94593AF8CFC80136D284E60C
:10E9200090E0909389008093880029813A814B81FF
:10E930005C81280F391F411D511D2093B50B309369
:10E94000B60B4093B70B5093B80B0CC08091B20B31
:10E950009091B30B90938900809388008091B10BC4
:10E960008093B40B209188003091890080918400BD
:10E970009091850040962817390748F480918400CB
:10E980009091850040969093890080938800BB20E9
:10E9900029F01092980B1092970BF2D9F89480916D
:10E9A000260D882321F080916E008B7F03C080911B
:10E9B0006E00846080936E0080916F00826080930F
:10E9C0006F000F900F900F900F90DF91CF91FF91FC
:10E9D000EF91BF91AF919F918F917F916F915F91D7
:10E9E0004F913F912F911F910F91FF90EF90DF90EA
:10E9F000CF90BF900F900BBE0F900FBE0F901F9047
:10EA000018950E9486BA8091220D81508093220D24
:10EA1000C4CB9FB7F89480910B01886080930B0161
:10EA20009FBF36CC9FB7F89480910B01877F80936E
:10EA30000B019FBF2DCDCF92DF92EF92FF92CF932C
:10EA4000DF936A017B01FC018491EF012196882309
:10EA500021F00E94593AFE01F7CF4AE0C701B60102
:10EA6000DF91CF91FF90EF90DF90CF900C94603AC0
:10EA7000CF92DF92EF92FF92CF93DF936A017B01F7
:10EA8000FC018491EF012196882321F00E94593ADC
:10EA9000FE01F7CF42E0C701B601DF91CF91FF90B1
:10EAA000EF90DF90CF900C94963CCF92DF92EF9254
:10EAB000FF92CF93DF936A017B01FC018491EF0108
:10EAC0002196882321F00E94593AFE01F7CF42E0B7
:10EAD000C701B601DF91CF91FF90EF90DF90CF900B
:10EAE0000C94963C0F931F93CF93DF938B01FC0103
:10EAF0008491EF012196882321F00E94593AFE016A
:10EB0000F7CFB801110F880B990BDF91CF911F91AF
:10EB10000F910C94023B0F931F93CF93DF931F929F
:10EB20001F92CDB7DEB7FC0184918F010F5F1F4F9D
:10EB3000811102C08B0108C069837A830E94593A0F
:10EB4000F80169817A81F0CFF80181918F018823E2
:10EB500019F00E94593AF8CF0F900F90DF91CF91A2
:10EB60001F910F9108954F925F926F927F928F92B3
:10EB70009F92AF92BF92CF92DF92EF92FF920F934C
:10EB80001F93CF93DF93CDB7DEB72C970FB6F894D2
:10EB9000DEBF0FBECDBF2B013C0129833A834B83DF
:10EBA0005C83ED82FE820F831887A986BA86CB86A6
:10EBB000DC8628A139A14AA15BA160E070E080E871
:10EBC0009FE30E94F3CD6B017C0129813A814B8147
:10EBD0005C810E9442CA4B015C012D813E814F81C4
:10EBE000588568A179A18AA19BA10E9442CA9B0174
:10EBF000AC01C501B4010E94F4CD4B015C01A3013D
:10EC00009201C701B6010E9442CA2B013C01298131
:10EC10003A814B815C8168A179A18AA19BA10E9464
:10EC200042CA9B01AC01C301B2010E94F4CD9B0119
:10EC3000AC01C701B6010E9442CA2B013C01A501EB
:10EC4000940168A179A18AA19BA10E9442CA9B015B
:10EC5000AC01C301B2010E94F4CD9B01AC01C7011C
:10EC6000B6010E9442CA2B013C01A5019401C701D3
:10EC7000B6010E9442CA4B015C012D813E814F8149
:10EC80005885C701B6010E9442CA6B017C012985E3
:10EC90003A854B855C8568A179A18AA19BA10E94D8
:10ECA00042CA9B01AC01C701B6010E94F4CD9B0191
:10ECB000AC0168A179A18AA19BA10E9442CA9B01D3
:10ECC000AC01C501B4010E94F4CD9B01AC0168A167
:10ECD00079A18AA19BA10E9442CA9B01AC01C301F8
:10ECE000B2010E94F4CD2C960FB6F894DEBF0FBE91
:10ECF000CDBFDF91CF911F910F91FF90EF90DF90EB
:10ED0000CF90BF90AF909F908F907F906F905F90CB
:10ED10004F9008950F931F93CF93DF93082FCBE06D
:10ED2000DCE06E817F8188A38DE189A311E01BA3C4
:10ED30008FEF8AA32BE23CE04BE38FE09CE00E9444
:10ED40006F6C6E817F8108A385E289A31BA380EE8F
:10ED50008AA32BE23CE04BE38FE09CE0DF91CF9174
:10ED60001F910F910C946F6CCF93C82F22E041E15B
:10ED7000682F8FE09CE00E94736C22E042E16C2FD0
:10ED80008FE09CE0CF910C94736CBC0180E090E02C
:10ED90004AE00E94603A8DE00E94593A8AE00C9461
:10EDA000593A80918D0C90918E0C0197029710F03A
:10EDB00080E0089510928E0C10928D0C0E94FB69D9
:10EDC0006093970C7093980C8093990C90939A0C85
:10EDD00081E008950F931F93CF93E0911D0CF09164
:10EDE0001E0C309719F08FE09CE019950091110CE2
:10EDF0001091120CE091400CF091410C82E01995B9
:10EE0000E091400CF091410C81E0199520E030E058
:10EE100045E1B8018FE09CE00E946F6CC82F882309
:10EE200041F022E43CE047E1B8018FE09CE00E9421
:10EE30006F6CE091400CF091410C80E019958C2FA3
:10EE4000CF911F910F910895E0910B0CF0910C0C54
:10EE50000190F081E02D682F8BE09CE019942091C7
:10EE6000130C3091140C2817390709F444C09093FF
:10EE7000140C8093130C009709F437C02091260CD2
:10EE8000FC01211107C03596E491E093270CFC01A9
:10EE90003C960FC0213039F43F96E491E093270C63
:10EEA000FC01709606C03D96E491E093270CFC01AE
:10EEB0003E9684918093280C8091270C082E000C9C
:10EEC000990B2091280C821B910927FD9395209185
:10EED000290C203441F0829FC001112426E0969530
:10EEE00087952A95E1F780932A0C83E698E690931C
:10EEF000250C8093240C08950F931F93CF93DF93D9
:10EF00008C01CBE0DCE0EDA9FEA982E01995EDA92A
:10EF1000FEA981E0199520E030E044E1B8018FE0DE
:10EF20009CE00E946F6C22E43CE047E1B8018FE076
:10EF30009CE00E946F6CEDA9FEA980E0DF91CF916B
:10EF40001F910F9119948091480C811107C081E0A5
:10EF50008093480C8FE09CE00E94D76C8091110C4C
:10EF60009091120CC9CF8F929F92AF92BF92CF9285
:10EF7000DF92EF92FF920F931F93CF93DF93E82ED0
:10EF8000C62FF42E5901242F220F220F220F03E146
:10EF9000462F682F8FE09CE00E94C35E882341F1DA
:10EFA0000C0F8F2C912C65011F2DDE2D1123D9F014
:10EFB000F60184916091110C7091120CD0932B0C7E
:10EFC000C0932C0C10922E0C80932D0C2BE23CE065
:10EFD0004BE38FE09CE00E946F6CFFEFCF1ADF0ADB
:10EFE0001150D85FE3CFA80CB91CCF5FC013DBCFA3
:10EFF000DF91CF911F910F91FF90EF90DF90CF9015
:10F00000BF90AF909F908F900895CF92DF92FF9224
:10F010000F931F93CF93DF931F921F92CDB7DEB74D
:10F02000F82E062FE091240CF091250C8FE09CE047
:10F0300049835A831995080F4981C42E5A81D52EC8
:10F0400010E0F60121916F01222349F0402F6F2D2E
:10F050008FE09CE00E943C6DF80E180FF2CF812FDC
:10F060000F900F90DF91CF911F910F91FF90DF9044
:10F07000CF9008952F923F924F925F926F927F921E
:10F080008F929F92AF92BF92CF92DF92EF92FF92B8
:10F090000F931F93CF93DF931F921F92CDB7DEB7CD
:10F0A0001C017A83698349015A0127013801D7FE7F
:10F0B000A9C001E010E001C08601C801880F991FB6
:10F0C000880F991F9C012556334F7901A3019201A6
:10F0D000F70160817181828193810E94DDC988235B
:10F0E000B1F0F7014082518262827382EE24E39490
:10F0F000F12C20E030E0A901C301B2010E941AD036
:10F10000181614F0E12CF12CF101F182E082F101EA
:10F110008081918182309105E9F08330910509F475
:10F1200056C0019709F085C0F801EE0FFF1FEE0FE2
:10F13000FF1FE556F34F2081318142815381C50184
:10F14000B4010E94DDC987FD74C082E090E0F10146
:10F1500091838083000F111F000F111FF801E556E6
:10F16000F34F20E030E040E251E460817181828120
:10F1700093810E94F3CD9B01AC01C501B4010E94B3
:10F180001AD087FD0FC00E94FB69DC01CB01805AB9
:10F190009541AF4FBF4FE981FA8180839183A2836C
:10F1A000B38347C00E94FB69E981FA810081118124
:10F1B00022813381DC01CB01801B910BA20BB30BAD
:10F1C000B7FD37C083E090E0F1019183808348E68A
:10F1D00052E268E772E28C2D0F900F90DF91CF9191
:10F1E0001F910F91FF90EF90DF90CF90BF90AF9065
:10F1F0009F908F907F906F905F904F903F902F9057
:10F200000C943C97F601E85FF34F8081882309F462
:10F2100053CFF10111821082F601EE0FFF1FEE0FA6
:10F22000FF1FE556F34F108211821282138286016E
:10F230006ECF0F900F90DF91CF911F910F91FF90A4
:10F24000EF90DF90CF90BF90AF909F908F907F9086
:10F250006F905F904F903F902F9008950F931F9362
:10F26000CF93DF938C01EB0190917B0C20917C0C70
:10F27000921307C08FE69CE00E9407350E94A89970
:10F28000F3CFF801A081B1814881598180917A0C36
:10F2900034E0839FF0011124ED58F34FB387A28728
:10F2A000558744879F5F90937B0C8F5F821719F07F
:10F2B00080937A0C02C010927A0CDF91CF911F914B
:10F2C0000F910895CF93DF93CDB7DEB78091070CF0
:10F2D000811112C09E01275F3F4F4F81588562E424
:10F2E00070E08CE392E00E94A5C90E94786483E0FC
:10F2F00080933B021092060CDF91CF9108950F93FB
:10F300001F9380918D0C90918E0C8130910509F4A2
:10F310005DC0029789F58091970C9091980CA0910F
:10F32000990CB0919A0C0091930C1091940C20912F
:10F33000950C3091960CBC01CD01601B710B820BBA
:10F34000930B28EE33E040E050E00E94B8CD80916E
:10F350008F0C9091900CA091910CB091920C820F17
:10F36000931FA41FB51F80938F0C9093900CA093B4
:10F37000910CB093920C18C01092930C1092940CB4
:10F380001092950C1092960C1092970C1092980C6B
:10F390001092990C10929A0C10928F0C1092900C63
:10F3A0001092910C1092920C81E090E090938E0C50
:10F3B00080938D0C0E94FB696093930C7093940C66
:10F3C0008093950C9093960C81E001C080E01F9192
:10F3D0000F910895CF92DF92EF92FF92C090F20BBF
:10F3E000D090F30BE090F40BF090F50B2091020C11
:10F3F0003091030C4091040C5091050CC701B601EB
:10F400000E9442CA0E9425D06093690C70936A0CD6
:10F4100080936B0C90936C0CC701B6010E9438CF9F
:10F420002FB7F8946093E20B7093E30B8093E40B97
:10F430009093E50B2FBF1092590C10925A0C10921A
:10F440005B0C10925C0CFF90EF90DF90CF900895D2
:10F45000FC01DB018C9120813181382798E0A901E2
:10F46000440F551F37FD06C09A019150C1F73183F3
:10F47000208308959A01B1E22B27B0E13B27F5CF15
:10F480000F93CF93C82F01E020E8482F60E08FE072
:10F490009CE00E94C35E882349F020E84C2F60E086
:10F4A0008FE09CE0CF910F910C94736CCF910F91F2
:10F4B00008958F929F92AF92BF92CF92DF92EF9278
:10F4C000FF92CF9320E030E04AE754E4FC016081F2
:10F4D0007181828193810E9442CA0E9438CF6B0160
:10F4E0007C01611571058105910561F097FF0AC0E6
:10F4F000F094E094D094C094C11CD11CE11CF11C88
:10F500008DE201C080E28093CF0BC701B60128EEE7
:10F5100033E040E050E00E94DFD08AE0882E912C5A
:10F52000A12CB12CCA01B901A50194010E94DFD020
:10F53000605D6093D00B8EE28093D10BC701B60162
:10F5400024E630E040E050E00E94DFD0CA01B9017B
:10F55000A50194010E94DFD0605D6093D20BC701CA
:10F56000B601A50194010E94DFD0C62FCA01B901DE
:10F57000A50194010E94DFD0605D6093D30BC05D54
:10F58000C093D40B8FEC9BE0CF91FF90EF90DF9076
:10F59000CF90BF90AF909F908F9008950F93CF938F
:10F5A000C82F02E022E041E1682F8FE09CE00E943A
:10F5B000C35E882321F08C2FCF910F91D5CBCF91B3
:10F5C0000F9108950F930BE020E84DE160E08FE08C
:10F5D0009CE00E94C35E882399F020E84DE160E042
:10F5E0008FE09CE00E94736C80E094DB8FE792DBFD
:10F5F00020E847E260E08FE09CE00F910C94736C90
:10F600000F910895CF92DF92EF92FF921F93CF93C5
:10F61000DF9310929D068091BC0B9091BD0BA09141
:10F62000BE0BB091BF0B81309048A105B10540F0F1
:10F630001092BC0B1092BD0B1092BE0B1092BF0B20
:10F64000C091BC0B8091BE0C1816DCF4282F082E3C
:10F65000000C330B215031094C2F0C2E000C550B94
:10F660004217530774F0CFEFC80F8C2F90E0A0E043
:10F67000B0E08093BC0B9093BD0BA093BE0BB093F6
:10F68000BF0B1092B80C80915606C81714F4C093A3
:10F69000560680915606082E000C990B04962C2FC6
:10F6A0000C2E000C330B8217930724F48CEF8C0F75
:10F6B0008093560610915606D0E081E0EE24E39444
:10F6C000F12C22E0C22ED12C111125C08823B1F0DB
:10F6D0001C16A4F08091BC0B9091BD0BA091BE0BA9
:10F6E000B091BF0B0196A11DB11D8093BC0B9093EF
:10F6F000BD0BA093BE0BB093BF0BCF5F80913B02BD
:10F70000882309F446C020E041E067EE73E28D2FC4
:10F710000E94D0C23EC01130E1F480919F06811159
:10F7200005C080913B028823A1F10BC0C130C9F70D
:10F73000D0925806C09257068091B80C882389F35E
:10F7400031C081E0C13009F080E020E24AED53E2AF
:10F750001DC01230F1F480919F06811105C0809187
:10F760003B028823B1F00BC0C230C9F7F0925806B3
:10F77000E09257068091B80C882389F313C081E08A
:10F78000C23009F080E020E24DEC53E26D2F0E9480
:10F79000DE63DF5F1F5F80E0D53009F095CF83E047
:10F7A0008093BE0CDF91CF911F91FF90EF90DF907F
:10F7B000CF9008950F931F93CF93DF9310929D06E0
:10F7C0008091BC0B9091BD0BA091BE0BB091BF0B73
:10F7D00081309048A105B10540F01092BC0B109209
:10F7E000BD0B1092BE0B1092BF0BC091BC0B809151
:10F7F000BD0C1816DCF4282F082E000C330B2150FA
:10F8000031094C2F0C2E000C550B4217530774F086
:10F81000CFEFC80F8C2F90E0A0E0B0E08093BC0B3E
:10F820009093BD0BA093BE0BB093BF0B1092B80C7E
:10F8300080915606C81714F4C09356068091560658
:10F84000082E000C990B04962C2F0C2E000C330B59
:10F850008217930724F48CEF8C0F80935606109137
:10F860005606D0E081E002E0111122C08823B1F0F9
:10F870001C16A4F08091BC0B9091BD0BA091BE0B07
:10F88000B091BF0B0196A11DB11D8093BC0B90934D
:10F89000BD0BA093BE0BB093BF0BCF5F80913B021B
:10F8A000882309F468C021E041E06EEB73E24DC0AB
:10F8B000113011F58823B1F0C230A4F48091BC0B53
:10F8C0009091BD0BA091BE0BB091BF0B0196A11DF5
:10F8D000B11D8093BC0B9093BD0BA093BE0BB09356
:10F8E000BF0BCF5F80913B02882309F444C020E026
:10F8F00040E069EA73E229C01230E9F480919F0682
:10F90000811105C080913B028823A9F109C0C23052
:10F91000C9F70E94E8938091B80C882399F333C00B
:10F9200081E0C23009F080E024E044EA53E26D2F28
:10F930000E94DE6320C0133061F480913B02882373
:10F94000D1F020E041E062EA73E28D2F0E94D0C244
:10F9500012C0143081F480913B02882351F021E0E1
:10F9600040E067E973E28D2F0E94D0C28D2F0E9484
:10F9700001C500933B02DF5F1F5F80E0D53009F0D7
:10F9800073CFD093BD0CDF91CF911F910F9108954C
:10F990002F923F924F925F926F927F928F929F929F
:10F9A000AF92BF92CF92DF92EF92FF920F931F938D
:10F9B000CF93DF9310929D068091BC0B9091BD0B6D
:10F9C000A091BE0BB091BF0B81309048A105B1054D
:10F9D00040F01092BC0B1092BD0B1092BE0B109217
:10F9E000BF0BC091BC0B8091BC0C1816DCF4282F07
:10F9F000082E000C330B215031094C2F0C2E000C1B
:10FA0000550B4217530774F0CFEFC80F8C2F90E0BF
:10FA1000A0E0B0E08093BC0B9093BD0BA093BE0B15
:10FA2000B093BF0B1092B80C80915606C81714F40F
:10FA3000C093560680915606082E000C990B04962A
:10FA40002C2F0C2E000C330B8217930724F48CEF11
:10FA50008C0F8093560610915606D0E083EB282E2B
:10FA60008CE0382E9CED892E95E0992EA12CB12C9E
:10FA700026ED422E26E0522E612C712C3FE3E32E20
:10FA80003EE4F32E46E5C42E44EBD42E11111DC0E6
:10FA900080919F06811106C080913B02882309F462
:10FAA00043C009C0C111F8CF0E94E8938091B80CFF
:10FAB000882391F3BDC081E0C11180E024E04FE8CC
:10FAC00053E26D2F0E94DE632FC0113069F58091E3
:10FAD0009F06811105C080913B02811112C024C094
:10FAE000C130C9F78091B70C8C278093B70C83E0A5
:10FAF00080933B020E9456B48091B80C882359F33E
:10FB000097C08091B70C811103C02EE733E202C089
:10FB100022E833E281E0C13009F080E001E046E80C
:10FB200053E26D2F0E9476C48091B70C882309F4AC
:10FB300077C0123009F072C080919F06811106C013
:10FB400080913B02882309F469C05AC0C230C1F7D2
:10FB500091E090939D061092990610929A06109249
:10FB60009B0610929C060E942D9023E020933B025E
:10FB700084E793E29093CB0B8093CA0B3092C90B2E
:10FB80002092C80B8092C40B9092C50BA092C60B1A
:10FB9000B092C70B4092C00B5092C10B6092C20B47
:10FBA0007092C30B20E030E04AE754E46091B30C5C
:10FBB0007091B40C8091B50C9091B60C0E9442CA21
:10FBC00020E030E84BEB54E40E94F3CD0E943DCF9F
:10FBD0006093BC0B7093BD0B8093BE0B9093BF0BD7
:10FBE000F0923A02E0923902D092BB0BC092BA0B6B
:10FBF0001092B90B8091B80C882309F4A1CF18C0DA
:10FC000083EB9CE056DC9C0181E0C23009F080E08F
:10FC100000E04AE653E26D2F0E9476C483E001C003
:10FC200082E0DF5F1F5FD53009F030CF8093BC0CDE
:10FC3000DF91CF911F910F91FF90EF90DF90CF90C8
:10FC4000BF90AF909F908F907F906F905F904F90FC
:10FC50003F902F9008951F93CF93DF9310929D06AE
:10FC60008091BC0B9091BD0BA091BE0BB091BF0BCE
:10FC700081309048A105B10540F01092BC0B109264
:10FC8000BD0B1092BE0B1092BF0BC091BC0B8091AC
:10FC9000BB0C1816DCF4282F082E000C330B215057
:10FCA00031094C2F0C2E000C550B4217530774F0E2
:10FCB000CFEFC80F8C2F90E0A0E0B0E08093BC0B9A
:10FCC0009093BD0BA093BE0BB093BF0B1092B80CDA
:10FCD00080915606C81714F4C093560680915606B4
:10FCE000082E000C990B04962C2F0C2E000C330BB5
:10FCF0008217930724F48CEF8C0F80935606109193
:10FD00005606D0E011111AC080919F06811106C0DD
:10FD100080913B02882309F48DC009C0C111F8CF3E
:10FD20000E94E8938091B80C882391F38AC081E007
:10FD3000C11180E024E042E653E279C01130E9F4D9
:10FD400080919F06811106C080913B02882309F4AF
:10FD500071C00BC0C130C1F78BE49EEA0E94BEC1E6
:10FD60008091B80C882381F36CC081E0C13009F028
:10FD700080E023E049E553E25AC01230E9F4809173
:10FD80009F06811106C080913B02882309F452C06E
:10FD90000BC0C230C1F785E59CEA0E94BEC18091CC
:10FDA000B80C882381F34DC081E0C23009F080E0B7
:10FDB00023E04CE453E23BC01330E1F480919F0612
:10FDC000811105C080913B028823A1F10BC0C33093
:10FDD000C9F78DE690E80E94BEC18091B80C8823D7
:10FDE00089F32FC081E0C33009F080E023E047E4CD
:10FDF00053E21DC01430F1F480919F06811105C0BB
:10FE000080913B028823B1F00BC0C430C9F785E272
:10FE10009FE70E94BEC18091B80C882389F311C06E
:10FE200081E0C43009F080E023E04EE353E26D2F1F
:10FE30000E94DE63DF5F1F5FD53009F063CFD09390
:10FE4000BB0CDF91CF911F910895FF920F931F93E9
:10FE5000CF93DF9310929D068091BC0B9091BD0BC8
:10FE6000A091BE0BB091BF0B81309048A105B105A8
:10FE700040F01092BC0B1092BD0B1092BE0B109272
:10FE8000BF0BC091BC0B8091BA0C1816DCF4282F64
:10FE9000082E000C330B215031094C2F0C2E000C76
:10FEA000550B4217530774F0CFEFC80F8C2F90E01B
:10FEB000A0E0B0E08093BC0B9093BD0BA093BE0B71
:10FEC000B093BF0B1092B80C80915606C81714F46B
:10FED000C093560680915606082E000C990B049686
:10FEE0002C2F0C2E000C330B8217930724F48CEF6D
:10FEF0008C0F8093560610915606D0E0FF24F394A1
:10FF000011111DC080919F06811106C080913B0296
:10FF1000882309F4D5C009C0C111F8CF0E94E89325
:10FF20008091B80C882391F3D2C081E0C11180E0A8
:10FF300024E047E353E26D2F0E94DE63C1C011301D
:10FF400071F580919F06811106C080913B02882344
:10FF500009F4B6C017C0C130C1F7C0939D06109216
:10FF6000990610929A0610929B0610929C0666EFD4
:10FF70007BE08DE293E20E94A1C38091B80C8823BC
:10FF800021F3A5C086EF9BE00E94E55E9C0181E025
:10FF9000C13009F080E000E043E253E28EC012304D
:10FFA00071F580919F06811106C080913B028823E4
:10FFB00009F486C017C0C230C1F7F0929D061092B6
:10FFC000990610929A0610929B0610929C066AEF70
:10FFD0007BE089E193E20E94A1C38091B80C882361
:10FFE00021F375C08AEF9BE00E94E55E9C0181E0F1
:10FFF000C23009F080E000E04FE053E25EC0133011
:020000021000EC
:1000000071F580919F06811106C080913B02882383
:1000100009F456C017C0C330C1F7F0929D06109284
:10002000990610929A0610929B0610929C066EEF0B
:100030007BE085E093E20E94A1C38091B80C882305
:1000400021F345C08EEF9BE00E94E55E9C0181E0BC
:10005000C33009F080E000E04BEF52E22EC01430D4
:1000600079F580919F06811105C080913B0288231C
:1000700039F117C0C430C9F7F0929D061092990665
:1000800010929A0610929B0610929C0662E07CE009
:1000900081EF92E20E94A1C38091B80C882329F3DA
:1000A00016C082E09CE00E94E55E9C0181E0C430C5
:1000B00009F080E000E047EE52E26D2F0E9476C426
:1000C000DF5F1F5FD53009F01BCFD093BA0CDF91F3
:1000D000CF911F910F91FF9008952F923F924F92D1
:1000E0005F926F927F928F929F92AF92BF92CF92C8
:1000F000DF92EF92FF920F931F93CF93DF931092B3
:100100009D068091BC0B9091BD0BA091BE0BB09150
:10011000BF0B81309048A105B10540F01092BC0B97
:100120001092BD0B1092BE0B1092BF0BC091BC0B76
:100130008091B90C1816DCF4282F082E000C330B14
:10014000215031094C2F0C2E000C550B4217530730
:1001500074F0CFEFC80F8C2F90E0A0E0B0E0809358
:10016000BC0B9093BD0BA093BE0BB093BF0B109232
:10017000B80C80915606C81714F4C09356068091A7
:100180005606082E000C990B04962C2F0C2E000CF2
:10019000330B8217930724F48CEF8C0F8093560651
:1001A00050905606D0E043E0442E5EED352E2224DA
:1001B000239460EBC62E62E2D62E78EBA72E72E275
:1001C000B72EE8EC8E2EE2E29E2EF0ED6F2EF2E2DC
:1001D0007F2E51101DC080919F06811106C0809115
:1001E0003B02882309F40FC109C0C111F8CF0E9456
:1001F000E8938091B80C882391F30CC181E0C11180
:1002000080E024E040EE52E26D2F0E94DE63FBC0EE
:1002100081E058123DC080919F06811106C08091F7
:100220003B02882309F4EFC016C0C130C1F7E12CAE
:1002300010E8F12E07E714E420E030E040E85FE347
:1002400063EA7CE088ED92E20E94C8BF8091B80C1E
:10025000882329F3DFC04F923F921F922F9283EAA7
:100260009CE09F938F939F928F927F926F92DF93E8
:1002700081E0C13009F080E08F930E94E6C4ADB701
:10028000BEB71C960FB6F894BEBF0FBEADBFBBC0C5
:10029000B2E05B123DC080919F06811106C0809143
:1002A0003B02882309F4AFC016C0C230C1F7E12C6D
:1002B00010E8F12E07E714E420E030E040E85FE3C7
:1002C00067EA7CE080EC92E20E94C8BF8091B80CA3
:1002D000882329F39FC04F923F921F922F9287EA63
:1002E0009CE09F938F93DF92CF92BF92AF92DF9368
:1002F00081E0C23009F080E08F930E94E6C48DB7A0
:100300009EB70C960FB6F8949EBF0FBE8DBF7BC0F4
:1003100093E0591236C080919F06811106C08091EA
:100320003B02882309F46FC01CC0C330C1F7E12C25
:1003300010E8F12E07E714E42DEC3CEC4CEC5DE307
:100340006BEA7CE088EA92E20E94D3C1AEE9BEE5A6
:10035000B0933A02A09339028091B80C8823F9F245
:1003600059C08BEA9CE00E945F609C0181E0C33031
:1003700009F080E000E040EA52E26D2F0E9476C46E
:1003800042C0B4E05B123FC080919F06811105C05E
:1003900080913B028823B9F116C0C430C9F7E12C23
:1003A00010E8F12E07E714E420E030E040E85FE3D6
:1003B0006FEA7CE088E992E20E94C8BF8091B80CA5
:1003C000882331F327C04F923F921F922F928FEADA
:1003D0009CE09F938F93A8E8B2E2BF93AF93A0E90C
:1003E000B2E2BF93AF93DF9381E0C43009F080E0C5
:1003F0008F930E94E6C48DB79EB70C960FB6F89403
:100400009EBF0FBE8DBFDF5F5394D53009F0E1CEA4
:10041000D093B90CDF91CF911F910F91FF90EF9086
:10042000DF90CF90BF90AF909F908F907F906F9014
:100430005F904F903F902F9008958F929F92AF9230
:10044000BF92CF92DF92EF92FF920F931F93CF93C1
:10045000DF9300D01F92CDB7DEB787E9882E8EE0FC
:10046000982E96EFA92E9BE0B92E07EC1CE0C12C2C
:10047000D12C7601C394F401619171918191919194
:100480004F01F50121913191419151915F012983F2
:100490003A834B835C830E94E1C929813A814B8175
:1004A0005C810E9442CA0E943DCFF8016193719322
:1004B000819391938F01C616D706E806F90610F4CA
:1004C0006B017C01F7EA8F16FEE09F06A1F66FEF45
:1004D0007FEFCB01A70196010E94B8CD2093DC0CE1
:1004E0003093DD0C4093DE0C5093DF0C0F900F9097
:1004F0000F900F90DF91CF911F910F91FF90EF9090
:10050000DF90CF90BF90AF909F908F9008952F92E3
:100510003F924F925F926F927F928F929F92AF9293
:10052000BF92CF92DF92EF92FF920F931F93CF93E0
:10053000DF9300D01F92CDB7DEB77B016A011901AE
:10054000A6EFBBE02D913D914D915C91FC01608146
:100550007181828193810E9442CA0E9425D02B0121
:100560003C010DE51CE0D8016D937D938D939C9328
:1005700013972091FA0B3091FB0B4091FC0B50919B
:10058000FD0BF70160817181828193810E9442CAD3
:100590000E9425D04B015C01D80114966D937D9388
:1005A0008D939C9317972091FE0B3091FF0B4091F8
:1005B000000C5091010CF601608171818281938160
:1005C0000E9442CA0E9425D06B017C01D801189676
:1005D0006D937D938D939C931B972091020C30918A
:1005E000030C4091040C5091050CF1016081718164
:1005F000828193810E9442CA0E9425D0D8011C9614
:100600006D937D938D939C931F9769837A838B83DE
:100610009C830E94A19A2FB7F894E6EDFBE04082FC
:1006200051826282738284829582A682B782C0865A
:10063000D186E286F38669817A818B819C81648789
:100640007587868797872FBF1092490C10924A0CA6
:1006500010924B0C10924C0C80E1EDE4FCE0DF01B9
:100660001D928A95E9F70F900F900F900F90DF91F0
:10067000CF911F910F91FF90EF90DF90CF90BF909F
:10068000AF909F908F907F906F905F904F903F9032
:100690002F9008950F931F93CF93DF93C6EFDBE066
:1006A00004EE15E0299139914991599160E070E08B
:1006B00080E89FE30E94D0CEF8016193719381930B
:1006C00091938F01FCE0C630DF0761F722EF3BE03A
:1006D0004EEE5BE06AEE7BE086EE9BE018DFDF919A
:1006E000CF911F910F91A9CE2F923F924F925F927F
:1006F0006F927F928F929F92AF92BF92CF92DF9232
:10070000EF92FF920F931F93CF93DF93CDB7DEB796
:10071000C557D1090FB6F894DEBF0FBECDBF3B0160
:100720004A015901EFA6FBAA0BAF21961FAF2197F3
:100730003C2C2091F60B3091F70B4091F80B509127
:10074000F90BDC016D917D918D919C910E9442CAC3
:100750000E9425D0AE966CAF7DAF8EAF9FAFAE97A7
:100760002091FA0B3091FB0B4091FC0B5091FD0B4B
:10077000F30160817181828193810E9442CA0E944B
:1007800025D0E2966CAF7DAF8EAF9FAFE297209100
:10079000FE0B3091FF0B4091000C5091010CD401E5
:1007A0006D917D918D919C910E9442CA0E9425D0AD
:1007B000E6966CAF7DAF8EAF9FAFE6972091020CAF
:1007C0003091030C4091040C5091050CF5016081AF
:1007D0007181828193810E9442CA0E9425D06A96CB
:1007E0006CAF7DAF8EAF9FAF6A9780915D0C90919B
:1007F0005E0CA0915F0CB091600CAE96CCACDDAC01
:10080000EEACFFACAE97C81AD90AEA0AFB0A80918F
:10081000610C9091620CA091630CB091640CE29613
:100820008CAC9DACAEACBFACE297881A990AAA0A10
:10083000BB0A8091650C9091660CA091670CB091F9
:10084000680CE6960CAD1DAD2EAD3FADE697081BCE
:10085000190B2A0B3B0B0FAB18AF29AF3AAF8091A6
:10086000BB0E83FF0EC06A962CAD3DAD4EAD5FADA5
:100870006A972093690C30936A0C40936B0C5093E9
:100880006C0C8091690C90916A0CA0916B0CB091EA
:100890006C0C6A964CAC5DAC6EAC7FAC6A97481A37
:1008A000590A6A0A7B0A09F495C0809116068111DB
:1008B00041C06091190270911A02072E000C880B3A
:1008C000990B0E94E3C99B01AC01609112067091E3
:1008D000130680911406909115060E94DDC987FFCA
:1008E00029C06A968CAD9DADAEADBFAD6A978093C1
:1008F000690C90936A0CA0936B0CB0936C0CEFE7AF
:10090000F9E084918F010F5F1F4F882321F00E942F
:10091000593AF801F6CFE6E1F4E284918F010F5FD6
:100920001F4F882321F00E94593AF801F6CF412C3D
:10093000512C32014BA65CA66DA67EA677FE0BC09D
:1009400000271127980104191509260937090BA753
:100950001CA72DA73EA76091020C7091030C8091FB
:10096000040C9091050C0E9438CF9B01AC01A8ECBF
:10097000B0E00E94DACD2BA53CA54DA55EA562177F
:100980007307840795074CF56A968CAD9DADAEADA7
:10099000BFAD6A978093690C90936A0CA0936B0C1F
:1009A000B0936C0CEFE7F9E084918F010F5F1F4F5C
:1009B000882321F00E94593AF801F6CFE7EFF3E2DD
:1009C00084918F010F5F1F4F882321F00E94593AB5
:1009D000F801F6CF412C512C3201D701C6018827EE
:1009E000B7FD83959927AA27BB27282EB7FE03C0FA
:1009F000E82FE2602E2E0FA918AD29AD3AAD37FFD2
:100A000003C0122D1460212E77FE03C0222D286012
:100A1000222E032D10E0C301B2010E94E3C9F801A8
:100A2000EE0FFF1FEE0FFF1FED53F34F20813181BB
:100A3000428153810E9442CA2B013C01000F111FC9
:100A4000F801E956FD4F60817181072E000C880B7B
:100A5000990B0E94E3C99B01AC01C301B2010E9442
:100A600042CA2AE037ED43E25CE30E9442CA2B010E
:100A70003C0120E030E0A9010E941AD018164CF485
:100A800020E030E040E05FE3C301B2010E94F4CD1A
:100A900008C0A301920160E070E080E09FE30E9443
:100AA000F3CD0E9438CF6CAF7DAF8EAF9FAF8091FA
:100AB0006D0C8F5F8F706F968FAF6F9780916E0CFC
:100AC0006F960FAD6F97801304C080E00E949DB4B5
:100AD000F5CFE0916D0C0E2F10E01CA70BA71DE4C5
:100AE000E19FF0011124EE53F94F108222A2D701A9
:100AF000C601F7FE07C088279927DC018C199D09DC
:100B0000AE09BF0982839383A483B5838DE40BA5CB
:100B10001CA5809FF001819FF00D1124EE53F94F29
:100B2000D501C401B7FE07C088279927DC018819C1
:100B30009909AA09BB0986839783A087B1878DE4A9
:100B40000BA51CA5809FF001819FF00D1124EE5391
:100B5000F94F8FA998ADA9ADBAADB7FF07C0B09551
:100B6000A095909581959F4FAF4FBF4F82879387F8
:100B7000A487B5878DE40BA51CA5809FF001819FFC
:100B8000F00D1124EE53F94F2CAD3DAD4EAD5FADE0
:100B900026873787408B518B4281538164817581D1
:100BA0000681178120853185041715072607370729
:100BB00014F48A019B018DE4ABA5BCA58A9FF001CA
:100BC0008B9FF00D1124EE53F94F82859385A485F8
:100BD000B58580179107A207B30764F48CAD9DAD6E
:100BE000AEADBFAD80179107A207B30764F4D9017A
:100BF000C8010DC00CAD1DAD2EAD3FAD08171907D6
:100C00002A073B0724F08CAD9DADAEADBFAD2DE402
:100C10000BA51CA5209FF001219FF00D1124EE5380
:100C2000F94F828B938BA48BB58B0697A105B105E9
:100C300010F40C941390DF01A95BBF4F80913E0626
:100C400090913F068D939C933182452B462B472BE9
:100C500009F05F988DE40BA51CA5809FF001819F92
:100C6000F00D1124EE53F94F86819781A085B1854F
:100C7000892B8A2B8B2B09F08A988DE40BA51CA558
:100C8000809FF001819FF00D1124EE53F94F828572
:100C90009385A485B585892B8A2B8B2B49F09FB72B
:100CA000F894809108018E7F809308019FBF479838
:100CB0002CAD3DAD4EAD5FAD232B242B252B71F01C
:100CC0008091DB0C882319F081508093DB0C31106C
:100CD0000EC0129880E28093DB0C09C020907F0E3A
:100CE0003090800E0091810E1091820E08C02090ED
:100CF000830E3090840E0091850E1091860E910126
:100D0000A8016FA57BA98BAD21969FAD21970E946D
:100D1000DDC987FD02C00C940B90C701B6010E948B
:100D2000E3C92091E4053091E5054091E605509135
:100D3000E7050E9442CA6FA778AB89AB9AAB698B73
:100D40007A8B8B8B9C8BC501B4010E94E3C92091E7
:100D5000E8053091E9054091EA055091EB050E94C4
:100D600042CA4B015C016D8B7E8B8F8B988F6FA974
:100D700078AD89AD9AAD0E94E3C92091EC05309120
:100D8000ED054091EE055091EF050E9442CA6B01BE
:100D90007C01698F7A8F8B8F9C8F2091F005309129
:100DA000F1054091F2055091F305C301B2010E9493
:100DB00042CA6D8F7E8F8F8F98A32DE44BA55CA5C3
:100DC000249FF001259FF00D1124EE53F94F42802E
:100DD00053806480758056E04516510461047104A7
:100DE000E4F44680578060847184A6E04A1651047A
:100DF0006104710494F44284538464847584B6E07D
:100E00004B1651046104710444F4DC01CB01BF773B
:100E100087A790ABA1ABB2AB34C02FA538A949A925
:100E20005AA9CA01B9010E9442CA2B013C01A5017D
:100E30009401C501B4010E9442CA9B01AC01C301E7
:100E4000B2010E94F4CD4B015C01A7019601C701DC
:100E5000B6010E9442CA9B01AC01C501B4010E94C7
:100E6000F4CD0E945FD02DE44BA55CA5249FF0013A
:100E7000259FF00D1124EE53F94F67A770AB81AB9E
:100E800092AB8DE4ABA5BCA58A9FF0018B9FF00DC2
:100E90001124EE53F94F27A530A941A952A960E0CA
:100EA00070E080E89FE30E94D0CE26966CAF7DAFC5
:100EB0008EAF9FAF26979B01AC01B101C8010E9484
:100EC00042CA6B017C0180916D0C90916E0C891B64
:100ED0008F702B968FAF2B97A701960160E074E27D
:100EE00084E799E40E94D0CE0E9425D04B015C019A
:100EF0002B968FAD2B978250863008F044C080919E
:100F0000BF0C9091C00CA091C10CB091C20C88167E
:100F10009906AA06BB06B8F588199909AA09BB095A
:100F2000BC01CD01660F771F881F991F2B96BFAD9F
:100F30002B970B2F10E020E030E0A90198010E94D0
:100F4000B8CDCA01B9010E94E1C90E9425D0680D3F
:100F5000791D8A1D9B1D0E94E1C99B01AC0160E0C7
:100F600074E284E799E40E94D0CE6B017C019B017E
:100F7000AC0160E074E284E799E40E94D0CE0E9464
:100F800025D04B015C012FB7F89480919406909185
:100F90009506A0919606B0919706880E991EAA1EF6
:100FA000BB1E8092940690929506A0929606B092EF
:100FB00097062FBF8DE4EBA5FCA58E9F80018F9F28
:100FC000100D11240E53194FD8019F962D913D916C
:100FD0004D915C91D297A3962CAF3DAF4EAF5FAFD2
:100FE000A397A7019601A3966CAD7DAD8EAD9FAD85
:100FF000A3970E9442CA2A966CAF7DAF8EAF9FAF77
:101000002A97F80163A374A385A396A32289338941
:10101000448955892FAB38AF49AF5AAFCA01B901DE
:101020000E94E1C96FA778AB89AB9AABA701960183
:101030000E9442CA0E94BACE0E943DCF62966CAF17
:101040007DAF8EAF9FAF6297F80167AB70AF81AF96
:1010500092AF8E010F5E1F4F22961FAF0EAF2297E9
:101060000051110966961FAF0EAF669707E81EE0A4
:101070006C961FAF0EAF6C978E010F5D1F4F1AA7B6
:1010800009A766960EAD1FAD669764961FAF0EAFAB
:101090006497212C312C10E81BAB0FE30BAF229689
:1010A000AEADBFAD22976D917D918D919D912296B0
:1010B000BFAFAEAF2297A70196010E9442CA6496C5
:1010C000EEADFFAD649761937193819391936496B4
:1010D000FFAFEEAF64974B015C01E894B7F86C96F4
:1010E000AEADBFAD6C974D905D906D907D906C9660
:1010F000BFAFAEAF6C97A3019201C501B4010E94CE
:101100001AD01816A4F4A5019401C301B2010E94DB
:10111000D0CE5B018C019B01AC01B1018BA99BADD1
:101120000E941AD018161CF415010BAB1BAF2296A7
:101130000EAD1FAD229729A53AA50217130709F096
:10114000AECF20E030E040E85FE3B1018BA99BAD7A
:101150000E94DDC987FF4BC07E0131E1E30EF11C27
:1011600066960EAD1FAD669791014BA95BADD80198
:101170006D917D918D919C910E9442CAF80161937D
:101180007193819391938F01EE15FF0569F78DE4BB
:101190002BA53CA5829F8001839F100D11240E5327
:1011A000194F91014BA95BAD2A966CAD7DAD8EAD0B
:1011B0009FAD2A970E9442CAD80193966D937D9362
:1011C0008D939C93969762966CAD7DAD8EAD9FADE1
:1011D00062970E94E1C991014BA95BAD0E9442CA8E
:1011E0000E943DCFF80167AB70AF81AF92AF2696FA
:1011F0002CAD3DAD4EAD5FAD26976FA578A989A901
:101200009AA90E9442CA6BAB7CAB8DAB9EAB8DE4BE
:101210000BA51CA5809FF001819FF00D1124EE53BA
:10122000F94F82809380A480B58081149104A10439
:10123000B10409F586819781A085B185892B8A2B18
:101240008B2BC9F482859385A485B585892B8A2B40
:101250008B2B89F42091AB0E3091AC0E4091AD0EEA
:101260005091AE0E6BA97CA98DA99EA90E9442CA7D
:101270000E94BACE27C22CAD3DAD4EAD5FAD232B43
:10128000242B252B49F06091AF0E7091B00E809108
:10129000B10E9091B20E08C06091A70E7091A80E89
:1012A0008091A90E9091AA0E2BA93CA94DA95EA9E7
:1012B0000E9442CA0E94BACE0E943DCF6B017C01BF
:1012C0008091DC0C9091DD0CA091DE0CB091DF0CD4
:1012D0000FA918AD29AD3AAD80179107A207B30742
:1012E00008F4E2C081149104A104B10441F12091F9
:1012F000C70C3091C80C4091C90C5091CA0C2C15E8
:101300003D054E055F05D8F46FA978AD89AD9AAD5E
:101310000E94A9CD2B013C01A7019601C501B40192
:101320000E94A9CD461657066806790640F4C30107
:10133000B201A50194010E94B8CD69017A018DE442
:101340000BA51CA5809FF001819FF00D1124EE5389
:10135000F94F86809780A084B18481149104A10400
:10136000B10441F12091CB0C3091CC0C4091CD0CCB
:101370005091CE0C2C153D054E055F05D8F46FA994
:1013800078AD89AD9AAD0E94A9CD2B013C01A70192
:101390009601C501B4010E94A9CD461657066806FC
:1013A000790640F4C301B201A50194010E94B8CDB1
:1013B00069017A018DE40BA51CA5809FF001819F36
:1013C000F00D1124EE53F94F82849384A484B584E4
:1013D00081149104A104B10441F12091CF0C30910A
:1013E000D00C4091D10C5091D20C2C153D054E05DE
:1013F0005F05D8F46FA978AD89AD9AAD0E94A9CDEB
:101400002B013C01A7019601C501B4010E94A9CDA1
:10141000461657066806790640F4C301B201A501D5
:1014200094010E94B8CD69017A018DE40BA51CA539
:10143000809FF001819FF00D1124EE53F94F8684B7
:101440009784A088B18881149104A104B10409F49F
:101450003DC12091D30C3091D40C4091D50C5091CA
:10146000D60C2C153D054E055F0508F02FC16FA960
:1014700078AD89AD9AAD0E94A9CD2B013C01A701A1
:101480009601C501B4010E94A9CD4616570668060B
:10149000790608F01BC1C301B201A50194010E94A5
:1014A000B8CD69017A0112C181149104A104B1047B
:1014B000A9F16091C70C7091C80C8091C90C9091F2
:1014C000CA0C6C157D058E059F0540F50E94E1C98B
:1014D0002FA538A949A95AA90E9442CA2B013C014B
:1014E000C501B4010E94E3C94B015C01C701B6010B
:1014F0000E94E1C9A50194010E9442CAA301920180
:101500000E941AD0181654F4A5019401C301B20127
:101510000E94D0CE0E943DCF6B017C018DE40BA5D3
:101520001CA5809FF001819FF00D1124EE53F94F0F
:1015300046805780608471844114510461047104B1
:10154000A9F16091CB0C7091CC0C8091CD0C909155
:10155000CE0C6C157D058E059F0540F50E94E1C9F6
:101560002FA538A949A95AA90E9442CA4B015C017A
:10157000C301B2010E94E3C92B013C01C701B601BE
:101580000E94E1C9A30192010E9442CAA5019401EF
:101590000E941AD0181654F4A3019201C501B40197
:1015A0000E94D0CE0E943DCF6B017C018DE40BA543
:1015B0001CA5809FF001819FF00D1124EE53F94F7F
:1015C0004284538464847584411451046104710419
:1015D000A9F16091CF0C7091D00C8091D10C9091B9
:1015E000D20C6C157D058E059F0540F50E94E1C962
:1015F0002FA538A949A95AA90E9442CA4B015C01EA
:10160000C301B2010E94E3C92B013C01C701B6012D
:101610000E94E1C9A30192010E9442CAA50194015E
:101620000E941AD0181654F4A3019201C501B40106
:101630000E94D0CE0E943DCF6B017C018DE40BA5B2
:101640001CA5809FF001819FF00D1124EE53F94FEE
:1016500086849784A088B18881149104A104B10480
:10166000A9F16091D30C7091D40C8091D50C90911C
:10167000D60C6C157D058E059F0540F50E94E1C9CD
:101680002FA538A949A95AA90E9442CA2B013C0199
:10169000C501B4010E94E3C94B015C01C701B60159
:1016A0000E94E1C9A50194010E9442CAA3019201CE
:1016B0000E941AD0181654F4A5019401C301B20176
:1016C0000E94D0CE0E943DCF6B017C018DE42BA502
:1016D0003CA5829F8001839F100D11240E53194F4A
:1016E000F801ED5BFF4FC082D182E282F382C70135
:1016F000B6010E94E1C96B017C012BA93CA94DA94F
:101700005EA90E94D0CE6E966CAF7DAF8EAF9FAFBC
:101710006E97D801D3966D937D938D939C93D697B6
:1017200020E030E040E85BE4C701B6010E9442CA15
:1017300020E034E244EF59E40E94D0CE0E9438CF3A
:10174000F801668F778F80A391A3F3A1FCAFD80136
:101750009496BC91BFABF801F5A1FFA7D80196966E
:10176000BC91BBAB03EA1CE0AA961FAF0EAFAA97D1
:101770002E0111E1410E511C33EA232E3CE0332EA1
:1017800066966EAC7FAC66970CAD0BAF1FA9219629
:101790001FAF21972396FFAF23972796BFAF2797B9
:1017A00010E0D3018D909D90AD90BD903D01E894E7
:1017B000B7F8F101C190D190E190F1901F01A7011C
:1017C0009601C501B4010E941AD01816E4F5112340
:1017D00079F12CAD3FA94FA55BA9C701B6010E94C5
:1017E00042CA6B017C012BAD21963FAD2197239618
:1017F0004FAD239727965FAD2797C501B4010E948F
:1018000042CAA70196010E941AD01816DCF4A5015D
:101810009401C701B6010E94D0CE6BAF21967FAF75
:10182000219723968FAF239727969FAF27970AC0BC
:10183000CBAE2196DFAE21972396EFAE2397279666
:10184000FFAE279711E06414750409F0AACF2B9618
:101850000FAD2B97023008F476C13090490C2090E0
:101860004A0C10914B0C00914C0C27E137EB41EDE9
:1018700058E3632D722D812F902F0E941AD01816D5
:101880000CF061C121E0A4962FAFA4972CAD3FA925
:101890004FA55BA9632D722D812F902F0E941AD026
:1018A0001816A4F0A4961FAEA4972CAD3FA94FA57F
:1018B0005BA9632D722D812F902F0E94D0CEA89608
:1018C0006CAF7DAF8EAF9FAFA89714C0232D322D84
:1018D000412F502F6CAD7FA98FA59BA90E94D0CE20
:1018E000A8966CAF7DAF8EAF9FAFA8973CAC2FA8EA
:1018F0001FA50BA94DE45CE064965FAF4EAF649703
:1019000080E090E0A0E8BFE32E968CAF9DAFAEAF35
:10191000BFAF2E972F961FAE2F976496AEADBFAD7B
:101920006497CD90DD90ED90FD906496BFAFAEAF23
:1019300064976696EEADFFAD669781909190A19009
:10194000B1906696FFAFEEAF6697A496FFADA497F1
:10195000FF2361F0A8962CAD3DAD4EAD5FADA897CD
:10196000C701B6010E9442CA6B017C012F962FADC0
:101970002F972223C1F02E962CAD3DAD4EAD5FAD1D
:101980002E97C701B6010E9442CA6B017C012E96B8
:101990002CAD3DAD4EAD5FAD2E97C501B4010E949B
:1019A00042CA4B015C01A5019401C701B6010E9426
:1019B0001AD020E030E0A90118162CF5C501B401B9
:1019C0000E941AD018164CF020E030E0A901C7019F
:1019D000B6010E94DDC987FF05C0A5019401C701BA
:1019E000B60124C02401350177FA709477F8709419
:1019F000A3019201C701B6010E941AD018165CF526
:101A00002601370128C0C501B4010E94DDC987FD48
:101A100009C020E030E0A901C701B6010E941AD038
:101A200018164CF4A7019601C501B4010E94F3CD2C
:101A30002B013C0110C02601370177FA709477F82A
:101A40007094A5019401C301B2010E941AD0181626
:101A500014F024013501AA96AEADBFADAA97CD9082
:101A6000DD90ED90FD90AA96BFAFAEAFAA97A7010B
:101A70009601C301B2010E941AD01816ECF4A3011A
:101A80009201C701B6010E94D0CE9B01AC012E96F7
:101A90006CAD7DAD8EAD9FAD2E970E9442CA2E9645
:101AA0006CAF7DAF8EAF9FAF2E972F96BFAD2F97A8
:101AB000BF5F2F96BFAF2F976496EEADFFAD6497D3
:101AC000ED55FC4009F029CF2F963FAD2F973323DA
:101AD00081F02E962CAD3DAD4EAD5FAD2E97632DB2
:101AE000722D812F902F0E9442CA362E272E182F3A
:101AF000092F24EA30E74DE75FE3632D722D812F34
:101B0000902F0E9442CA6B017C019B01AC01609145
:101B1000D70C7091D80C8091D90C9091DA0C0E945E
:101B20001AD018163CF5A70196016BAD21967FAD32
:101B3000219723968FAD239727969FAD27970E94D5
:101B40001AD01816BCF48DE40BA51CA5809FF001DB
:101B5000819FF00D1124EE53F94F808184608083C2
:101B60003BAC21962FAC219723961FAD2397279648
:101B70000FAD27978DE42BA53CA5829FF001839F95
:101B8000F00D1124EE53F94F832D922DA12FB02F7C
:101B900083A794A7A5A7B6A76E966CAD7DAD8EADB5
:101BA0009FAD6E9790589B01AC010E94F4CDA39617
:101BB0002CAD3DAD4EAD5FADA3970E9442CA9B01D7
:101BC000AC016BE077ED83E29BE30E94F3CD0E94D2
:101BD0005FD06B017C019B01AC01632D722D812FC5
:101BE000902F0E94DDC987FD04C03C2C2D2C1E2D9A
:101BF0000F2D8DE44BA55CA5849FF001859FF00D12
:101C00001124EE53F94F832D922DA12FB02F87A3CE
